:1000000000000120CDC10000F5C10000F7C10000D3
:10001000F9C10000FBC10000FDC1000000000000AC
:10002000000000000000000000000000FFC1000010
:1000300001C200000000000003C2000005C2000071
:1000400007C2000007C20000F9C6000007C2000096
:10005000E577000007C2000007C2000007C20000E9
:1000600007C2000007C2000007C2000007C200006C
:1000700007C2000007C2000007C2000007C200005C
:1000800007C2000045C9000007C2000007C2000007
:1000900007C2000007C2000007C2000007C200003C
:1000A00007C2000007C2000007C2000007C200002C
:1000B00007C2000007C200000000000000000000AE
:1000C00007C2000007C2000007C2000007C200000C
:1000D00007C2000007C2000007C2000000000000C5
:1000E0000000000000000000000000000000000010
:1000F0000000000000000000000000000000000000
:1001000000000000000000000000000000000000EF
:1001100000000000000000000000000000000000DF
:1001200000000000000000000000000000000000CF
:1001300000000000000000000000000000000000BF
:1001400000000000000000000000000000000000AF
:10015000000000000000000000000000000000009F
:10016000000000000000000000000000000000008F
:10017000000000000000000000000000000000007F
:10018000000000000000000000000000000000006F
:10019000000000000000000000000000000000005F
:1001A000000000000000000000000000000000004F
:1001B000000000000000000000000000000000003F
:1001C000000000000000000000000000000000002F
:1001D000000000000000000000000000000000001F
:1001E000000000000000000000000000000000000F
:1001F00000000000000000000000000000000000FF
:1002000010B5054C237833B9044B13B10448AFF350
:1002100000800123237010BD880200200000000030
:10022000C03D010008B5034B1BB103490348AFF3C0
:10023000008008BD000000008C020020C03D0100CD
:10024000154B002B08BF134B9D46A3F5803A0021A8
:100250008B460F461348144A121A0EF06CFE0F4BD1
:10026000002B00D098470E4B002B00D09847002061
:10027000002104000D000D48002802D00C48AFF307
:1002800000800EF0ABFD200029000CF071FB0EF099
:10029000F3FB00BF00000800000001200000000088
:1002A0000000000088020020540800200000000028
:1002B00000000000002070470020704700207047B9
:1002C000F0B5044685B00E46684611461F4606F056
:1002D00019FF23686A465D6A31463B462046A847B7
:1002E00005B0F0BDF0B5044685B00E46104669462F
:1002F0001F4606F017FE23686A465D6A31463B4694
:100300002046A84705B0F0BD70B590B00C46154624
:100310001E4603F0C1FD48B364B32146402268463F
:100320000FF0DDFD2F2168460FF070FD28B9234640
:1003300003224021684606F067FE402231466846A7
:100340000FF0A7FD0C480AF0CDFE78B10B4B93F9E6
:100350000030062B0CD10A4B93F9003043B901232E
:100360002A46694604480BF0F4F8012010B070BD2D
:100370000020FBE72046F9E7BC030020B003002083
:100380008803002007B5002300931A461946034846
:100390000BF052FD03B05DF804FB00BFA402002087
:1003A00007B5002300931A46194603480BF044FD95
:1003B00003B05DF804FB00BFAC02002000207047D2
:1003C00013B5002204461146684602F079FB6068C6
:1003D00001F00EF902280CD005280AD0616800222D
:1003E000684602F0D7FE0021684602F0C9FD02B05F
:1003F00010BD0020FBE7406808B510B1022101F0F4
:1004000005F9012008BD13B50022044611466846CF
:1004100002F056FB2046FF22694602F02CFE2046E1
:1004200002B010BD07B5002300931A4619460348D1
:100430000BF002FD03B05DF804FB00BFB402002026
:10044000704743683BB1B0F90A00012806D002DBCF
:100450000338012801D900207047022070470000AE
:100460002DE9FF4102AC84E8060006463C493D48C0
:100470009DF828501F460BF01FFD204602F0DCFFC0
:10048000204602F06CFC40BB204602F075FE0528B9
:1004900004D8DFE800F0152216030316054632499A
:1004A00030480BF009FD0A2229462E480BF06DFD5D
:1004B0002C480BF011FD204602F0BEFF002009E0A1
:1004C000012533680095DD6B94E806003B46304615
:1004D000A847012004B0BDE8F0812046756802F00D
:1004E000BBFD0146284601F091F8204602F0B4FD1C
:1004F000012812D002282FD01C491A480BF0DCFC2E
:10050000204602F0A9FD0A22014616480BF056FDCE
:1005100014480BF0E1FC0125C1E70021204602F060
:1005200081FC18280DDC2821204602F0EBFC7168C4
:100530000022204603F0A2FA4FF42061706801F017
:1005400031FC336801250095D3F83C8094E806001F
:100550003B463046C047BCE700230393F1E700BFAA
:1005600088240100400300209E2401009124010002
:1005700008B511B9B0F9080008BDB0F90A208A42DF
:1005800003DC0089084400B2F6E7406801F0B6F8E1
:10059000F9E7000007B5002300931A4619460348FF
:1005A0000BF04AFC03B05DF804FB00BFBC02002066
:1005B00007B5002300931A46194603480BF03CFC8C
:1005C00003B05DF804FB00BFC402002038B500236F
:1005D00083608380036804460D46002B47D0274A7A
:1005E0001268002A43D0002908BF1D462B7C03F067
:1005F0000F03062B10D1224A224829460AF0ABFAF3
:1006000008B143692371204A1E4829460AF0A3FA1B
:1006100000282DD0436963711C4A216819480AF0EB
:100620009AFA054608BB1A491A480BF045FC0A22FB
:10063000617918480BF0C2FC174916480BF03CFCD6
:100640000A22217913480BF0B9FC12480BF044FC44
:100650002B460E4A21680B480AF0B8FA0B4A21686B
:1006600008480AF078FA054608B11435A56038BD87
:1006700028680EF0E9F96071CEE700BF0C04002095
:10068000E9370100540600200531010074250100FE
:100690007725010040030020032D010010B504461A
:1006A00001601146FFF792FF204610BD41790C4AC8
:1006B000002352F82300884203D10A4A52F823004B
:1006C000704752F8230028B942F82310054A42F82F
:1006D000230070470133052BEBD10020704700BF8A
:1006E000D4020020E802002010B50A4A4079002315
:1006F00052F82340844203D1074A42F8231010BD28
:1007000052F8234014B952F82320F5E70133052BA2
:10071000EED1F4E7D4020020E8020020F0B52DED80
:10072000028B9BB00546FFF7C1FF04460CF0E2F8D0
:100730004FF0FF33014643F69822204606F00EFDA7
:10074000002800F0D68006231622697905A80AF051
:10075000C5FF372105A80AF0D1FF0022114605A8E0
:100760000BF0E6F8002108EE900A05A80BF078F9E6
:10077000624908EE100A62480BF09EFB0A22697972
:100780005F480BF01BFC5F495D480BF095FB18EED2
:10079000900A0DF09BFD022402460B460094584837
:1007A0000BF0D2FC584956480BF086FB18EE100AA5
:1007B0000DF08CFD00940B46024651480BF0C4FC32
:1007C00052494F480BF078FB4D480BF085FB504ADF
:1007D000296850480AF0BFF94F4A296807464D4832
:1007E0000AF0B9F90AAC064618EE901A204602F053
:1007F00074F994E80C004FF0FF31384606F0C8FC5D
:1008000018EE101A204602F068F994E80C004FF038
:10081000FF31304606F0BCFC404A29683D480AF0EA
:100820009AF9064600285ED0037C03F00F03042BE0
:1008300059D1F5EE408AF1EE10FA54D0B5EE408A67
:10084000F1EE10FA4FD0F4EE688AF1EE10FA4AD1C8
:10085000B4EE488AF1EE10FA45D100213C220BA8F3
:100860000A910EF068FB7169402220460FF037FBB9
:100870002F2120460FF0CAFA28B9736903224021BC
:10088000204606F0C1FB264920460FF0B0FA18EECC
:10089000900A02A906F046FB22480AF023FC40B168
:1008A000214B93F9003023B902AA21461D480AF0D2
:1008B0003BFE20460FF0E5FA1AAB1844482300F837
:1008C000413C02A918EE100A06F02CFB15480AF06C
:1008D00009FC40B1144B93F9003023B902AA214618
:1008E00010480AF021FE0CF005F801462846FFF7F3
:1008F000FBFE1BB0BDEC028BF0BD00BF70250100FC
:10090000400300207C2501008C2501009325010077
:1009100095250100540600209A2501009E2501001E
:10092000E9370100BC03002088030020F8B5044625
:1009300000680D461646002800F08880A068002850
:1009400000F084800378FF2903F0100340D1002BCE
:100950007BD0032A79D04578664967482D090BF08A
:10096000ABFA0A22294664480BF028FBA3685B789F
:1009700003F00F03AB4220D060495F480BF09CFAB4
:100980000A2261795C480BF019FB5D495A480BF06B
:1009900093FAA368584859780A2201F00F010BF026
:1009A0000DFB584954480BF087FA0A222946524851
:1009B0000BF004FB50480BF08FFA0C2D40D8DFE809
:1009C00005F00B46377577375437797B657D7F00A7
:1009D000002BCBD0002039E0A3685B7803F00F0335
:1009E000023B082B24D8DFE803F00523232B230F39
:1009F00023231900444A216844480AF0ACF8A3684C
:100A0000197801F0010119E0414A21683F480AF0D4
:100A1000A2F8A3681978C1F340010FE03D4A2168AC
:100A20003A480AF098F8A3681978C1F3800105E004
:100A30002168394A35480AF08EF80021002841D152
:100A4000A3685A7865F303025A700120F8BD334A4F
:100A500021682E480AF07FF8A2681378DF4303F07C
:100A6000010167F300031370E8E72D4A2168274866
:100A70000AF071F8A7683B7883F00202C2F34002E3
:100A8000C3F3400162F341033B70D7E7254A216875
:100A90001E480AF060F8A7683B7883F00402C2F3AE
:100AA0008002C3F3800162F38203EDE71E4AA2E7EE
:100AB0001E4AA0E71E4AA8E71E4AA6E71E4AAEE75E
:100AC0001E4AACE7A368032E5A780AD065F30302E6
:100AD0005A7006F087FCA3681A786FF304121A7034
:100AE000B3E7C2F3030161F307125A701A7842F0B8
:100AF0001002F4E7F8240100400300200531010052
:100B0000B83701001025010014250100540600200B
:100B1000132501001A2501002125010026250100C9
:100B20002B25010031250100372501003C2501005E
:100B300042250100482501004F25010055250100EF
:100B40002DE9F0435C4A95B00746884601685B484A
:100B50000AF001F85A4A39688146584809F0FBFF03
:100B60000646B9F1000F01D1002879D0554A3968FD
:100B7000524809F0F0FF544A396805464F4809F0D9
:100B8000EAFF5249044652480BF096F90A22797955
:100B90004F480BF013FA4F494D480BF08DF90A22DC
:100BA00041464B480BF0F1F949480BF095F95EB31B
:100BB000337C03F00F03042B26D14022716904A873
:100BC0000FF08DF944480AF08DFAE8B1434B93F9E0
:100BD0000030CBB92F2104A80FF018F928B9736998
:100BE0000322402104A806F00FFAB8F1000F40D00C
:100BF00025B12B7C03F00F03042B34D0384A01239A
:100C000004A935480AF0A5FCB9F1000F28D099F8DD
:100C1000103003F00F03042B22D1D9F8141004A8CC
:100C200000F0E6FE04A800F03FFEB0B1B8F1000FFE
:100C300033D025B12B7C03F00F03042B24D002AC5E
:100C400001220021204601F03BFF0123009394E89C
:100C50000600002304A801F0FFF804A800F0BEFC81
:100C600015B0BDE8F0836A691378002BCCD001235E
:100C7000C6E724B1237C03F00F03042B02D0012329
:100C8000184ABDE76269EFE769690B78002BE4D089
:100C9000002204A801F0A2FCDFE724B1237C03F0CA
:100CA0000F03042B02D002AC0222CAE761690B7861
:100CB000002BD2D04246ECE7642501005406002008
:100CC0009E2501002625010021250100692501003E
:100CD0004003002091250100BC0300208803002070
:100CE000D2290100D629010070B598B0054602ACA2
:100CF00084E80600374838490BF0DEF80A226979A3
:100D000034480BF05BF9354932480BF0D5F82046F2
:100D100002F092FB2968324A324809F01CFF94E83D
:100D20000C004FF0FF3106F033FA29682E4A2D48A7
:100D300009F011FF29682D4A06462A4809F00BFFE1
:100D4000054660B3037C03F00F03042B27D14169F0
:100D5000402208A80FF0C3F82F2108A80FF056F87A
:100D600028B96B690322402108A806F04DF9002339
:100D7000102200930DEB02014FF40073204602F0A5
:100D80005FFA1B480AF0AEF948B11A4B93F90030EC
:100D90002BB9012304AA08A915480AF0DAFBBEB151
:100DA000337C03F00F03042B12D1716908A800F003
:100DB0001FFE08A800F078FD38B10123009394E8E5
:100DC0000600002308A801F047F808A800F006FC78
:100DD00018B070BD4003002070250100912501006E
:100DE0006025010054060020642501009E250100B5
:100DF000BC0300208803002010B503788B42044612
:100E000004D14378402B01D1408810BD402321708C
:100E1000637008460BF024FE80B26080F5E70000A6
:100E2000F8B5836804460D46002B00F051810A4650
:100E3000FF21FFF77BFD637926790E3B072BC6F375
:100E400040062ED8A64A2168A64809F084FE074627
:100E500038B3037C03F00F03052B22D16179A2483C
:100E6000FFF7CAFF0022064639469E4809F06BFE8E
:100E700043699E421CDA0026A3685A7802F00F02EA
:100E8000013A0B2A56D8DFE812F01E00E3004000BA
:100E90006700E3006E00E3008C009C00A300CB0021
:100EA000DC0060790BF00CFF311A4E424E41E3E753
:100EB000012239468B4809F046FE43699E42CCBF69
:100EC00000260126D8E75F880BF014FD4FF6FF736C
:100ED00081B24FF47A72384606F040F950B3834A33
:100EE0002168804809F037FE28B12A4603212046B0
:100EF000FFF71CFD1EE07E4A21687A4809F02BFEB0
:100F00000028F2D12A460D21F1E75F880BF0F2FCB0
:100F10004FF6FF734FF4967281B2384606F01EF911
:100F200040B12A4604212046FFF700FD0BF0E2FC09
:100F3000A3685880A2681378C3F3C001B14200F0DF
:100F40000F8113F0E00F00F09480C3F342110139D8
:100F500061F347131370BBE05F880BF0CBFC4FF6D7
:100F6000FF739622D8E75F880BF0C4FC4FF6FF733F
:100F700081B24FF47A72384606F0F0F80028D9D0E2
:100F80005C4A2168574809F0E6FD10B12A4608215D
:100F9000ADE7594A2168534809F0DDFD0028F5D135
:100FA000B0E75F880BF0A6FC4FF6FF734FF4967224
:100FB00081B2384606F0D2F80028BBD02A46092173
:100FC000B1E75F880BF096FC4FF6FF739622EFE7D0
:100FD0005F880BF08FFC4FF6FF7381B24FF47A728B
:100FE000384606F0BBF80028A4D0444A21683D48A2
:100FF00009F0B1FD10B12A460B2178E7404A21687B
:10100000384809F0A8FD0028F5D13E4A2168354846
:1010100009F0A1FD00287FF475AF2A46062166E796
:101020005F880BF067FC4FF6FF734FF4967281B246
:10103000384606F093F800283FF47CAF2A460C218E
:1010400071E75F880BF056FC4FF6FF739622EEE7D0
:101050005F880BF04FFC4FF6FF7381B24FF41672AE
:10106000384606F07BF800283FF464AF2A4600219A
:101070003DE70BF03FFCA36858802279D2070BD5DF
:1010800036B3197841F008011970204601F00101CA
:10109000BDE8F840FFF754BD31462046FFF750FD4C
:1010A000A3685B7803F00F0376B3072B0BD8DFE858
:1010B00003F0040A100A0A100A132A4601212046E6
:1010C000FFF734FC20B1A3681A7866F3C3021A70E4
:1010D000F8BD2A460621F2E72A460A21EFE700BFBB
:1010E0005C25010054060020FC0200203725010089
:1010F0003C25010042250100482501004F25010043
:101100005525010031250100013B0C2BDBD801A244
:1011100052F823F049110000C71000004F110000E1
:101120004F110000C710000055110000C71000004B
:101130005B1100005B1100005B1100005B110000FF
:101140005B1100004F1100002A460221B7E72A4632
:101150000521B4E72A460721B1E72A460021AEE778
:101160000321F5E62DE9F0470168634A86B0814620
:10117000624809F0F0FC99F8051006466048FFF750
:101180003BFE05B2002E69D0337C03F00F03052B24
:1011900064D13146594809F0CEFC032853D90022C6
:1011A0003146564809F0CFFC012244695348314684
:1011B00009F0C9FC0222D0F814A05048314609F0C9
:1011C000C2FC43694D480A270322314607FB03F856
:1011D00009F0B9FC43695F432146009743465246F4
:1011E00028460BF0B4FA04463146444809F0A3FC03
:1011F000052830D104223146404809F0A4FCB0F95A
:1012000014A03E48BC42C4BF3C4640F2FF353146C4
:101210004445BCBF4446002509F08DFC022826D178
:1012200000223146354809F08EFC4369AB4251DC5F
:1012300001223146314809F086FC4369AB4258DB54
:1012400006B0BDE8F08705EB850464004FF00008A8
:101250004FF42057C8E74FF0010AD2E705EB8504A9
:1012600064004FF000084FF420574FF0010AD9F8FE
:101270000830B3F902002A1A002AB8BF5242524578
:1012800007DC1A785109052907D8013161F34712A3
:1012900002E01A786FF347121A701B789F2B03D95C
:1012A000444501D0BC42CBD1A842C9D0002211464E
:1012B00004AE02A801F004FC224602A9304601F067
:1012C000FAFE96E806004846FFF70EFDD9F808300A
:1012D0005D80B5E70024D9F80830B3F90230A342A5
:1012E000AED021464846FFF72BFCD9F808305C8089
:1012F000A6E70124EFE700BF5C25010054060020AB
:10130000FC02002008B583680246F3B1012916D01B
:101310000ADB032908DC0379402B0CD006D8032B09
:1013200002D81046FFF77CFD002010E0422B02D0CF
:10133000FAD3803BF3E71046FFF714FFF4E7037995
:10134000042BF1D1FFF7EAF9EEE74FF0FF3008BDCB
:101350007FB5037C03F00F03062B054623D101461E
:10136000124A134809F0F7FB90B1037C03F00F0316
:10137000052B0DD1C4680026ACB1294601A8019403
:10138000FFF724F9039B1E600BF0F0FA6468F3E7A3
:1013900004AC002144F80C5D2046FFF717F9022148
:1013A0002046FFF7AFFF04B070BD00BF602501000D
:1013B0005406002038B583680446BBB1124B1B6845
:1013C000A3B10068FFF7C4FFA36800251D6023795F
:1013D000032B0CD8012B94BF0221294660790BF016
:1013E00035FCA3685A7865F303025A7038BD402B68
:1013F00003D0422BFAD1294600E002216079BDE8F2
:1014000038400BF023BC00BF0C04002000230380F5
:101410007047000013B5002423460094224621465D
:1014200003480AF009FD034B1C8002B010BD00BF49
:10143000CC020020FC02002010B5044670B3204905
:101440000EF0F1FC58B31F4920460EF0ECFC40B3FF
:101450001D4920460EF0E7FC28B31C4920460EF03B
:10146000E2FC10B31A4920460EF0DDFCF8B1194930
:1014700020460EF0D8FCE0B1174920460EF0D3FC10
:10148000C8B1164920460EF0CEFCB0B11449204632
:101490000EF0C9FC002814BF00200E2010BD012052
:1014A000FCE70220FAE70520F8E70620F6E70A2025
:1014B000F4E70B20F2E70C20F0E70D20EEE700BF89
:1014C000CC250100E325010005260100F7250100D8
:1014D0000A26010000260100FB250100C3250100AA
:1014E000D325010010B50446002836D00378002B20
:1014F00034D024490EF097FC90B3234920460EF0D7
:1015000092FC78B3214920460EF08DFC60B320494F
:1015100020460EF088FC48B31E4920460EF083FC9E
:1015200030B31D4920460EF07EFC18B31B492046FF
:101530000EF079FC00B31A4920460EF074FCE8B1B5
:10154000184920460EF06FFCD0B1174920460EF026
:101550006AFC002814BF00200C2010BD1846FCE7D0
:101560000220FAE70120F8E70820F6E70520F4E773
:101570000620F2E70720F0E70920EEE70A20ECE773
:101580000B20EAE7EF250100CF2501000F2601001F
:10159000DB250100E7250100D7250100DF2501003B
:1015A000EB25010014260100F325010010B50446C7
:1015B000406960B103689B69984718B16069036826
:1015C0005B69984760690368DB689847012010BD34
:1015D000406910B103685B691847704710B504464D
:1015E000406910B103685B689847204610BD000051
:1015F00008B503220168044809F0A5FA08B1007D86
:1016000008BDFF20FCE700BF5406002010B50322F0
:101610000C4601680B4809F096FA90B143690A49F3
:1016200003F47F432343436108480AF045FC214605
:101630000A2206480AF0C2FC0448BDE810400AF03D
:101640004BBC10BD540600203E2701004003002083
:1016500010B503220C460168044809F074FA20B161
:10166000406924F0FF04204000B210BD5406002061
:1016700010B503220C4601680B4809F064FA90B1DA
:1016800043690A4904F47F421343436108480AF05E
:1016900013FC21460A2206480AF077FC0448BDE8FC
:1016A00010400AF019BC10BD54060020522701005A
:1016B0004003002010B503220C4601680C4809F0D5
:1016C00042FA98B1E34363F47F4243690949134006
:1016D000436109480AF0F0FB21460A2206480AF055
:1016E00054FC0548BDE810400AF0F6BB10BD00BF31
:1016F000540600207F2701004003002038B50C4627
:101700004168054609B9002038BD0B7C03F00F0382
:10171000022B03D1002CF6D14869F5E7052BF2D155
:10172000054809F008FA8442EDDAE2B26968024835
:1017300009F009FA4069E7E75406002008B5416856
:1017400069B10B7C03F00F03022B06D0052B06D1E9
:10175000044809F0F0F900B208BD0120FCE70020C0
:10176000FAE700BF5406002008B5816809B90020D7
:1017700008BD0B7C03F00F03022B01D14869F7E78A
:10178000052BF4D10022034809F0DDF90028EED042
:101790004069EDE75406002008B5816809B90020CA
:1017A00008BD087C00F00F039A1E012A01D8000929
:1017B000F6E7052BF3D10022034809F0C4F900280D
:1017C000EDD0007CF3E700BF54060020826862B1D0
:1017D000137C03F00F03023B012B06D85161836891
:1017E0001A7C022161F303021A747047826842B1C5
:1017F000137C03F00F00023801289CBF61F307132C
:101800001374704708B5C16809B9002008BD0B7C86
:1018100003F00F03022B01D14869F7E7052BF4D140
:101820000022034809F08FF90028EED04069EDE767
:10183000540600202DE9F041C36804460E46ABB9BA
:1018400001681648154F09F076F90546042D0DDCA0
:1018500000213846D4F8008009F0ACF94146024630
:10186000E060384609F084F90135EFE7E3689BB1A1
:101870001A7C02F00F02022A0ED15E610849094863
:101880000AF01AFB31460A2206480AF05CFB0548BA
:10189000BDE8F0410AF020BBBDE8F081540600200D
:1018A0004627010040030020006828B1007C00F0BA
:1018B0000F00431F5842584170470000F8B50446D6
:1018C000FFF7F2FF002831D021682A48294F09F09C
:1018D00032F90546032D26680ADC0021384609F056
:1018E00069F931460246384609F042F90135F1E717
:1018F000002231461F4809F026F94369237401226A
:1019000021681C4809F01FF902226060216819480B
:1019100009F019F90422A0602168164809F013F9AA
:10192000237CE060032B02D00C2B19D0F8BD1020D3
:101930000BF032F8104B036005464460002120464E
:10194000FFF7DCFE03B2002BB6BF40422B8128819B
:101950006868FFF7F3FE094B68812B606561E5E776
:1019600014200BF019F8064B44600360054604F0A0
:1019700027FDF3E754060020B8240100F0330100EE
:101980008033010010B500230446016043610376F3
:101990004362FFF793FF204610BD000070B5056855
:1019A00006462F2128460EF0BBFA044698B10023C4
:1019B00000F8013BFFF796FD0B4905460B480AF07E
:1019C0007BFA0A22294609480AF0DFFA07480AF09A
:1019D00083FA284670BD2846FFF784FD0546002897
:1019E000F7D03460F5E700BFA325010040030020D5
:1019F0002DE9F04389B0002400F118080546CDF820
:101A000004804461047644620E4600293BD01F4B9B
:101A10001F68002F37D02F2130460EF0F7F981468E
:101A200050B3234602AAF05C19B238B12F2805D072
:101A3000142B02D0D0540133F5E7194608AB1944F2
:101A4000002301F8183C1248394609F084F80A22AC
:101A5000286009F1010140460EF041FA01A8FFF7A4
:101A60009DFF019B686203B92B762846FFF726FF8E
:101A7000284609B0BDE8F08332463946044809F0EB
:101A80006AF82860F1E700232B60EEE7AC03002042
:101A90005406002018B1034903480AF00DBA03495F
:101AA000FAE700BFAF25010040030020B825010080
:101AB00070B500229AB005460C4603A8114600F006
:101AC000FFFF0122294603A801F064FB4FF4407197
:101AD0002846FFF7BDFD00260443314610220AA820
:101AE00009960DF028FACDE90566E60518D503A894
:101AF00001F0B2FA172855D8012303FA00F041F695
:101B00004243184208D1984B0340002B4ED110F0AD
:101B1000240F47D0954900E0954905A80EF08DF9AE
:101B200003A801F09BFA082866D8012606FA00F0FF
:101B300010F4837F60D08F4809F0D4FA002800F0B9
:101B4000A3808D4B93F90030002B40F09D80032241
:101B500030210EA805F058FA2B682F2219680EA81C
:101B60000EF097F900964FF40073142209A903A808
:101B700001F066FBA0051CD4E1053DD5012305AAB3
:101B80000EA97C4809F0E5FC7C497D480AF094F9EF
:101B90000EA97B480AF099F97A4979480AF08CF93C
:101BA00005A923E0784976480AF086F924F4807480
:101BB000B6E703A801F050FA0228DDD003A801F02F
:101BC0004BFA0528D8D0334609AA0EA9694809F06E
:101BD000C0FC6A496A480AF06FF90EA968480AF021
:101BE00074F9684966480AF067F909A964480AF077
:101BF0006CF963480AF070F9A2055CD50023032252
:101C000030210EA805F000FA2B682F2219680EA8C3
:101C10000EF03FF95D490EA80EF0E9F803A801F0B7
:101C20001DFA0438012836D8172203A907A801F0A5
:101C30009CFA002300934FF44073142209A903A8CF
:101C400001F0FEFA03A801F009FA51490EA80EF0BE
:101C5000CEF84A494A480AF02FF90EA948480AF036
:101C600034F9484946480AF027F909A944480AF0D6
:101C70002CF943480AF030F93E4809F033FA18B11C
:101C80003D4B93F900305BB1284621B2FFF7F0FCE1
:101C900000201AB070BD002300934FF40073CCE70E
:101CA0000EA9012309AA334809F053FC4FF400712F
:101CB0002846FFF7FFFCE3054DD503A801F0CCF95A
:101CC00001380B280BD8DFE800F04A0A0A0A0A4A52
:101CD0000A0A0A06484D2F4905A80EF0AEF800235F
:101CE000032230210EA805F08FF92B682F221968E6
:101CF0000EA80EF0CEF825490EA80EF078F8264969
:101D00000EA80EF074F81D491D480AF0D5F80EA96A
:101D10001B480AF0DAF81B4919480AF0CDF805A962
:101D200017480AF0D2F816480AF0D6F8114809F018
:101D3000D9F90028A8D0104B93F90030002BA3D17B
:101D40000EA9012305AA0B4809F003FC4FF480718A
:101D50002846FFF7AFFC01209BE71049BCE72B7C2E
:101D6000052BBCD10E49B7E701008000E325010037
:101D7000CC250100BC030020880300203826010088
:101D800040030020102501002A260100032D010038
:101D9000EF2501000A260100CF25010000260100E1
:101DA000FB25010038B50B0505460C460CD405F0A3
:101DB000B2F8952808D902F06FF828B121462846D4
:101DC000BDE83840FFF774BE04F440712846FFF7C1
:101DD0004FFC034903480AF06FF84FF0FF3038BD5D
:101DE000192601004003002010B54FF4407104464D
:101DF000FFF72EFC014670B1074B93F90030062B1C
:101E000009D12046FFF7CEFF20464FF44071BDE8D0
:101E10001040FFF74FBC10BDB0030020012970B582
:101E200005460C4601D1FFF7DFFF686950B1036832
:101E30009B69984730B16869036821B29B68BDE827
:101E400070401847002070BD43691BB11A681846DE
:101E5000526B1047007C70472DE9F04F8FB004AEF5
:101E6000039304469DF860300293304686E80600EE
:101E700001F082F90746054602F00EF8039B8346FF
:101E80001BB11A78002A40F05B83237E13B104F162
:101E900018030393002D40F05F83039B002B40F059
:101EA0005083676A002F00F05783304601F064F9D1
:101EB000002840F05183FAB231460CA801F060F9D5
:101EC0004AE3304601F0B8FA2368002B00F0738330
:101ED000204600F025FD00288146A448D4BF4FF0DD
:101EE00000084FF0010809F0F7FF237C072B1AD0F8
:101EF0000398FFF7A1FA82462046FFF779FB05B267
:101F00000DB90FFA88F5BAF1000F0CD055450AD07B
:101F10009749964809F0D0FF0A22294693480AF0CB
:101F200034F8924845E3002206AD1146284600F0F9
:101F3000C7FD00222146284601F02CF98246E0B96F
:101F40008C498A4809F0B8FF2046FFF77DFF2946F3
:101F500002B20CA800F0E4FD29460CA800F0F2FD46
:101F600021465246284601F089FD284601F064FAD0
:101F70004FF420612046FFF715FF304601F06CF862
:101F8000092800F25281DFE810F0B0005001500142
:101F90001E000A00500150013B0062006200B9F1CE
:101FA000000FCCBF0222012229460CA801F0DDF867
:101FB000284601F051F8314602460CA801F0D5F848
:101FC0004FF0010806E1237C072B00F00381204637
:101FD000FFF70EFB0528804636D16749634809F0B4
:101FE0006BFF0A224146614809F0CFFF5F4809F0C4
:101FF00073FF237C052B0CBF0C2201222946DCE752
:10200000237C072B00F0E6802046FFF7F1FA062834
:1020100080460DD15949554809F04EFF0A224146E4
:10202000524809F0B2FF514809F056FF0222E5E795
:1020300053494E4809F040FF0A2241464B4809F0F7
:10204000A4FF4A4809F048FF6FF002064DE10CA8D2
:102050000022294601F089F8304600F085FEA8B933
:102060004FF0050A304600F0F7FF092804BFCAF117
:10207000000A0FFA8AFA0A2F00F2AC80DFE807F0B4
:102080000FAA11AAAAAAAAAAAA233000304600F0D1
:102090007EFE0FFA80FABAF1000FE1D0E2E74FF0CE
:1020A00001085146284600F0E9FD002800F0928022
:1020B00021460022284601F0E1FC4FF42061204631
:1020C000FFF770FE86E05146284600F016FE002815
:1020D00000F08080022229460CA801F051F8E7E7C1
:1020E0005146284600F02BFEF1E7304600F03CFE5A
:1020F000824600286ED00C2F6CD8DFE807F0076B03
:10210000346B6B6B6B6B6B867E8E6700B9F1000F67
:10211000304640F3F48100F03AFE20B9022229460D
:102120000CA801F022F8284600F096FF0146204650
:10213000FFF76CFA4FF410612046FFF733FED046EC
:10214000284600F08BFF04281CD1304600F086FFA3
:1021500002281CD1304600F081FF294602460CA817
:1021600000F07FFF13E04FF0000AE9E74003002092
:10217000622601007826010095260100A4260100B0
:10218000B5260100284600F069FF0528DDD0237C34
:10219000072B08D1304600F0EEFD20B1022229467F
:1021A0000CA800F05EFF2046FFF74EFE00B2009044
:1021B00096E80C0029460CA801F0B8F9BAF1000F16
:1021C0003FF476AF284601F081FC71E796E8030002
:1021D00085E80300D4F814A0BAF1000F00F0CB801A
:1021E000304600F039FF092800F2AE80DFE800F049
:1021F0009EA983ACAC5F2BAC9E9E304600F03CFDAC
:10220000C1B2284600F0E2FC61E7304600F02DFD47
:102210000146284600F0C0FC59E7304600F00BFDAF
:102220000146284600F0E3FC42E7304600F014FF88
:10223000294602460CA800F098FFFAB229460CA8DD
:1022400000F09EFFBCE6B9F1000F2BDCAF49B048AF
:1022500009F032FE676908AE3B6830460122294624
:10226000D3F8288000F081FF0123009396E8060050
:10227000039B3846C047062106462046FFF7C6F9AD
:102280004FF480712046FFF78DFDA249A04809F068
:1022900013FE0A2231469E4809F077FE9C4809F059
:1022A0001BFE22E09C499A4809F006FECCE6B9F1F3
:1022B000000F1EDD67690AAE3B68304602222946E0
:1022C000D3F8288000F051FF0123009396E8060020
:1022D000039B3846C047052106462046FFF796F97E
:1022E0004FF480712046FFF75DFD30460FB0BDE82A
:1022F000F08F8A49D7E72046FFF77AF9052813D0EF
:1023000067690CAE3B68304602222946D3F8288024
:1023100000F02BFF0123009396E80600039B38464C
:10232000C04702210646A8E77D49BCE7606903680B
:10233000CDF800809C6A039B95E80600A0470646FE
:10234000A3E7B9F1000F13DC606901220368009272
:102350009E6A039B95E80600B0470646284600F0B3
:10236000FEFC002891D0284600F076FE014684E766
:102370004FF0FF3689E7237C062B5AD0072B42D03B
:10238000052B4FD1022F00F09D800C2F4AD1204603
:10239000FFF738FA030C074605D1236861491A682C
:1023A000614809F0C1F8284600F012FD0BF08EFFDD
:1023B0005E4B00220BF0E2FF0CF090FA0FFA80FA6D
:1023C000082005F020F86AF30F07804660F31F47E6
:1023D00057494F4809F070FD0A2251464C4809F010
:1023E000D4FD54494A4809F067FD1FFA88F10A22D2
:1023F000474809F0CAFD464809F06EFD39462046B7
:10240000FFF718FA0EE0029B63B16068037C03F0EB
:102410000F03052B06D1BBF1000F03D0039A314601
:1024200000F006FA284600F09AFC002850D1012658
:102430005BE751462046FFF761F90FFA80F807463F
:10244000284600F009FEB8F1000FEBD0BCBFC7F181
:1024500000080FFA88F808F1FF339BB2B8BF4FF0BD
:10246000010A132BDED807B2012140460AF0EEFB29
:10247000BAF1000F20D0012F1CD0063F18BF012752
:10248000394640460AF00AFC2B49214809F014FD60
:102490000A2241461E4809F078FD28491C4809F0E7
:1024A0000BFD0A2239461A4809F06FFD184809F059
:1024B00013FDB7E70027E3E7012FE1D0BB1F5F4221
:1024C0005F41DDE752462146284601F0D7FAA9E7E9
:1024D000304600F0C1FD052801460BD1B9F1000FCF
:1024E000A5DD2046FFF792F84FF480712046FFF7F4
:1024F00059FC9CE7284600F0AFFD0146F1E700F0EB
:1025000046FC00283FF40FAE012208E6CD2601006C
:10251000400300200C270100DA260100EA26010012
:10252000FC2601001D270100BC03002000005940CB
:102530002C270100302701001827010091250100F8
:1025400057B91B78002B3FF4ACAC03A8FFF726FA71
:10255000074600283FF4A5AC04F0DDFC174905460A
:10256000174809F0A9FC0A222946154809F00DFD73
:102570001449134809F0A0FC23681148196809F0B0
:10258000A4FC11490E4809F097FC03990C4809F086
:102590009CFC0E490A4809F08FFC0D49084809F0D7
:1025A0008BFCC72D3FF78DAC0A490B4809F084FC22
:1025B000094809F091FC4FF0FF3696E66D290100BD
:1025C000400300203E260100452601004B26010065
:1025D00051260100542601005C0300202DE9F0473C
:1025E0008EB00746CDE90221002900F01B810AB117
:1025F000137823B93B7E13B107F118030293029BB2
:102600005BB9D7F824800024039D2E5D7EB130464F
:102610000DF026FE28550134F6E71B78002BF0D08C
:1026200002A8FFF7BBF980460028EAD0EBE728466E
:1026300000F014FA7C4905467C4809F03DFC0A226A
:1026400029467A4809F0A1FC04AC784809F044FC1A
:10265000EAB23146204600F033FAB8F1050F21D036
:10266000B8F1060F08BF17255FFA88F60DF12809A3
:1026700032462146484600F083FD092D14DC082D22
:102680003DDAAA1C03DB6B1C40F3CC80B5B10123FF
:10269000009394E80600029B3846FFF7DDFB0EB07E
:1026A000BDE8F0871825DFE7172D00F08980182D89
:1026B000EDD100222146484600F057FD06AD03A9A2
:1026C000284604F0DEFB32462946484600F058FD15
:1026D000284600F0C3FC061C18BF01264FF0000A74
:1026E000039A0FFA8AF3A2B1BAF1030F10D003A82C
:1026F00004F0A6FB49F82A000AF1010AF0E703A852
:1027000004F09EFB21460246484600F0C8FCBEE7A6
:102710005346B8F10A0F0DD0B8F10B0F12D0B8F133
:10272000090F17D1284600F032FB81B2204600F095
:1027300033FAACE7284600F02AFBC1B2204600F08D
:1027400045FAA4E7284600F022FB0146204600F0A7
:102750004EFA9CE733449BB2013B032B97D8DFE84A
:1027600003F00207122095E8030084E803008EE7D7
:10277000284600F00CFB9DF8283082B2214608A8BC
:1027800000F0BCFC83E7284600F001FB9DF82C20FC
:1027900000929DF8283082B2214608A800F097FCEC
:1027A00075E7284600F0F3FA9DF82C2000922146A8
:1027B00082B29DF8283008A800F089FC0C99C5E782
:1027C00000222146484600F0D0FC0025039A2BB297
:1027D00042B1042D0BD003A804F032FB49F82500C8
:1027E0000135F3E7032B11D0042B7FF450AF9DF894
:1027F000341001919DF8301000919DF82C309DF817
:102800002820214608A800F09DFC40E79DF83010E4
:1028100000919DF82C309DF82820214608A800F052
:1028200081FC34E700203AE735270100400300200F
:102830002DE9F0470E468CB09146002853D0037C1A
:1028400003F00F03052B62D1324DC4682B78DFF8FB
:10285000C8A0DFF8C88001332B70002C54D0237C33
:1028600003F00F03042B4DD16269DAF800104046E3
:1028700008F071F90746002844D0037C03F00F03E9
:10288000052B3FD1014602A8FFF77CF85EB102A8F4
:10289000FFF70AF838B100230093316872684B469D
:1028A00002A8FFF7D9FA00223946404608F04BF952
:1028B000E0B1037C03F00F03022B17D14369072B10
:1028C00014D101223946404608F03DF94A463146C6
:1028D000FFF7AEFF9EB990B12B7802A8013B2B7099
:1028E000FEF77CFE01200CB0BDE8F0873EB902A8DF
:1028F000FEF7DAFF18B102A800F012F8EBE702A821
:10290000FEF76CFE6468A8E72B78013B2B70002073
:10291000E9E700BF3D030020AC030020540600207F
:1029200073B5002205461146684600F0C9F82B68C9
:102930003D48196809F0C9FA2846FEF7B5FF58B9AD
:102940003A49394809F0B8FA374809F0C5FA4FF062
:10295000FF34204602B070BD2846FEF749FE2B7CAE
:10296000072B16D001300D2813D8012606FA00F0E7
:1029700043F68404044006D110F0490F09D02046E4
:10298000FFF788F8E5E72A49274809F095FA344621
:10299000DFE76A693AB113681046DB6A9847041C9E
:1029A00018BF0124EBE72946684600F0F3FB2B7CB7
:1029B000033B062B2FD8DFE803F02A152E2E042A1E
:1029C00015006B681B7C03F00F03052B29D11949F7
:1029D000154809F071FA002211466868FFF728FFD0
:1029E0000446CDE70021684600F0CAFA04461249C1
:1029F0000D4809F061FA21460A220B4809F0C5FA90
:102A0000094809F069FA003418BF0124A1E76846B3
:102A100000F0BDF9EAE70949034809F04DFA00243E
:102A200097E70024E3E700BF400300205B27010095
:102A3000AF25010064270100742701006A27010007
:102A400007B5002300931A461946034809F0F4F924
:102A500003B05DF804FB00BF00030020F8B5064694
:102A6000F0B10378E3B12D2B1ED0A3F13002092A77
:102A70001AD9252B1AD07B2B1AD0232B1BD00F4F02
:102A8000012404EBC4053D4428460DF0FAF929461B
:102A9000024630460DF011FA20B10134192CF0D164
:102AA0004FF0FF342046F8BD0024FBE70824F9E787
:102AB0006FF00104F6E71724F4E700BF8827010050
:102AC00010B500234370C370037143718371C371E8
:102AD00061F307138370027010BD10B50023072443
:102AE00003704370C37064F307138370416010BDBB
:102AF00089B20C2910D8012000FA01F141F25923C2
:102B000019420CD111F4A46F08D140F60603194202
:102B10000CBF00200220704700207047082070473B
:102B200038B50C46054611462046FFF7E1FFA3786D
:102B300060F30713A37023682B6063686B602846FB
:102B400038BD00008B781B09013B082B1AD8DFE841
:102B500003F0160E0E19191919050C000C4B4B60D9
:102B60000B6803604B68436070470A4BF7E76423C8
:102B70008B71CB7923F00103CB7100234B71FF23C1
:102B80000B71EDE700230B714B718B71CB71E7E794
:102B90000000A0410000964283781A0903D0022A5F
:102BA00005D000207047022262F30713837040F2C1
:102BB0006D139942A8BF1946C379817123F00103AF
:102BC000C1F300211943C1710120704783781A09AC
:102BD00003D0022A05D000207047022262F30713B7
:102BE00083706429A8BF642141710120704713B527
:102BF000642304460093084600234FF4FA72992197
:102C000009F0A5FDA3781A090ED0032A11D820EAED
:102C1000E0706428E379A8BF6420013060F34703C3
:102C2000E371012002B010BD022262F30713A3700A
:102C3000EDE70020F6E707B5C27912F0FE0F11D0DC
:102C400083781B09013B022B0CD850084FF4FA7310
:102C50000093642299230021013809F078FD03B024
:102C60005DF804FB4FF0FF30F9E7C379827903F098
:102C7000010342EA032070474079704783781B09BB
:102C8000013B0A2B37D8DFE803F006063636362A32
:102C90001616160D0D000379194481F30801017110
:102CA000012070474368194421EAE1716429A8BFF3
:102CB00064214160F4E7436807EE903AFDEEE77A5D
:102CC00017EE903A194421EAE1716429A8BF642102
:102CD00007EE901AF8EEE77A17EE901AE9E74368E4
:102CE0000A2211FB023121EAE171B1F57A7FA8BF16
:102CF0004FF47A71DDE70020704783781B09022BBF
:102D00001BD1C279837902F0010243EA02231944FC
:102D1000B1F5B77F0FDA40F26D1331EA210128BF18
:102D20001946C379817123F00103C1F300211943CE
:102D3000C171012070470021F3E7002070478378BC
:102D40001B09022B09D14379194421EAE171642955
:102D5000A8BF6421417101207047002070470078AE
:102D6000003018BF01207047837813F0F00F14BFB4
:102D7000012000207047807800F0E000202804D077
:102D8000A0F14003584258417047012070478378B2
:102D90001B09013B0A2B18D8DFE803F008081706C7
:102DA00006120A0A0A060600406870470079704752
:102DB000406807EE900AFDEEE77A17EE900A70473A
:102DC00040680A2390FBF3F0704700207047000032
:102DD00083781B09013B0A2B1ED8DFE803F013138D
:102DE0001D06060E191919060600436807EE903AEB
:102DF000F8EEE77A17EE900A704743680A2293FBD1
:102E0000F2F3F3E7037907EE903AF8EE677AF1E729
:102E1000436807EE903AEDE7DFED017AEAE700BF9D
:102E20000000000083781B09013B07B50A2B5FD81F
:102E3000DFE803F016165E5E5E44245E5E06060062
:102E4000406839B1D0F1640055D46428A8BF64202B
:102E500001B201E00028F8DA084603B05DF804FB8F
:102E6000007931B1002100916423FF2209F06FFC49
:102E7000EEE764230093FF220B46F7E7436807EE73
:102E8000903A99B19FED1E7A77EE677AF5EEC07AA7
:102E9000F1EE10FA2FD4F4EEC77AF1EE10FA2CDC32
:102EA000FDEEE77A17EE903A19B2D5E7F5EEC07A63
:102EB000F1EE10FAD0D49FED127AECE7406861B1E0
:102EC00040F2F133984216DC10F1090F15DB6FF078
:102ED000090390FBF3F06430BAE710F1090FBBDB94
:102EE00040F2F133984208DC0A2190FBF1F0AFE7A1
:102EF0004FF0FF31B0E70021AEE76421ACE700BF3F
:102F00000000C84213B504460846A3781B09013BDC
:102F10000A2B32D8DFE803F00F0F313131281A3194
:102F200031060600FF23009300236422194609F0AE
:102F30000EFC606007E0FF23009300236422194623
:102F400009F005FC2071012002B010BDFF230093A1
:102F500000236422194609F0FAFB07EE900AF8EE06
:102F6000E77A17EE900AE4E740F6F61300930023A1
:102F70006422194609F0EBFB60600020E4E70000E2
:102F800083781B09013B0A2B5FD8DFE803F0171792
:102F90005E5E5E461E5E5E060600406841B1002829
:102FA00039DBFF28A8BFFF20C0F1FF0001B20AE013
:102FB000002808DBFF28A8BFFF20F7E700790029D9
:102FC000F4D0C0F1FF01084670474368A9B107EE8D
:102FD000103AB5EEC07AF1EE10FA1CD4DFED1D7A8E
:102FE000B4EEE77AF1EE10FA32DC77EEC77AFDEE56
:102FF000E77A17EE903A19B2E5E707EE903AF5EE68
:10300000C07AF1EE10FADED49FED127AF4EEC77AB0
:10301000F1EE10FAEBDDFF21D5E7406859B110F170
:10302000090FF8DBB0F5206F12DA6FF0090190FBA1
:10303000F1F0FF30BAE710F1090FC4DBB0F5206FF3
:10304000E9DA0A2190FBF1F0B0E74FF0FF31BAE77F
:103050000021B8E700007F430078704780780009BE
:1030600070478B7810B562F307138B700B680360A1
:103070004B68436010BD8B7810B51C09013C012CD6
:1030800084BF012464F3071382F30802D2B288BF1D
:103090008B700B680A7103604B68436010BD8B78BE
:1030A0004A6030B50A2565F307138B700B6803601F
:1030B0004B68436030BD8B784A6030B5062565F3B8
:1030C00007138B700B6803604B68436030BD70B5AD
:1030D0008C788A71022666F307148C70C2F3002480
:1030E000CA794B7122F001029DF810300B71224316
:1030F0000B68CA7103604B68436070BD70B58C7813
:103100008A71032666F307148C70C2F30024CA790F
:103110004B7122F0010222430B68CA7103604B68B5
:10312000436070BD70B58D784B71042666F307154A
:103130009DF810308D700B718A710B6803604B68BD
:10314000436070BD70B58D784B7105269DF81030C9
:103150000B7166F307159DF814308D70CB718A7171
:103160000B6803604B68436070BD10B50A700B6854
:1031700003604B68436010BD807800F00F0070471B
:103180008B7810B562F303038B700B6803604B6898
:10319000436010BD2DE9F041044690460D4619B933
:1031A00000263046BDE8F0810846FEF77DFB064666
:1031B0000028F5D02846FEF7EFFA074680B12846EA
:1031C000FEF7D2FAA378606067F30713A370B8F133
:1031D000000FE6D02846FEF70BFA46462070E0E7DF
:1031E000AA68137C03F00F03022B03D0032B09D032
:1031F0000646D6E7A378526962600A2161F3071395
:10320000A370CEE75369A27807EE903AF8EEE77A1A
:10321000072117EE903A61F30712A2706360C0E7CE
:1032200010B500220446027042708270C2700271B2
:1032300042718271C271FFF7ADFF204610BD0000E0
:103240002DE9F0432DED028B85B0044615469846D6
:103250009DF838900F4600293ED0002A00F0D28019
:1032600000230B70017821B318F4807F21D0664BC6
:1032700001EBC101194438460CF031FE2A4663497E
:1032800038460CF006FE38460CF0FBFD2D1A3E18B1
:10329000013D18F4007F1FD0A3781B09013B0B2BC5
:1032A0001AD8DFE803F00835669BA12570707022FC
:1032B0001FA93E46EDE72079B9F1000F06D064233F
:1032C00000930023FF22194609F041FA504A0346B1
:1032D000294630460CF0CAFC384605B0BDEC028BDE
:1032E000BDE8F08363684B4AF2E763684A4AEFE758
:1032F00061680A2291FBF2F302FB1312002AB8BFA5
:1033000052420092454A294630460CF0AFFCE3E7B2
:103310002046FFF790FCE279A37994F8058001B28A
:103320000029207902F0010202DBB9F1000F14D06C
:1033300043EA0224B9F1000F06D06423009300236E
:10334000FF22194609F003FACDE900802346344AEA
:10335000294630460CF08AFCBEE7CDE90101CDF8E4
:10336000008043EA02232F4A294630460CF07EFCB7
:10337000B2E7E379A2796179009103F0010342EAAF
:103380000323294ABFE7636808EE103AB5EEC08A06
:10339000F1EE10FA4CBFF1EE487AF0EE487AFDEE0D
:1033A000E78AB8EEE87A77EEC77A9FED207A67EE83
:1033B000877A17EE900A09F037FD07EE900AB5EE0E
:1033C000C08AFDEEE77AF1EE10FACDED007A18EE44
:1033D000903A01D5164A96E7164A94E72279A379DE
:1033E000019262790092B2E7E279A379029222799E
:1033F000019262790092B6E72A46616830460CF085
:103400006EFD69E7174667E788270100B8370100B6
:10341000D5280100D8280100DC280100E02801009F
:10342000EA280100E7280100ED2801000000C84259
:10343000F3280100F428010030B58BB0134C0023B1
:103440002022009302A94FF440730546FFF7F8FECF
:1034500002A9204608F039FD0D49204608F02CFD50
:10346000A9780A220909204608F0A8FD0949204642
:1034700008F022FDA9780A2201F00F01204608F089
:103480009DFD204608F028FD0BB030BD4003002014
:10349000C2280100C728010070B58B78B2EB131F5A
:1034A00086B005460C46164606D123682B60636835
:1034B0006B60284606B070BD1849194808F0FCFC3E
:1034C000A17817480A22090908F078FD154914481F
:1034D00008F0F2FC0A223146114808F06FFD12494B
:1034E0000F4808F0E9FC0023CDE9043366F3071325
:1034F00022788DF812304FF0FF338DF810200093B2
:1035000002A86368226804A900F010F8029B2360F7
:10351000039B63602046FFF78FFFC6E7FC2801008E
:103520004003002010250100B83701002DE9F04FBD
:103530008DB00C4604ADBDF958108046204685E894
:103540000C00FFF7D5FA02902846FFF774FB011E26
:1035500002DB2046FFF74BFB9DF81230A278C3F345
:10356000030161F30302A270C2F303120B2A38D8DD
:10357000DFE812F098000C000C009C001401F00031
:103580009800A700A700A700980098001B095A1EE2
:103590000A2A6ED8DFE802F0514317090638546D45
:1035A0006D2F2F009DF81720E2719DF81620A27153
:1035B0009DF8152062719DF814202271A27863F3A2
:1035C0000712A2700DE0BDF81630C3F30802E379CC
:1035D000A27123F0010343EA1223E3719DF8153031
:1035E0006371029B002B00F0CF801A46214606A88B
:1035F000FFF752FFC8E0059B002B36DBFF2BA8BF6F
:10360000FF23DBB22371ECE7059B13F1090F2CDBE1
:10361000B3F5206F2BDA0A2293FBF2F3F1E7BDF842
:103620001630C3F30802E379A27123F0010343EAE1
:103630001223E3719DF8153063719DF81430E1E7B2
:10364000DDED057AF5EEC07AF1EE10FA0DD49FEDBE
:10365000BF7AF4EEC77AF1EE10FA08DCFCEEE77AF6
:10366000CDED037A9DF80C30CCE70023CAE7FF23A9
:10367000C8E7B749B74808F01FFC9DF81210B548D5
:103680000A22090908F09AFCB349B24808F014FC70
:10369000A178B0480A22090908F090FCAD4808F06A
:1036A0001BFC9EE7059A62601B0987E700212846FC
:1036B000FFF766FC2071A378022262F30713A37060
:1036C0008FE71B095A1E0A2AD3D8DFE802F0112916
:1036D0002F29290623232318200005980AF0E4FD4A
:1036E00000229E4B0AF074FF0BF040F9606078E70F
:1036F0009DF8143007EE903AF8EE677A03E0DDEDBE
:10370000057AF8EEE77A17EE903A636069E7DDED47
:10371000057AF1E7A27863F30712A270059BF4E73C
:10372000A278059863F30712A270DFE70021204614
:10373000FFF726FCBDF816302071C3F30802E379C9
:10374000A27123F0010343EA1223E3719DF81530BF
:103750006371B0E701271B0903F10F0202F00F01AB
:103760000A2986D801228A4040F265610A4217D1AF
:10377000910735D412F0180F3FF47BAF059A6260C1
:10378000A27863F30712A2702368C8F80030636858
:10379000C8F8043040460DB0BDE8F08F0027DAE7E6
:1037A000013B0A2B00F2C380DFE803F0B0C106C181
:1037B000C1B5BAC1C1B3B300FF23BDF816208DF85F
:1037C0001430642161F30802ADF8162000228DF850
:1037D00015209DF81220022161F307128DF81220A6
:1037E0000023FF259DF8150000956422194608F076
:1037F000AEFF0028C0F29D8000239DF815000095C3
:103800006422194608F0A3FFA84208DC00230095B3
:103810009DF815006422194608F099FF05469DF8A9
:103820001400FCF70DFE0646002F47D09DF81770D8
:103830007F08013F3FB27B1C40F098807F2D4FF006
:10384000FF0778DC0023C5F17F00194647F6816247
:103850007043009708F07BFF4FF4FF730093002341
:103860001946E0717F22284608F071FF00231946AF
:1038700000903A46304608F06AFF009706466423F7
:1038800028467F22002108F062FFBE420546A8BFFD
:103890003E4633492F4808F00FFB0A2229462D489F
:1038A00008F073FB2F492B4808F006FB0A2231462B
:1038B000284808F06AFB274808F00EFB00231A4648
:1038C000194606A808F079F9BDF816004FF6FF73FF
:1038D00000930023194640F26D12C0F3080008F06F
:1038E00036FFF2B2E9B280B208F07DF9030CA371A1
:1038F000030A637120711C49164808F0DDFA20465E
:10390000FFF79AFD06A808F0EDF86AE69DF8143076
:1039100053E7059B51E7059B0A2293FBF2F34CE723
:10392000DDED057AFDEEE77A17EE903A45E70023E4
:1039300043E7002573E76423284600973A46802131
:1039400008F005FF00230546E371A2E700007F436E
:1039500069280100400300201025010000002440D8
:103960007B28010088280100BB2801004FF01E0BB6
:1039700064231A46CDF800B00021384608F0E7FE6F
:103980004FF064095B468246CDF8009038464A46BF
:10399000002108F0DCFE7F2D83464FF0FF0754DC4A
:1039A000C5F17F000023704319462D4A00970BFB99
:1039B00000F008F0CCFE4FF4FF730093002319468B
:1039C000E071E32205EB0A0008F0C1FE002319466E
:1039D000039000903A46304608F0B9FE00230646B0
:1039E000009728467F22194608F0B1FEBE420546E0
:1039F000A8BF3E461B491C4808F05EFA0A22514601
:103A0000194808F0A0FA1949174808F055FA0A228F
:103A10005946154808F097FA1549134808F04CFA2A
:103A20000A222946104808F0B0FA12490E4808F058
:103A300043FA0A2231460C4808F0A7FA0E490A4810
:103A400008F03AFA0A22039932E74B4628460097D3
:103A50003A46802108F07BFE00230546E371C9E762
:103A6000646A310096280100400300209C28010070
:103A7000A2280100AA280100B2280100F8B50546D5
:103A800017460C4611B900263046F8BD0846FDF72A
:103A90000BFF06460028F6D069682046FDF796FE23
:103AA000A97820460909FDF7A1FE1FB12978204613
:103AB000FDF7ACFD0349044808F0FEF92846FFF77E
:103AC000BBFCE1E7CE2801004003002083781B09FE
:103AD000013B012B37B5054620D80023FF24007990
:103AE00000946422194608F032FE002814DB0023FB
:103AF000287900946422194608F029FEA04207DCC8
:103B00000023009428796422194608F020FEC4B2EC
:103B10002C71012003B030BD0024F9E70020F9E743
:103B200007B5002300931A461946034808F084F9A4
:103B300003B05DF804FB00BF0803002002F016BAD2
:103B400002F0D8B907B5002300931A461946034876
:103B500008F072F903B05DF804FB00BF1003002009
:103B6000704700002DE9F041044692B00D464748E9
:103B70004749164608F0A0F92146444808F0A5F93F
:103B80004449424808F098F965B10023AB5503F069
:103B9000C2F9F92809DC4049404808F08DF93F484E
:103BA00008F09AF912B0BDE8F08104213C48DFF832
:103BB000DC8003F083F82F462E44BE4205D017F870
:103BC000011B404608F085F9F7E7304808F084F912
:103BD000344B93F90030052B4FF0000314D103222E
:103BE000412101A803F010FA01A80CF04AF906B22D
:103BF000324601A920460CF060F900B2B8B12A495A
:103C0000224808F059F9CDE70222412101A803F02A
:103C1000FBF901A80CF035F906B2324601A920469D
:103C20000CF04BF900B210B100230122D8E7344464
:103C30001E4920460CF0F7F840B928460CF021F94F
:103C4000012803D9284607F031F8ABE72F21204699
:103C50000CF0DCF8064628B1002303704378242BCF
:103C6000A0D001362378242B9CD0214601A8FDF753
:103C7000BFFE01A8FDF718FE20B13246294601A873
:103C8000FEF7ACFC01A8FDF7A9FC8BE74003002080
:103C9000DA290100DD290100E02901005C03002090
:103CA0001C030020B0030020ED290100F8290100C9
:103CB00038B5084D01244FF47A7008F035FE2146DE
:103CC00001340A222846E4B208F078F9142CF2D123
:103CD00038BD00BF8C03002008B50449044808F033
:103CE000EBF8BDE8084003F029BA00BF352C01000D
:103CF0008C03002010B586B00F4C10494FF0FF32F6
:103D000003920F4A009200234C222046CDE904235F
:103D1000CDE9013308F0D0F80A4B0B4819686A4620
:103D200006F0E2FE684606F0F5FA0849204608F07B
:103D3000C3F806B010BD00BF8C030020AB2B010000
:103D4000883801000C04002054060020C52B010017
:103D500010B50024214600220F48013406F04DFA28
:103D60004D2CF7D14C2246210B4806F046FA48224A
:103D70004721094806F041FA43224821064806F047
:103D80003CFA49214622044806F037FA0349044820
:103D9000BDE8104008F090B818030020E82E01009C
:103DA0008C03002030B52DED028B8DB0304B049389
:103DB0000C4608EE102A00211C2205A80BF0BBF8C7
:103DC00004AA0821204602F0F3FF00238DF82130D9
:103DD000284B1B68002B47D0274808F07DF827495F
:103DE000254808F069F818EE100A0AF06FFA022365
:103DF0000246009320480B4608F0A6F920491E48C9
:103E000008F05AF804A91C4808F05FF81D491A4840
:103E100008F052F8184808F05FF81B4B1B48196867
:103E200004AA06F098FEDFED1A7AB4EE678AF1EE86
:103E300010FA054618D0DFED177AB4EE678AF1EE76
:103E400010FA11D0B5EE408AF1EE10FA0CD002ACA7
:103E500018EE101A2046FEF740FE94E80C004FF0D2
:103E6000FF31284603F094F90DB0BDEC028B30BD54
:103E70004E494C000C040020400300202D27010077
:103E800048310100112501000004002054060020E3
:103E90000000FEC20000AA42034B93F9000005385F
:103EA00018BF0120704700BFB00300202DE9F0418A
:103EB00016491748174E184F154D07F0FDFF0024FF
:103EC00006F1010816F8013F0F2B03D839462846A2
:103ED00007F0FBFF052C4FF010020DD0317828467B
:103EE00008F031F80D49284607F0E6FF0134E4B246
:103EF000062CE7D1BDE8F08198F80510284608F0B7
:103F000022F8284607F0E8FFF0E700BFD52B0100B4
:103F10008C030020B00300206C380100242E010027
:103F200070B5184C88B00DF11F030493631E029303
:103F3000A31E01930D46E31E00930394231F621FEB
:103F4000114968680BF0C6FE052809DC0F491048C6
:103F500007F0B2FF69680E4807F0B7FF08B070BD00
:103F6000FFF7A4FF0B4E0025053C625D2946304655
:103F7000013506F042F9062DF7D10749074807F049
:103F80009BFFEBE7B6030020472C01005B2C0100F0
:103F90005C030020180300206D2C01008C0300201E
:103FA00008B508B9002008BD037C03F00F03052BFA
:103FB000F8D1CAB20146064806F0C5FD0028F1D086
:103FC000037C03F00F03042BECD14069EBE700BF47
:103FD000540600202DE9F0430024C9B03C222146BC
:103FE00009A808940AF0A7FF7C22214629A8289452
:103FF0000AF0A1FF23460122402108A803F004F89B
:104000007F49804E804D08A80BF0F1FE80227F4949
:1040100028A80BF064FF012328AA08A97C4807F010
:1040200098FA23460122402108A802F0EDFF7949C1
:1040300008A80BF0DCFE8022774928A80BF04FFF80
:10404000764928A80BF0D3FE012328AA08A97048B6
:1040500007F07FFA23460122402108A802F0D4FF8E
:104060006F4908A80BF0C3FE80226E4928A80BF008
:1040700036FF012328AA08A9654807F06AFA2346F3
:104080000122402108A802F0BFFF674908A80BF0F1
:10409000AEFE8022654928A80BF021FF28AA012343
:1040A00008A95B4807F055FA32782F680132327060
:1040B000002F00F09E805E4BDFF8A091B3F80080E7
:1040C000ADF8008021461E220DF102000AF033FFF8
:1040D00021463E220DF16200ADF860800AF02BFF10
:1040E000DFF87C81FC68534F2A68002A77D0002CC7
:1040F00075D0237C03F00F03052BF6D121463846FB
:1041000006F019FD0028EFD000222146384606F0BF
:104110001AFD4369092B0ED8DFE803F059515159B4
:104120005905464659592022434968460BF0D7FEA7
:1041300000238DF8603000230122402108A802F0FE
:1041400063FF4022216808A80BF0A3FE3B4908A8A2
:104150000BF04DFE3A4908A80BF049FE01236A46D0
:1041600008A92B4807F0F5F99DF86030C3B100238A
:104170000122402108A802F047FF4022216808A838
:104180000BF087FE2D4908A80BF031FE2D4908A839
:104190000BF02DFE012318AA08A91D4807F0D9F934
:1041A00008F0E4FB64689FE72022274968460BF08B
:1041B00096FE2649402218A80BF091FEBBE720226C
:1041C000234968460BF08BFE40222249F3E7202268
:1041D000414668460BF083FE40224946EBE740210A
:1041E0000023012208A802F00FFF1B4908A80BF0CA
:1041F000FEFD3378013B337049B0BDE8F08300BF6A
:10420000DF3201003D030020AC030020D932010061
:10421000BC030020B93201000F330100FC32010061
:10422000E632010053320100CB3201004D32010071
:104230000829010054060020C5320100032D0100A9
:104240003A320100ED320100B43201007532010052
:10425000BF320100A8320100D232010063320100F6
:10426000AC32010010B5114C1149204607F024FE74
:104270001049204607F029FE4FF4FA7008F054FB6D
:104280000121152008F0E2FC0021152008F006FDB0
:104290004FF4FA7008F048FB1520012108F0FEFCED
:1042A0004FF4FA70BDE8104008F03EBB8C030020CC
:1042B000173201003732010013B50E4C0E490F487A
:1042C00007F0FAFD2146684604F00DF8684602F052
:1042D00075FE2146684604F01EF8684602F06EFE40
:1042E0002146684604F00BF8684602F067FE02B00B
:1042F00010BD00BFE4050020002E01008C0300204B
:1043000070B588B02F231522002102A801930AF06E
:1043100012FE16491648174D174C07F0CDFD0DF14A
:1043200005020621154802F043FD002614498DF8C8
:10433000116001A80BF05BFD01A9284607F0C5FD3F
:1043400001A9204607F04EF90E498DF8116001A829
:104350000BF04DFD01A9284607F0B7FD0A4A01A957
:10436000204607F0E1F8012008B070BD762C01006E
:104370008C03002040030020BC030020B103002078
:104380008B2C0100932C0100C2370100FFF7B8BF4E
:1043900018B10349034807F08FBD0349FAE700BF8E
:1043A000153201008C030020BB3D010010B5224CEA
:1043B0002249204607F080FD2149204607F07CFD78
:1043C000204B1868003018BF0120FFF7E1FF1E499D
:1043D000204607F071FD1D4B1868003018BF012002
:1043E000FFF7D6FF1A49204607F066FD194B1868FB
:1043F000003018BF0120FFF7CBFF1749204607F018
:104400005BFD164B1868003018BF0120FFF7C0FF96
:10441000204607F061FD1249204607F04DFD02F0ED
:104420007AFD0A220146204607F0BBFD2046BDE882
:10443000104007F051BD00BF8C030020932D0100F8
:10444000A02D0100AC030020A82D0100A80300202E
:10445000B12D0100B8030020B82D01000004002098
:104460006D2901002DE9F843074608460E460BF07A
:1044700008FD04B21F2CDFF83080A8BF1F2435468A
:10448000A7EB0609AB1B9C4207DD09EB0501404683
:1044900015F8012B05F0B1FEF4E7E11900220248FE
:1044A000BDE8F84305F0A9BE1803002007B50023B6
:1044B0008DF8043050B149683620FFF7D3FF044926
:1044C000044807F0F9FC03B05DF804FB01A9F3E729
:1044D000182A01008C0300202DE9F04780460F4682
:1044E00001461148164605F086FE0138C0B2FD2887
:1044F00018D8DFF834A00024013E25B208EB0401EF
:10450000B54209B207EB050906DA504605F073FE1D
:10451000013478550028F0D1002389F800300120BB
:10452000BDE8F0870020FBE7180300202DE9F04FDD
:10453000A7B0002395488DF81330CDE90533CDE9B8
:10454000073306F0CFFD924F054610B105233B70AF
:10455000FAE0904C216809B90E23F8E78E4806F07E
:10456000EAFA0FFA80F8B8F1010F0646F4DD2946A1
:1045700020688A4DFFF714FD89492860894807F0B3
:104580009BFC2968874807F0A0FC864807F0A4FC3C
:104590008549864807F090FC0A223146834807F097
:1045A000F4FC824807F098FC01212068FFF7F8FC32
:1045B000B8F1020F824600F0CA80022221687648D4
:1045C00006F0C1FAB8F1030FD0F8149000F0C180E2
:1045D00003212068FFF7E4FC0646102205A93620D7
:1045E000FFF77AFF002840F0B780B8F1040F40F3DE
:1045F000B38004212068FFF7D3FC6D490446694865
:1046000007F05AFC674807F067FC1FFA89F2514629
:104610005E4807F019F80DF1240866495B4807F079
:1046200016F80DF1340B1022634940460BF057FC8D
:10463000002301222021584602F0E6FC5F4958463B
:104640000BF0D5FB5E49574807F036FC51465548FC
:1046500007F03BFC5B49534807F02EFC0A22494611
:10466000504807F092FC58494E4807F025FC314667
:104670004C4807F02AFC55494A4807F01DFC33789E
:104680000BB91C461E46CDF80C804FF002094FF0C6
:104690000108CDE90198CDF800B0324623462968DB
:1046A0003A484B4E06F034FE002857D0494B4A4951
:1046B0003C4800241C6007F0FFFB2968394807F0DC
:1046C00004FC384807F008FC444B032283F80080C0
:1046D0004121234615A802F097FC414915A80BF08B
:1046E00086FB15A9294806F07DFF23464A4641214D
:1046F00015A802F089FC3B4915A80BF078FB15A919
:10470000394807F0F9FB15A9204806F06BFF23464E
:104710004246412115A802F077FC324915A80BF05A
:1047200066FB15A9304807F0E7FB15A9174806F006
:1047300059FFFFF74FFC05233B7008F0DBF82B49CE
:104740003060184807F0B8FB27B0BDE8F08F40F2A2
:104750005B790DF1130640E705AC56E7244925487F
:1047600007F0AAFB094806F074FF0A220146214817
:1047700007F00BFC20491F4807F09EFB1D4807F07F
:10478000ABFB08F0B7F80C233060E0E6BC03002078
:10479000B0030020B8030020540600205803002076
:1047A0009F3001008C030020712501004003002090
:1047B000AC300100653B000096320100DF320100A1
:1047C000CC300100242E0100EC300100DA31010070
:1047D00018040020FC030020F33001003E030020F9
:1047E0000131010005310100B00600200731010050
:1047F000243101005C03002030310100F8B5074E80
:1048000007460D1D0024E11915F8012B09B23046A9
:10481000013405F0F2FC042CF5D1F8BD180300209A
:1048200030B587B00023044600931A460D4602A80F
:10483000194607F001FB04A807F0F6FA042C12DD74
:1048400004A9286902F06FFB68B104A91220FFF7E0
:10485000D5FF04A9E86802F066FB50B104A90E2058
:10486000FFF7CCFF0BE002A91220FFF7C7FF032CD4
:10487000EFDC02A90E20FFF7C1FF022C17DD04A90F
:10488000A86802F050FB90B104A90A20FFF7B6FF18
:1048900004A9686802F047FB78B104A90620FFF775
:1048A000ADFF0D490D4807F007FB07B030BD02A969
:1048B0000A20FFF7A3FF012CEADC02A90620FFF77C
:1048C0009DFF012CEDD102A90620FFF797FF0449B7
:1048D000024807F0F1FAE4E7112A01008C030020F6
:1048E000012A01002DE9F041104F80460C460E1DB3
:1048F000002508EB050109B2384605F07CFC0135BE
:10490000042D06F8010BF4D1207958B1FF280BD102
:104910006379FF2B08D1A379FF2B05D1E079FF380C
:1049200018BF0120BDE8F0810120FBE7180300203B
:10493000F0B593B002A807F077FA04A807F074FA6C
:1049400006A807F071FA08A807F06EFA5849594806
:10495000594E07F0B1FA574807F0BEFA02A90620EF
:10496000FFF7C0FF00287CD054495248544C10AD8A
:1049700007F0A2FA039B10942846119302F01EFB45
:1049800004A90A20FFF7AEFF002861D04D4949482D
:1049900007F092FA059B11932846109402F00EFB43
:1049A00006A90E20FFF79EFF0EAF002843D0464910
:1049B000404807F081FA079B10942846119302F0B3
:1049C000FDFA08A91220FFF78DFF18B33F493948B7
:1049D00007F072FA099B11932846109402F0EEFA40
:1049E000039B3B493B480A94CDE90B34059BCDE939
:1049F0000D34079BCDE90F34099B1193CDE9007568
:104A00000CAB0AAA03F0BEFB2A4807F065FA0223A2
:104A100033703FE0039B0095CDE90D34059B2C4995
:104A20002C480C94CDE90F34079B11930CAA3B46FC
:104A300003F0C4FBE8E7039B254926480E94CDE923
:104A40000F34059B11933A462B4603F0E1FBDBE75D
:104A5000039B1F491F4810942A46119303F0F2FB51
:104A6000D2E71D49134807F027FA4FF47A6342F65C
:104A7000E0621749174803F023FB68B91749184843
:104A800007F01AFA1749164807F016FAF62333709A
:104A9000FFF7E8FB13B0F0BD1349064807F00CFA26
:104AA00010A80C4903F01FFC10A802F087FAAEE72B
:104AB000262E01008C030020B0030020332E0100BD
:104AC00078390100492E01004F2E0100542E0100BB
:104AD000B1030020E40500205B2E0100672E0100D9
:104AE0005C030020A92E0100D82E010010B53E4C19
:104AF0003E49204607F0E0F93D49204607F0DCF941
:104B00003C49204607F0D8F93B49204607F0D4F944
:104B1000204607F0E1F93949204607F0CDF9384938
:104B2000204607F0C9F93749204607F0C5F936494C
:104B3000204607F0C1F93549204607F0BDF9344950
:104B4000204607F0B9F93349204607F0B5F9324954
:104B5000204607F0B1F93149204607F0ADF9304958
:104B6000204607F0A9F92F49204607F0A5F92E495C
:104B7000204607F0A1F92D49204607F09DF92C4960
:104B8000204607F099F92B49204607F09EF92A495B
:104B9000204607F091F92949204607F08DF9284968
:104BA000204607F089F92749204607F085F926496C
:104BB000204607F081F92549204607F07DF9244970
:104BC000204607F079F92349204607F075F9224974
:104BD000204607F071F92046204907F06DF920467C
:104BE000BDE8104007F078B98C030020F82E0100D2
:104BF0001A2F01002D2F01003B2F0100432F010030
:104C0000502F0100602F01006C2F0100832F010045
:104C1000972F0100AC2F0100BB2F0100CA2F01000C
:104C2000D22F0100DD2F0100E72F0100EF2F01003F
:104C3000FB2F01003732010011300100303001003C
:104C40004530010052300100603001006C3001003D
:104C5000743001007F3001008C300100943001007D
:104C600008B5FFF743FFFFF727FB03490348BDE8FB
:104C7000084007F021B900BF2A2A01008C03002058
:104C800070B594B002F047F9064607F033FE0546CA
:104C9000234806F027FA00283FD0224B93F9004022
:104CA000002C3AD123460122402104A802F0ACF99D
:104CB0001D4904A80BF09BF81C4904A80BF097F8B9
:104CC0001B4904A80BF093F83146684602F01AFA23
:104CD00001236A4604A9124806F03BFC2346012240
:104CE000402104A802F090F90F4904A80BF07FF8C6
:104CF0000E4904A80BF07BF80E4904A80BF077F8D6
:104D000068464FF47A71B5FBF1F102F0FBF901232B
:104D10006A4604A9024806F01CFC14B070BD00BF2E
:104D2000BC03002088030020E6320100032D0100AF
:104D300044320100F53201002DE9F041144FDFF853
:104D40005C8000252E463C462946404605F053FA35
:104D5000E8550138C0B2FD2805F1010598BF0126CC
:104D6000062DF1D17EB90B490B4807F0A5F8DE23DB
:104D70002370AD236370BE23A370EF23E370FE2383
:104D80002371FF236371BDE8F041FFF78FB800BFC7
:104D9000B10300200E2C01008C030020180300201A
:104DA00008B54FF4E13006F029F81949194807F021
:104DB00083F81949194805F0BBFF1949194805F04E
:104DC000B7FF1949194805F0B3FF1949194805F00B
:104DD000AFFF1949194805F0ABFF1949194805F00B
:104DE000A7FF1949194805F0A3FF1949194805F00B
:104DF0009FFF1949194805F09BFF1949194805F00B
:104E000097FF19491948BDE8084005F091BF00BF58
:104E1000DA2B010040030020614C0000DE2B010072
:104E2000F53C0000E32B0100695F0000E82B010066
:104E3000DD5F000059330100213F0000ED2B010030
:104E4000B13C0000F12B01008D430000F62B010066
:104E500021480000FA2B0100AD440000FD2B0100A9
:104E6000513D0000012C0100D93C0000072C01003D
:104E70002DE9FF473E4E3368002B76D03D4D3E4F27
:104E80002B783C6801332B7007F034FD4FF0FF3373
:104E900001460F22204602F061F900283CD0336819
:104EA000DFF8E090DC68DFF8E0A07CB3237C03F05F
:104EB0000F03062B26D14A462146504605F04BFEED
:104EC000B8B1037C03F00F03052B12D1D0F80C808E
:104ED000B8F1000F16D02246414601A8FBF7DEFBD1
:104EE000022101A8FCF70EFA07F040FDD8F8048073
:104EF000EEE72146002201A8FBF7D0FB022101A822
:104F0000FCF700FA07F032FD6468CEE707F0F2FC28
:104F100038601A48FCF77AFA194C276807F0EAFC5F
:104F20004FF0FF33014641F28832384602F016F95D
:104F30002746B8B13368DC688CB1237C03F00F03DB
:104F4000062B08D12146002201A8FBF7A7FB01216F
:104F500001A8FCF7D7F907F009FD6468ECE707F052
:104F6000C9FC38602B78013B2B7004B0BDE8F0879A
:104F7000A80300203D03002014040020FC020020B0
:104F800020040020602501005406002010B5064CC6
:104F900023780133237007F0E9FCFFF769FF2378DA
:104FA000013B237010BD00BF8803002030B5104BBB
:104FB000196885B0C9B10F4CCD68227801322270D2
:104FC00085B12B7C03F00F03062B07D10022294665
:104FD00001A8FBF763FB01A8FCF7ECF907F0C6FC9E
:104FE0006D68EDE72378013B237005B030BD00BF4D
:104FF000A80300203D0300202DE9F043354E364D37
:105000003278013232702A688BB012B3D468334FD1
:105010002A68F2B1ECB1237C03F00F03052BF8D121
:105020002146384605F087FD0128F1D9214668461A
:10503000FCF7A8FC6846FCF737FC18B1022168466B
:10504000FCF7ECFE07F092FC68466468FCF7C6FAD1
:10505000DEE73378013B3370214B93F90030052BA9
:1050600035D0204E346807F045FC4FF0FF33014641
:105070004FF47A72204602F071F8804638B3DFF8B8
:10508000689000274C46D9F8001001B3FFB90B7C9B
:1050900003F00F03052B0ED16846FCF773FC0121CA
:1050A0006846FCF7BBFE18B107F024FC47463060A9
:1050B0006846FCF793FA23684BB107F057FC236866
:1050C0005B682360002BDED12B68DB6823600BB0AC
:1050D000BDE8F0833D030020AC030020540600200F
:1050E000B00300201C0400200804002070B580EAF2
:1050F000E074A4EBE0740E4605460121204607F05B
:10510000A5FD6EB1E943C90F204607F0C7FD074969
:10511000074806F0D1FE0648BDE8704006F0DCBE48
:10512000E90F204607F0BAFD0249F1E7D129010055
:1051300040030020D52901002DE9F04F2DED048B0F
:10514000884B93B01C6807F0D5FB4FF0FF33014646
:1051500047F23052204602F001F8002800F0ED80BE
:10516000814B1A68002A00F0E8808049D4680B78E7
:10517000DFF83CA29FED7E9A01330B700025002CD6
:1051800000F0C180237C03F00F03052B13D1002214
:105190002146504605F0D7FC4369052B0BD121462B
:1051A00008A8FCF7EFFB08A8FCF77EFB074620B930
:1051B00008A8FCF713FA6468E1E708A906A8FEF757
:1051C0002FF808A8FCF71EFB0021064608A8FCF7EC
:1051D00095FA054606A8FDF7FBFD08EE900A08A81B
:1051E000FCF706FA33B207EE903AF8EEE77A834618
:1051F00087EE898A08A8FDF793FB5E4980465E48E2
:1052000006F05AFE4FF0020918EE900A09F05EF817
:10521000CDF8009002460B46CDE90401564806F051
:1052200093FF5649544806F047FE18EE100A09F05D
:105230004DF8CDF8009002460B46CDE902014E48EC
:1052400006F082FF4E494C4806F036FE0A225946C7
:10525000494806F09AFE5FEA16494FD0082002F04E
:10526000D2F84FF6FF7381B240F62712484601F09C
:1052700075FFC8B12168434806F027FE42494148FE
:1052800006F01AFE41492268414806F04DF9B1B2D4
:1052900008A8FCF7CFFA00212846FFF727FF08A847
:1052A000FCF79CF93D4686E7DFED3A7AB4EEE78AF3
:1052B000F1EE10FA04DD22683749354806F034F97A
:1052C000B8F1000FE7D00022344BDDE9040108F00B
:1052D0009DFEDDE9022309F0E1FA014608B1012152
:1052E000DAE7F4EEC88AF1EE10FAD5D92C49224853
:1052F00006F0E2FD204806F0EFFDD0E729491E4800
:1053000006F0DAFDCBE7194A1378013B137007F07A
:10531000F1FA144B1860FFF7B3FC9DB1224916480F
:1053200006F0CAFD01F0F7FD0A220146124806F018
:1053300038FE1E49104806F0C8FD13B0BDEC048BC2
:10534000BDE8F08F19490C4806F0B6FD01F0E3FD09
:105350000A220146084806F024FE1449064806F0D1
:10536000ABFDEAE724040020AC0300203D0300204D
:105370000000C84228290100400300202E29010016
:10538000C72601005C0300203429010044290100E4
:10539000BC03002000001842502901000000F03F2B
:1053A0005D2901003A2901006C290100B83701008C
:1053B00054060020F0B5464E33688BB0002B00F049
:1053C000848044494448454C454D464F06F074FDA1
:1053D000414806F081FD94F90030ABB105F002FDC3
:1053E0002B781BB13B680BB101F0F0FB3E4B93F9FE
:1053F0000030052B01D0FFF7FFFDFFF79DFEFFF703
:1054000037FD07F0B3FAE6E738493348384D394FEE
:1054100006F052FD304806F05FFD2B68DC682B6813
:10542000E3B1DCB1237C03F00F03052B14D121463B
:10543000384605F080FB78B121686846FCF7D8FA59
:105440006846FCF731FA10B16846FCF7C1F807F07E
:105450008DFA6846FCF7C2F86468E0E7264B2749F6
:105460001D4800241C6006F027FD1B4806F034FD93
:10547000234B244918481C7006F01EFD01F04BFD1B
:105480000A220146144806F08CFD3168194804F0E0
:1054900051FF1D4B1D491C601D4B0F481C601D4BCF
:1054A00034601C600F4B2C601C6006F005FD01F0A1
:1054B00032FD0A220146084806F073FD064806F050
:1054C0000BFD154B1C70154B1C700BB0F0BD00BFD5
:1054D0000C040020CA310100400300203D030020DD
:1054E0000404002000040020B0030020DF3101008C
:1054F000AC0300205406002008040020F531010010
:1055000010040020FD310100A80300207A270100CB
:1055100028040020B80300203C0300203E030020A4
:105520002DE9F3410024214F0094234622462146D1
:105530001F48204E204D06F07FFC384602F0CAFF7F
:105540001E4804F055FE304603F0E4F931461C4E87
:105550000122284606F09EFB4FF0010800942B46DE
:1055600031460722174801F0E7FB2B463146CDF8BC
:1055700000800322144801F0DFFB2B460622009432
:105580003146124C124801F0D7FB4146114801F058
:1055900093FB3946204606F077F80F4A0F4920461C
:1055A00002B0BDE8F04107F039BC00BF7403002031
:1055B00024030020500400202C04002018030020A5
:1055C000B0060020400300205C030020BC03002044
:1055D0008C0300201C0300200000002055AE0000BA
:1055E000F7B53C4C2678002E6ED13B4B93F900303A
:1055F000012B69DD394D2B68002B65D040F202216B
:10560000374803F061F92968364A374805F0A3FAAC
:105610000546002858D00146334805F08CFA07B2F9
:10562000002F51D031462846FEF7BAFC012F06461E
:105630004CD0294601222C4805F085FA45692B49B2
:10564000684602F050FE10222949684601F090FC9D
:105650002849294806F030FC3146274806F035FC39
:105660002649254806F031FC0A222946224806F040
:105670008CFC2249204806F028FC1D491E4806F0F3
:1056800024FC1D4806F028FCAAB231461C481D4DDA
:1056900006F018FB16491A4806F018FB1A4B186852
:1056A00018B10021FEF77CFC2860296811B114486C
:1056B00006F014FB0021124806F018FB01231349E1
:1056C0000D48237006F0F8FB03B0F0BD40F2022550
:1056D000B5E700BF10040020B00300200C04002038
:1056E00050040020A229010054060020E4050020F7
:1056F0002C030020A92901008C030020242E010086
:105700002C04002058030020B8030020B829010011
:105710002DE9F04F7C4C21688DB0002900F0EE801F
:105720007A4F7B4A3B787B487B4D01333B7005F0D9
:1057300012FA7A4A28602168764805F00CFA784B0C
:10574000784A18602168734805F005FA764B774A65
:10575000186021686F4805F0FEF9754B1860FFF777
:105760003FFF744A21686B4805F0F5F9724BA94672
:10577000186030B3714D2B781BBBC468704801F0C2
:10578000FFF8002814BF012300232B7003D06D49BC
:105790006D4806F091FB6D4B00221A608CB12B789E
:1057A0007BB1237C03F00F03062B06D1206802A9EE
:1057B00001F02FFB02A801F01FFA07F0D7F8646888
:1057C000ECE7634A00231360D9F800309246002BBF
:1057D00000F08780D3F80C80DFF890B15D4CD9F8E9
:1057E0000030002B00F08D80B8F1000F76D098F8D3
:1057F000102002F00F02052AF3D14146454805F07A
:105800009AF90128EBD9414602A8FCF7BBF802A897
:10581000FCF74AF8A8B102A8FBF7C8FE064680B913
:10582000014602A8FBF76AFF051E02A8BCBF6D4235
:105830000126FBF7DDFE9DF81820052A09D0062A6F
:1058400026D007F093F802A8D8F80480FBF7C6FE2C
:10585000C5E718B9022102A8FBF7D8FE01212846A6
:1058600007F0F4F90021284607F018FA59462046B7
:1058700006F022FB29460A22204606F086FB36491E
:10588000204606F019FB3549204606F015FBD8E7FF
:1058900001900121284607F0D9F9019BD6B113F1F7
:1058A000FF3618BF01263146284607F0F7F92C4984
:1058B000204606F001FB0A222946204606F065FB39
:1058C0002849204606F0F8FA0A223146204606F01A
:1058D0005CFBD8E7013B5E425E41E4E7DB68CAF867
:1058E00000301C4806F0F8FAFFF760FBFEF75EFD9B
:1058F0001D4B01221A703B78013B3B700DB0BDE897
:10590000F08FDB68FFDE00BF0C0400203D030020A9
:105910007229010054060020AC0300201D31010053
:105920002804002078290100A80300207B29010019
:10593000B803002080290100000400200404002096
:10594000A53D0000832901008C030020B004002045
:1059500008040020400300209B290100A029010029
:1059600018270100912501003C0300209329010024
:1059700030B5BFB005460C461C22002112A811917B
:1059800009F0D9FA012D40F3B6801F22616811A8F1
:105990000AF0A5FA11A91620FEF764FD11A97348B3
:1059A00006F093FA7249714806F086FA6F4806F0DD
:1059B00093FA704A51791378049111790391D1784F
:1059C0000291917801915278009240216A4A19A877
:1059D0000AF04CF96949654806F06EFA11A9634866
:1059E00006F073FA19A9614806F06FFA5F4806F0ED
:1059F00073FA0CA802F06EFD614906A806F005FFD7
:105A000011AA0CA9502329A804F01AF94FF47A63BB
:105A100029A8399304F043F919A929A804F066FAD2
:105A2000044629A804F05FFA002C40F09C8029A8C5
:105A300004F06AFA29A9044609A804F07BFB09A925
:105A400006A806F02AFF09A806F09AFE29A804F085
:105A50001BF94C49454806F02FFA0A2221464348D3
:105A600006F093FA414806F037FAC82C79D1464936
:105A7000464806F021FA06A909A806F004FF09A97C
:105A8000424806F01DFA414806F026FA09A806F039
:105A900077FE3F493D4806F00FFA01F03CFA0A2232
:105AA00001463A4806F07DFA384806F015FAFFF745
:105AB00081FC3849354806F0FFF9344806F00CFA05
:105AC0003349324806F0F8F901F025FA0A22014676
:105AD0002E4806F066FA2D4806F0FEF906992E4883
:105AE00004F044FF2D4B1860D8B92D492D4806F01D
:105AF000E3F90E242AE0202211A91620FEF7ECFC7F
:105B000000287FF456AF2022274911A80AF0E7F9B0
:105B10002649164806F0D0F911A9144806F0D5F91F
:105B200044E72349194806F0C7F901F0F4F90A22BD
:105B30000146164806F035FA144806F0CDF9FFF78D
:105B4000E7FD1C49094806F0B7F904241A4B2993CC
:105B50003BA806F015FE06A806F012FE20463FB050
:105B600030BD1649C2E71649C0E700BF8C030020CC
:105B70009D2C0100B1030020C22C0100F12C01007A
:105B8000CE380100052D0100182D01004003002032
:105B90005C2D0100272D0100540600200C0400207C
:105BA0003D2D01005C03002069320100A42C01009E
:105BB000542D0100622D0100F4370100692D010010
:105BC000832D010010B52049204886B006F074F9F5
:105BD0001E4806F081F94C211D4804F00CFB7B287F
:105BE0002BD14FF0FF3203921A4A009200234C222D
:105BF000CDE90133CDE90423FFF7DCFB6946164804
:105C000004F0B0FE154B186040B91549154806F070
:105C100053F9144806F060F900200CE012490B48D3
:105C200006F04AF9094806F057F9FFF771FD0F48E9
:105C300002F036FD012006B010BD0D49034806F004
:105C40003BF90248E6E700BFC12D01008C030020AC
:105C50001803002088380100540600200C0400209E
:105C6000DC2D01005C030020E82D010074030020FE
:105C7000EF2D010030B58D4C94F900300B3393B00B
:105C8000192B2BD8DFE813F0B000A0002A002A005F
:105C90002A002A002A002A002A002A002A001A00C4
:105CA0003D004000490061006D0090002A002A007C
:105CB0002A002A002A00C100CE00DD007C4B7D486E
:105CC0001B78002B14BF0921012100F0F6FF7A4850
:105CD00002F036FB022801D0FEF72AFE94F90030CC
:105CE000012B40F3BD80744802F0C2FA0138042849
:105CF00000F2B680DFE810F0B800BD00C900D600A1
:105D0000AB0002232370E9E76C4D2B781BB9FFF73A
:105D100067FC01232B700323F4E7654B65481B7870
:105D2000002B14BF0B21032100F0C7FF644B93F934
:105D30000030002B40F0B880624B1978002941D127
:105D40000846FFF715FE2070C8E7594B59481B78E5
:105D5000002B14BF0B21032100F0AFFFFEF7E6FB81
:105D6000BCE7594B1D6806F0C5FD4FF0FF330146F7
:105D700041F28832284601F0F1F90028AED0002324
:105D80000322412101A801F03FF9504901A80AF07E
:105D90002EF801A94E4805F028FC06234D494E482F
:105DA000237006F089F899E7414B42481B78002B95
:105DB00014BF0A21022100F080FF454805F092F946
:105DC00000288BD104239DE706F094FD3E4B18601C
:105DD000F5232370364B37481B78002B14BF09215D
:105DE000012100F06AFF79E7374B1D6806F082FD5C
:105DF0004FF0FF33014641F28832284601F0AEF9F8
:105E000000283FF46BAF00237CE7314805F06AF9C6
:105E100010B12F4805F033F906F06CFD2A4B1860DD
:105E20000D236FE7284B1D6806F064FD4FF0FF332C
:105E3000014642F21072284601F090F90028C1D1C3
:105E40004CE7FFF7BFFE0028BCD1F6235AE72349F1
:105E5000234806F031F8224806F03EF8F623237076
:105E600094F9000013B030BD1E491D4806F024F817
:105E7000F4E71D49184806F01FF801A80E4902F082
:105E800032FA01A801F09AF8EAE71849144806F036
:105E900013F80F4805F026F90028DFD00C4805F06C
:105EA000EEF8DBE71249E5E70320DBE7B00300206B
:105EB0003C0300201C030020E4050020A403002074
:105EC0003D0300203E0300201804002001310100A2
:105ED000BC0300204A3101008C0300206131010025
:105EE0005C0300206A3101007E3101009B3101001A
:105EF000AE31010008B5164800F0E1FE06F036FDAF
:105F000004F070FFFFF7B6FE022802DD114805F02D
:105F100011FA06F02BFD104B1B7823B10F4B1B68B9
:105F20000BB100F053FE0E4B1B6853B10D4B93F9B0
:105F30000030052B01D0FFF75FF806F017FDFFF7E3
:105F4000FBF806F013FDBDE80840FEF791BF00BF67
:105F50001C030020BC0300200404002000040020D7
:105F6000AC030020B0030020FFF72CBE70B5FEF795
:105F700017FFFEF7BBFD144E144D46242146304654
:105F800004F039F92B1913F8463C834217D000214D
:105F90000846FDF7DDFEFEF7CFFE142006F0C4FC38
:105FA0000B4800F071FE0B490B4805F050FB4FF415
:105FB000FA7006F0B9FCBDE87040FFF703BE01348B
:105FC0004A2CDBD1E7E700BF18030020A332010011
:105FD000613B0000653B0000BC03002008B5FFF7F3
:105FE000C7FC034B18700348BDE8084002F058BBDB
:105FF000B00300207403002007B5002300931A4665
:106000001946034805F018FF03B05DF804FB00BF14
:106010007404002001207047014B1868704700BFCE
:1060200084040020032070477047000010B5044628
:106030000B490C4805F060FFA17C94F9080006F0BC
:106040002DFEA17C94F9090006F028FE606800216D
:10605000FBF7F0FB044B00221A60012010BD00BFCB
:106060005D330100B006002084040020F7B56E46C1
:106070000546304686E80600FDF77EF804463046C1
:10608000FCF76DFE10B1002C08BF01244FF48051C5
:106090006868FBF7EDFA012C1CD0022C04D044BB3D
:1060A0002049214805F008FF3046FCF75DFE002836
:1060B00036D06868FBF7A6FB18B90124204603B068
:1060C000F0BD00206C6801F09EF901462046FBF708
:1060D000B1FBF2E730466F68FCF7BEFF0146384679
:1060E000FBF794FA3046FCF7B7FF01280AD00228E4
:1060F00008D00E490C4805F0DFFE0B4805F0ECFE19
:106100000024DBE76868FBF77DFB0028D5D0002082
:106110006D6801F078F901462846FBF78BFBCDE767
:106120000446CBE719330100400300202A33010065
:1061300010B5044606F034FC204610BD2DE9F043AE
:106140004FF4805185B004464068FBF781FA00287F
:1061500000F0AF804FF400516068FBF779FA68B93E
:106160008D4D95F90030002B00F0A3804FF40051C5
:106170006068FBF77DFA2B78013B2B706068FBF7BA
:1061800041FB00221146814602A8FCF799FC00223F
:10619000616802A8FCF7FEFF002102A8FCF7F0FEF0
:1061A00080466068FBF724FA022801D0052801D157
:1061B0004FF0000894F90A00A0F10E03DBB2072BA0
:1061C00000F2CF8006F04CFCFF25E289218A009581
:1061D0000023074606F0BBFA061EC0F2BE80AE42A0
:1061E00000F3BD80B9F1000F40F0C180A8EB0605B7
:1061F00007E06A496A4805F05FFE694805F06CFEF1
:1062000000256849664805F057FE0A2294F90A10ED
:10621000634805F0BAFE6449614805F04DFE0A2264
:1062200039465F4805F0B1FE60495D4805F044FE1F
:106230000A2231465A4805F0A8FE5D49584805F043
:106240003BFE0A224146564805F09FFE59495448F4
:1062500005F032FE0A222946514805F096FE5048C4
:1062600005F03AFE15F10A0F2CDA94F90900A17C29
:1062700006F014FD6068FBF7C5FA30B9666801F0F6
:10628000C2F801463046FBF7D5FAA37C6842A3B1B9
:1062900000210091FF23192206F059FAFF28014638
:1062A000A8BFFF21462994F90800B8BF462106F08F
:1062B0007BFC002005B0BDE8F083FF220092194668
:1062C0001922E9E70A2D27DD94F90800A17C06F0E0
:1062D000E5FC6068FBF796FA30B9666801F093F860
:1062E00001463046FBF7A6FAA37C83B1002100915A
:1062F000FF233322284606F02AFAFF280146A8BFCA
:10630000FF214629B8BF462194F90900CFE7FF22B3
:10631000009219463322EDE72749284805F0ECFDA5
:10632000A17C94F9080006F0B9FCA17C94F909005D
:1063300006F0B4FC00216068FBF77CFA4FF4805152
:106340006068FBF7B7F94FF400516068FBF7B2F9EA
:10635000114A137801331370ABE7002642E72E464B
:1063600040E74FF0FF37B9F1000F10D03E4606F07E
:10637000C1FA4FF0FF330146B4F90C20484600F053
:10638000EDFE00287FF435AF731C7FF42FAFA8F12A
:106390007F054FF0FF3634E704000020363301005C
:1063A000400300204433010048330100032D010065
:1063B000102501004E33010056330100B0060020C5
:1063C000002110B5044681744068FBF797F943B289
:1063D000002BBBBF4042207223720123B8BFA374BD
:1063E000237A6068013B122B84BF20232372012192
:1063F000FBF784F943B2002BBBBF4042607263726B
:106400000123B8BFA374637A6068013B122B84BF79
:10641000212363720221FBF771F9C3B2132B8ABFE8
:106420000023A072A37203216068FBF767F980B2B2
:10643000431EB3F5806F26BF0023E381E081042172
:106440006068FBF75BF980B2B0F5806F8ABF4FF4EC
:1064500080632082238205216068FBF74FF900B238
:106460000028D6BF42F21073A081A38110BD0000A6
:1064700010B50446F9F7BFFF2046FFF7A1FF184902
:10648000184805F039FD94F90800012106F0DEFBFB
:1064900094F90900012106F0D9FBA17C94F90800C8
:1064A00006F0FCFBA17C94F9090006F0F7FB94F9D7
:1064B0000A00002106F0CAFB60680021FBF7BAF968
:1064C00060684FF48051FBF7F5F860684FF40051B5
:1064D000FBF7F0F8044B01201860044B187010BD56
:1064E0006B330100B006002084040020040000206B
:1064F00007B5002300931A461946034805F09CFC93
:1065000003B05DF804FB00BF7C040020014B186859
:10651000704700BF900400200020704770470000C3
:1065200010B51A4904461A4805F0C6FC184805F08B
:10653000D3FC236820465B6B9847012805D00228CE
:106540000AD00021B4F9080019E003212046FAF727
:106550000FF8002106F07AFB00212046FAF708F830
:10656000002106F073FB01212046FAF701F8002113
:1065700006F06CFB02212046F9F7FAFF002106F035
:1065800065FB044B00221A60012010BDCD330100D1
:1065900040030020900400202DE9F041044688B01B
:1065A00040689DF8383002AE86E8060000286ED0BC
:1065B000B4F90820002A69D0002B6BD00021FBF72A
:1065C0009DF8236880465B6B2046984705B2022DF4
:1065D00051D0032D2BD0012D0CBF0521012100220C
:1065E00004A8FCF76DFA4FF0FF33009396E80C0017
:1065F00004A906A8FCF79AFF012D3ED0022D38D140
:106600009DF81610B4F9080006F0CEFA01212046D4
:10661000F9F7AEFF9DF8151006F0C6FA02212046E4
:10662000F9F7A6FF9DF8141006F0BEFA21E04FEA34
:10663000D8713046B4F90870FCF7A2FC0146054653
:10664000384606F0B1FA1449144805F035FC0A2220
:10665000B4F90810114805F098FC11490F4805F0ED
:106660002BFC0A2229460D4805F08FFC0B4805F04B
:1066700033FC01200BE00421B1E703212046F9F7A8
:1066800077FF9DF8171006F08FFAB9E7104608B0AB
:10669000BDE8F0811846FAE7182701004003002002
:1066A0009125010010B5044606F07AF9204610BD88
:1066B00038B50446F9F79FFE1D491E4805F0FCFB5E
:1066C0001C4805F009FC606870B3B4F9083063BB7E
:1066D000236820465B6B98470128054605D00228B1
:1066E0000AD00121B4F9080019E003212046F9F786
:1066F0003FFF294606F0AAFA00212046F9F738FFA5
:10670000012106F0A3FA01212046F9F731FF01210A
:1067100006F09CFA02212046F9F72AFF012106F033
:1067200095FA054B0120186038BD0020FCE700BF3A
:10673000DA330100400300209004002010B5044625
:106740004068E0B1B4F90A30032B10D0042B17D005
:106750000A22017C0F4805F031FC0F490D4805F075
:10676000ABFB0C4805F0B8FB6368187C07E00B49ED
:10677000084805F0A1FB074805F0AEFB022010BD5C
:106780000749044805F098FB024805F0A5FB0120E5
:10679000F5E700BF40030020BF330100BC33010018
:1067A000C433010007B5002300931A461946034875
:1067B00005F042FB03B05DF804FB00BF8804002035
:1067C0002DE9F04F85B006F095F8604902906048D9
:1067D00005F088FB5F4B18689A4608B101F066F82F
:1067E0005D4C5E4F2568386800210BB2AB4201F169
:1067F0000101C0F294805A4DDFF88091DAF8000070
:10680000002800F0938021682B6803EBC10101F0A0
:10681000DDF9002840F38A802368132B00F386807B
:1068200006F068F84FF0FF33014641F288320298D3
:1068300000F094FC0646002878D12B6820680721D8
:1068400003EBC00001F022F82B680193019A236842
:1068500002EBC30B9BF807208242CFD10FFA86F8D8
:106860004345039325DD019B082203EBC8005946ED
:1068700008F02EFB0136039B0028EFD13968019008
:1068800031F81830374843F0010321F81830364901
:1068900005F012FB2B682068019A03EBC000082169
:1068A00000F066FA31492F4805F01CFBB8F1000FE3
:1068B000A4DAD9F80030002BA0D03B682268294820
:1068C000012123F812102A4905F0F6FA0A2221685C
:1068D000244805F05AFB2749224805F0EDFA2B68B9
:1068E0002068002203EBC000082100F041FA1D4897
:1068F00005F0F2FA22682B6803EBC20113F832307C
:10690000282B08D10C22D9F8000001F092FADAF80D
:10691000000001F0A5F82368013323606EE730F82A
:10692000132022F0010220F813205EE712490D48DF
:1069300005F0C2FA0A2221680A4805F026FB094838
:1069400005F0CAFA012005B0BDE8F08FDE34010081
:10695000B00600209C040020B0040020B8040020F1
:10696000B404002040030020F7340100FE3401008D
:10697000053501000A350100E8340100A8040020B3
:10698000F8B5424D2B6807460BB1012054E0404951
:106990004048414E05F090FA3E4805F09DFA3F49C7
:1069A0003C4805F089FA00F0B6FA0A220146394857
:1069B00005F0F7FA374805F08FFA142005F0ECFFE0
:1069C000044600F02DFFA0202C6005F0E7FF3449BD
:1069D00030603048334C05F06FFA00F09CFA0A2220
:1069E00001462C4805F0DDFA2A4805F075FA282002
:1069F00005F0D4FF2C492060264805F05DFA00F030
:106A00008AFA0A220146234805F0CBFA214805F00C
:106A100063FA33680BB123687BB92449244805F035
:106A20004BFA00F078FA0A220146214805F0B9FA3B
:106A30001F4805F051FA0020F8BD1E4B1E481F608C
:106A400000F054FD286800F005FF0446B8B11B496A
:106A5000104805F047FA286801F040F8286800F06F
:106A600005FF17490B4805F03DFA286801F07AF850
:106A700000288AD01349074805F034FA85E71249FF
:106A8000044805F02FFA2046D6E700BF9C040020FA
:106A90003F34010040030020B40400205C2D0100BD
:106AA00060340100B80400206C3401007934010026
:106AB0005C030020A0040020280500209134010080
:106AC000A4340100C4340100D03401002DE9F041A8
:106AD000364E306800F0B6FE02280DD134493548F4
:106AE00005F0EAF9334805F0F7F9306801F03AF8B3
:106AF00042F21070BDE8F0812F4C304F2568EDB99F
:106B00001C2005F049FF31682D4E804601F0F4F855
:106B10004046C4F8008001F0CFF93A6820682BB2F3
:106B2000934205F1010506DA31680C2201EBC3013D
:106B300001F07FF9F1E7002101F012FA214E3A68E5
:106B4000B6F900309342374606DBFFF739FE0023E3
:106B500033804FF4FA50CDE7194D286800EBC3019C
:106B600010F8330028281AD1206801F089FA164B52
:106B70001B6802462BB1B6F90000296801EBC00181
:106B800098472B68B7F90010206803EBC10101F0AA
:106B90001DFA3B8801333B8040F6C410AAE701335D
:106BA0004FF4FA60338090FBF2F0A3E79C040020DE
:106BB0003034010040030020A8040020B00400206D
:106BC000B4040020AC040020A004002038B5094C17
:106BD000256805F08FFE4FF0FF33014641F2883201
:106BE000284600F0BBFA20B1FFF770FF05F082FEE7
:106BF000206038BDA404002070B51C4C2368132B02
:106C000032DC1B4A1B4D1268012122F8131029683F
:106C1000026841F8332001EBC306426872601649EE
:106C2000164805F049F90A222168144805F0ADF923
:106C30001349124805F040F92B682068002203EB45
:106C4000C000082100F094F80C4805F045F92268CE
:106C50002B6813F83230282B03D10A4B186800F048
:106C6000FFFE23680133236070BD00BFB004002025
:106C7000B8040020B40400200535010040030020C2
:106C80000A3501009C040020034B0146186808B136
:106C900000F0D6BD704700BF9C04002007B500235C
:106CA00000931A461946034805F0C6F803B05DF88C
:106CB00004FB00BF94040020704770477047704782
:106CC00007B5002300931A461946034805F0B4F8A7
:106CD00003B05DF804FB00BFBC040020134B1B781D
:106CE00070B505460C4673B1114A0A291368164659
:106CF00011D1104A0021D154006910B1298905F041
:106D000061F800233360E86870B1036821461B68AE
:106D1000BDE8704018474E2BF5DC0D291FBF591CEC
:106D20001160044AD454EEE7012070BD1004002025
:106D3000CC040020D004002030B50025456003615C
:106D4000034D9DF80C300560C1600281037530BDB4
:106D50001C35010007B5002300931A461946034865
:106D600005F06AF803B05DF804FB00BFC40400201E
:106D7000F8B5441E0D4D16466718BC420ED014F8E7
:106D8000011F10220909284605F0FFF8217810227A
:106D900001F00F01284605F0F8F8EEE726B10348A8
:106DA000BDE8F84005F098B8F8BD00BFB006002077
:106DB00070B501380C4D13464618B04203F102037A
:106DC0000CD010F8014F24112C5D03F8024C04780C
:106DD00004F00F042C5D03F8014CEEE709B2002328
:106DE00002F8113070BD00BF5A350100A0F16103F7
:106DF000052B02D85738C0B27047A0F14103052BCC
:106E000001D83738F7E73038C0B20A2828BF002049
:106E1000704738B50139841C00F1120514F8020CD2
:106E2000FFF7E4FF0001C2B201F8012F14F8010CD2
:106E3000FFF7DCFF02341043AC420870EED138BDDE
:106E400038B50546D8B10468ACB124789CB128683F
:106E500003783BB12D2B05D0303B092B02D90130F3
:106E60002860F4E707F0F0FD2C210446286808F0BC
:106E7000CDFF10B92860204638BD0130FAE704463E
:106E8000F9E72DE9F34100220D4606210646FBF7FE
:106E900017FE85B32B6873B31B7863B32868037838
:106EA0003BB12D2B05D0303B092B02D90130286096
:106EB000F4E707F0C9FDD5F8008007462E214046CB
:106EC00008F0A4FFD8B144782F2C18D9392C18D841
:106ED000303C2C21404608F099FFA0B92860A4B1AD
:106EE0000A22002F02FB07F2D8BF64422244314637
:106EF0006846FCF7E0F8304602B0BDE8F0810024B7
:106F0000E7E70924E5E70130E8E73A463146684615
:106F1000FCF7C5F8EFE708B5002009F099F9ADEBEB
:106F2000000008BD704730B5441E224612F8013FEC
:106F3000002BFBD11A460A2514F8010F70B1032A61
:106F400014DC2E2806D1FF2B10DC881801320371C7
:106F50000023F1E7303805FB0303EDE7FF2B04DCEA
:106F6000032A02DC114401200B7130BD0020FCE734
:106F70002DE9F3410024DFF840800C700D461746E0
:106F8000061D0A2201A916F8010B07F06CFF3A460C
:106F900001A9284608F07DFF032C04D03A4641465B
:106FA000284608F076FF0134A3B2042B1CB2E8D1C6
:106FB000284602B0BDE8F081DD3101002DE9F04145
:106FC0000E4D0F4FDFF83C8006460024032C0ED0F8
:106FD00033190A221979284604F0B5FF414628469C
:106FE000013404F069FF042CF0D1BDE8F081F1799F
:106FF0000A22284604F0A7FF3946F0E740030020A4
:107000003D350100DD3101002DE9F047DFF8F0A04A
:10701000DAF8005004460E4617469946002D49D02E
:107020002B7C03F00F03062B43D12C4A2C48294616
:1070300003F091FD022F804637D0032F37D1294A24
:10704000DAF80010264803F086FD0546B8F1000F77
:1070500030D098F8103003F00F03042B2AD1D8F861
:1070600014103246204608F03AFF32461E492046A8
:1070700008F00FFF0DB32B7C03F00F03042B1CD182
:1070800069693246204608F004FF32461649204618
:1070900008F0FFFEB9F1000F04D032464946204601
:1070A00008F0F7FE2046BDE8F087104AC8E7002543
:1070B000CCE7002532460E49D4E7022F0AD0032F31
:1070C00005D0012FE1D10B4B32461968DAE7324681
:1070D0000949D7E732460949D4E700BF50350100D6
:1070E00054060020A3360100032D01005535010090
:1070F00074350100580300206E3501006B35010026
:107100002804002030B585B0002301AA0A2541B12A
:10711000B1FBF5F405FB14113031D1542146013394
:10712000F5E71A44411EC41812F8015D01F8015F29
:10713000A142F9D10022C25405B030BD10B5054CB2
:107140000549204604F0C1FE2046BDE8104004F089
:10715000C3BE00BF4003002040350100024410B50B
:10716000B2FBF3F404FB13238B420DD2884206D901
:10717000012003E0884294BF0020012010BD984206
:107180002CBF00200120F9E79842F3D30020F5E757
:107190002DE9F04399B002AE0F4686E80C00044694
:1071A00030B1037C03F00F03052B03D0062B13D063
:1071B00000201DE07E4DC4682A7801322A703CB15F
:1071C000204696E80C003946FFF7E2FF6468F6E7D0
:1071D0002B78013B2B70EBE70146764A764803F0AB
:1071E000BAFC054638B196E80C003946FFF7D0FFE7
:1071F00019B0BDE8F083714A6F48214603F0ABFC3B
:107200006F4A814621466C4803F0A5FC804677B161
:10721000012F5CD02C460023102200930DEB0201BD
:107220004FF440733046FCF70BF805461BE0654A07
:107230006148214603F08FFC0546634A5E482146BB
:1072400003F089FC0746002D5BD02B7C03F00F0375
:10725000042B56D16C69002FDDD03B7C03F00F036B
:10726000042BD8D17D69B9F1000F5CD0D9F8141086
:107270005648002C47D004F028FE5549534804F0E6
:107280001BFE2146514804F020FE504804F024FE25
:107290003046FCF7D1F8B8F1000F47D199F810301B
:1072A00003F00F03042B7CD1D9F8141008A8FAF7C7
:1072B0009FFB08A8FAF7F8FA28B15CB30022214630
:1072C00008A8FBF78BF908A8FAF788F969E0414AA2
:1072D0003948214603F03FFC3F4A054621463648DF
:1072E00003F039FC0746002D5DD1364A324821466D
:1072F00003F031FC0546002F9FD00028A5D104469D
:10730000ABE70024A7E704F0E0FD31492F4804F083
:10731000D3FDBDE70123009396E80600234608A8A5
:10732000FAF79AFDCFE7B8F1000F3AD0D8F8141069
:10733000264804F0CAFD2649244804F0BDFD29462C
:10734000224804F0C2FD214804F0C6FD2DB398F890
:10735000103003F00F03042B1FD14022D8F8141073
:1073600008A808F0BCFD1D4803F0BCFEA8B11C4BEA
:1073700093F900308BB92F2108A808F047FD30B9E8
:10738000D8F814300322402108A8FFF73DFE01235E
:107390002A4608A9114804F0DCF8B9F1000F7FF47F
:1073A0007DAF012024E700287FF44FAF45E700BF01
:1073B0003D030020602501005406002064250100E3
:1073C0009E250100243501002935010040030020DD
:1073D000383501002E35010033350100BC03002093
:1073E0008803002073B500226C4605460E462046F1
:1073F0001146FBF765FB94E80C0031462846FFF781
:10740000C7FE02B070BD10B5044605F073FAE04047
:1074100008BF012010BD000007B5002300931A46E5
:107420001946034804F008FD03B05DF804FB00BFF3
:10743000200500202DE9F84380460D46174601EB54
:1074400002090C464C45A4EB05060BD0D8F80030D9
:1074500014F8011B1B68404698470028F2D13046BB
:10746000BDE8F8833E46FAE77047203004F097BE47
:10747000203004F086BE203004F097BE38B5437F3C
:107480000D460BB9002038BD00F16804204604F019
:1074900094FE0028F6D12046294604F063FE012020
:1074A000F1E700002DE9F0411E4600254FF47A7304
:1074B000C0E901530C4B044640F8203B8846174670
:1074C00004F047FE04F1680004F043FE9DF8183014
:1074D00063769DF81C302676C4E90487A376657729
:1074E0002046BDE8F08100BF84350100817E284A36
:1074F0000123C37670B552F82140417E52F8211025
:107500004FF0A04504F5E07401F5E07140F20C661F
:1075100045F8246045F8216001694FF0CC74C1F84A
:10752000244501690624C1F80045847E016952F8AA
:107530002440C1F80845447E016952F82420C1F86E
:107540000C2590F91820510902F01F029340603178
:10755000104A42F8213090F91830002BBDBF03F0DB
:107560000F0302F6FC32D2189B18B5BF402340220D
:10757000137683F8002390F918300122590903F09B
:107580001F0302FA03F3034A42F8213070BD00BF23
:107590000839010000E100E02DE9F0410446884689
:1075A0001F461546002A50D000F12006304604F050
:1075B000E4FD2369C3F88885236901221A622369DF
:1075C000C3F834652369C3F8385523691A60226902
:1075D000D2F84C311BB9D2F82431002BF8D000235B
:1075E000C2F84C312269D2F85C311BB9D2F824318F
:1075F000002BF8D00023C2F85C3122696FB9D2F8B1
:10760000243153B90123D3612369D3F84821002AD7
:10761000FBD00022C3F8482109E00123536123690C
:10762000D3F80421002AFBD00022C3F804212369E7
:10763000D3F8242112B10022C3F824212369D3F8FE
:107640003C052066C0B2BDE8F0811046FBE701238F
:10765000FFF7A2BF10B5044680F8B010683004F000
:107660008CFD0123637710BDF8B5002343770369D0
:1076700090F8B020C3F88825036901261E620369CB
:1076800000F168050446C3F8445528460F4604F047
:1076900086FD2369C3F8480523699E602369D3F8F2
:1076A00050211AB9D3F82421002AF8D00022C3F8B7
:1076B0005021284604F073FD236930B1D3F86021CE
:1076C0001AB9D3F82421002AF8D00022C3F8602187
:1076D00023696FB9D3F8242152B90122DA612369F1
:1076E000D3F84821002AFBD00022C3F8482109E042
:1076F00001225A612369D3F80421002AFBD0002219
:10770000C3F804212369D3F8240168B10022C3F827
:1077100024212369D3F8C404C3F8C404022803D085
:1077200004280CBF03200420F8BD0121FFF79CBFF3
:1077300070B54369D3F86421044692B10022012553
:1077400000F12006C3F864210577304604F015FDEA
:107750006369C3F8346563694022C3F838256369F7
:107760001D636369D3F86821DAB10025C3F8685155
:1077700004F16806012363772577304604F0FDFCA9
:10778000D4F8B43003B19847636965773046C3F8DD
:10779000446504F004FD6369C3F848056369012288
:1077A0005A636369D3F8042162B10022C3F804214B
:1077B000237F3BB16369D3F83C05D4F8B830206629
:1077C00003B198476369D3F8242152B10022C3F86A
:1077D00024216369D3F8D024C3F8D024636901223B
:1077E0005A6170BD0148FFF7A3BF00BF2805002004
:1077F00007B516231722CDE900324FF040220423AB
:1078000011460348FFF74EFE03B05DF804FB00BFCE
:10781000280500200148FFF788BF00BF2805002089
:1078200010B54FF4C05303800023044683700361F6
:107830000248FFF75BFE204610BD00BF2805002070
:10784000016170478078704741780148FFF702BFB7
:107850002805002008B5FFF7F7FF0348FFF765FF8D
:10786000B0FA80F0400908BD28050020012303700C
:107870007047FF23C37200230373C3700371437106
:107880008371C371037243728372704710B5064AE5
:1078900001440023884204D010F8014B6340D35CBC
:1078A000F8E7184610BD00BF9C350100FFF7E1BFA7
:1078B00038B5084C0D46FFF7C7FFE1212046FFF71A
:1078C000DDFD29462046FFF7D9FDBDE83840FFF72A
:1078D000A1BF00BF2805002010B5054C417801224A
:1078E0002046FFF7B4FE2046FFF7C2FDC0B210BD30
:1078F0002805002010B5F0210446FFF7D9FF2046E7
:10790000BDE81040FFF7E8BF70B5054604F0F2FF90
:10791000002400F57A7604F0EDFFB04246D2284606
:10792000FFF7E8FFC307044646D52B6903B1984724
:107930001420013800BF00BF00BF00BF00BF00BF60
:1079400000BF00BF00BF00BF00BF00BF00BF00BF3F
:1079500000BF00BF00BF00BF00BF00BF00BF00BF2F
:1079600000BF00BF00BF00BF00BF00BF00BF00BF1F
:1079700000BF00BF00BF00BF00BF00BF00BF00BF0F
:1079800000BF00BF00BF00BF00BF00BF00BF00BFFF
:1079900000BF00BF00BF00BF00BF00BF00BF00BFEF
:1079A00000BF00BF00BF00BFC3D1B4E70123AB706D
:1079B0000249034804F0A0FA204670BD9C3601003D
:1079C000B006002010B5E1210446FFF771FF204604
:1079D000BDE81040FFF780BF10B50446FFF794FFE5
:1079E0002046FFF731FF96210648FFF747FDFFF7D6
:1079F00011FF2046FFF788FF2046BDE81040FFF743
:107A0000E1BF00BF28050020FFF7E6BF10B5C32186
:107A10000446FFF74DFF2046BDE81040FFF75CBF6E
:107A200038B504460D46FFF76FFF2046FFF70CFF01
:107A3000D2210A48FFF722FDE94345EA0111C9B204
:107A40000648FFF71BFDFFF7E5FE2046FFF744FF62
:107A5000A8421CBF0423A37038BD00BF2805002026
:107A600010B50446FFF7D2FF40F00401C9B220462A
:107A7000BDE81040FFF7D4BF70B5164604460D466A
:107A8000FFF742FF16B12046FFF7EAFF2046FFF757
:107A9000DBFEA5210548FFF7F1FC29460348FFF767
:107AA000EDFCBDE87040FFF7B5BE00BF2805002023
:107AB00070B500220C4655210646FFF7DDFF651E16
:107AC000073415F8011F00223046FFF7D5FFA54205
:107AD000F7D170BDFFF7ECBFFFF7CEBF10B504467E
:107AE000FFF7B2FE20460022F021FFF7C5FFBDE8F8
:107AF0001040FFF78FBE000070B5164605460C46D5
:107B0000FFF702FF16B12846FFF7AAFF2846FFF746
:107B10009BFE87210648FFF7B1FC002C0CBF2146D5
:107B200080210348FFF7AAFCBDE87040FFF772BE52
:107B30002805002010B5002204460121FFF7DCFFD4
:107B40002046FFF7E1FEC0F3401010BDFFF7F2BF83
:107B500010B50446FFF75AFF20460021BDE810404B
:107B6000FFF75EBF38B50446FFF7CEFEC30729D442
:107B70002046FFF7EDFF2046FFF7C6FE2046FFF741
:107B800063FEB4211048FFF779FCFFF743FE20465F
:107B9000FFF7BAFE10F00403054602D00223A370DB
:107BA00002E0A278022AFAD0237843B12046FFF7F8
:107BB0002DFF40F00101C9B22046FFF731FFC5F3A8
:107BC000400038BD0020FCE7280500202DE9F74FD4
:107BD000057B04460F46002D7AD1FFF7C3FF40B95D
:107BE0003C493D4804F088F94FF0FF3003B0BDE850
:107BF000F08F2046FFF788FE2A46F0212046FFF747
:107C00003BFFDFF8DC804FF0FF394FF0010A94F9B9
:107C10000B30EEB24FEAD60B9D4206F007060AFA89
:107C200006F62CDA04EB0B03DB7833402046019395
:107C3000FFF76AFE2046FFF707FE78214046FFF770
:107C40001DFC019B002B0CBF194680214046FFF70D
:107C500015FCFFF7DFFD2046FFF756FE82060146C2
:107C600000F040030FD59BB102221B4804F0A6F997
:107C70001A49194804F040F96FF00100B6E70CBF4B
:107C800001230023D2E71BB9080658BF4FFA85F934
:107C900004EB0B03090693F9032076B205F1010505
:107CA0004CBF3243B243402DDA70B0D1B9F1FF3F3F
:107CB00004BF0123237384F80B90E31C013F0B34B2
:107CC00013F8012B07F8012FA342F9D101208DE70A
:107CD00000208BE7A7360100B0060020B336010074
:107CE0002805002008B5FFF771FF20EAE070C0B258
:107CF00008BDFFF737BF7047054A82610022027155
:107D0000027009224270012281608270C270704745
:107D1000F77C000010B50C4620460721FFF7B6FDA2
:107D2000E3791B1A5842584110BD70B5044680686B
:107D30000E461546FFF7DDFFB8B13146A068FFF7E4
:107D4000C9FE0022BE21A068FFF7C6FE6E1E0835E0
:107D5000A068FFF759FE06F8010FAE42F8D1A068FF
:107D6000FFF7C7FF431E5842584170BD10B5144677
:107D7000FFF7DBFF38B108212046FFF787FD237AA4
:107D80001B1A5842584110BD70B504460D46806814
:107D90001646FFF7AEFF2946A068FFF79BFE0022BC
:107DA0004E21A068FFF798FE0022B178A068FFF787
:107DB00093FE0022F178A068FFF78EFE2B78102B3F
:107DC00004D000223179A068FFF786FEA068FFF793
:107DD00090FF2946A068FFF77DFE2278A068482121
:107DE000FFF77AFE142004F09FFD237813B10A20D8
:107DF00004F09AFDA068BDE87040FFF77ABF38B57F
:107E000004460D468068FFF774FF2946A068FFF717
:107E100061FE0022B421A068FFF75EFEA068FFF7B4
:107E200095FE0546A068FFF764FFB5FA85F04009A6
:107E300038BDF0B585B0144601AA07460E46FFF7D7
:107E400095FF054690B13378102B0FD00B2C10D036
:107E50000C2C03D00A2C0ED13F2300E07F2301AA73
:107E6000314638468DF80830FFF78EFF284605B0BA
:107E7000F0BD5F23F3E71F23F1E71FB50B78102B4D
:107E800010D001AAFFF772FF78B19DF808303F2BA0
:107E90000ED003D81F2B0DD0002006E05F2B03D09F
:107EA0007F2BF9D10C2000E00B2005B05DF804FB1E
:107EB0000A20FAE70920F8E72DE9F04387B00446E5
:107EC00004F018FD00F51C55A068224F224EDFF883
:107ED0008C80FFF7EBFC00231035237101A9A0680B
:107EE000FFF700FF90B304F005FDA8422ED201A9D0
:107EF0002046FFF70FFF20B34146304603F0E5FF71
:107F0000237833B901A92046FFF779FF08B101238F
:107F1000237003AA01A92046FFF707FF01A9204605
:107F200094F80190FFF7A9FF814505D9607823797E
:107F3000607001332371D1E701A92046FFF79DFF4F
:107F4000F5E73946304603F0C0FFC7E707B0BDE8A4
:107F5000F08300BFC6360100B0060020C436010021
:107F6000817070471FB501AAFFF7DFFE9DF804007E
:107F7000003018BF012005B05DF804FB0939C9B213
:107F80000229F8B598BF104B0546164694BF33F941
:107F9000114040F2EE248AB1C3787BB103786BB90B
:107FA00004F0A8FC074631462846FFF7DBFF20B95E
:107FB00004F0A0FC001BB842F5D3F8BD2046BDE894
:107FC000F84004F0B1BC00BFBE360100F8B504466D
:107FD0000F46FFF752FF064610B900252846F8BDA8
:107FE000A068FFF786FE0028F7D03946A068FFF7A3
:107FF00071FD2278A0684421FFF76EFDA5782DB1B0
:108000003A4631462046FFF7B9FFE7E70125E5E7A5
:1080100010785378C00040EAC3200B78102B00B2D0
:108020000BD1D1799379C000CB1ADB0120F07F000E
:1080300093FBF1F3103B184400B2704730B585B0A4
:1080400001AA04460D46FFF791FE30B101AA294668
:108050002046FFF7DDFF05B030BD0148FBE700BF5C
:1080600080E4FFFF10F5DC5FCABF07EE900ADFED8A
:10807000037AFAEEEC7A17EE900A70470000FEC21F
:1080800008B5FFF7DBFFBDE80840FFF7EBBF0423AF
:1080900002461946012000F03FBE0423024619465D
:1080A000052000F039BE024606230421092000F015
:1080B00033BE0423024619460F2000F02DBE0000F7
:1080C0002DE9FF41044600690E461746984608B15F
:1080D00004F066FC782004F05FFC7822054600215D
:1080E00006F029FF05F1540000F014FC217D256104
:1080F000234800F067FE00253046FFF7D4FF2B46EB
:108100002A462946009502A803F096FE03A8FFF729
:10811000D0FF29462E2000F02DFE10F001052BD0B7
:1081200043463A463146206901F059FA012805468E
:1081300022D1216902A800F078FF03A8FFF7B9FF58
:10814000216902A800F07FFF03A8FFF7A0FF2169C3
:1081500002A800F071FF03A8FFF79FFF216902A8A2
:1081600000F078FF039B6360206900F07AFFA06055
:10817000206900F078FFE060284604B0BDE8F08197
:1081800027060020F8B504460F46017D0A4816462A
:108190001D4600F017FE3846FFF785FF301DFFF73C
:1081A00088FF06980430FFF772FF07980430FFF746
:1081B00074FF6B686360F8BD27060020F0B58DB0D2
:1081C0001E46002317460093FF2304460D461A4619
:1081D000194602A803F030FE7A680C4B0493CDE9EF
:1081E00005237268CDE90723129A5268CDE9092365
:1081F000039B0B930AAB019308AB009304AA06AB55
:1082000029462046FFF7BEFF0DB0F0BD78390100CA
:1082100010B554685B680A4A8AB0CDE90732012379
:1082200003948DF80F30039B099308ABCDE9042428
:108230000692009304AA06ABFFF7C0FF0AB010BD78
:10824000783901007FB5094B52680493CDE90232B9
:10825000012301928DF80730019B059302AA04AB1C
:10826000FFF7D6FF07B05DF804FB00BF78390100C7
:1082700037B5044600212E2000F07CFDC3072ED523
:10828000206970B301F0C4F90228054601D0042822
:1082900022D12169684600F0C8FE01A8FFF709FF56
:1082A0002169684600F0CFFE01A8FFF7F0FE2169C2
:1082B000684600F0C1FE01A8FFF7EFFE216968469D
:1082C00000F0C8FE019B6360206900F0CAFEA06058
:1082D000206900F0C8FEE060284603B030BD0525E7
:1082E000FAE70546F8E710B5044603F09DFD0423C0
:1082F000E21800210F2000F00BFE204610BD10B543
:10830000044603F091FD0423E2180021052000F04B
:10831000FFFD204610BD10B5044603F085FD042383
:10832000E2180021012000F0F3FD204610BD0000FE
:10833000024A02604A684260704700BF7839010013
:1083400008B5017D064800F03DFD00212E2000F01B
:1083500011FD10F0010F0CBF0220012008BD00BF6D
:108360002706002037B500240A4D009423462146F5
:108370002246094803F060FD284603F055FD0A2314
:108380002B75064B2C611878012103B0BDE83040F5
:1083900004F05CBCE4050020FC050020260600205B
:1083A00008B503681B6B984780F00100C0B208BD98
:1083B00013B502AB026803F8011D54681946012287
:1083C000A04702B010BD007C083818BF01207047DC
:1083D000037C087C984203D1083818BF01207047FD
:1083E0000020704770B590B0044604A815460E46AC
:1083F00003F01AFD07A800F08DFA684603F014FD9B
:108400000D4902A8FFF794FF02A904A801F04BF957
:108410006A46314604A801F0F7FA012809D1236819
:10842000064A9B690292019A039202A92A462046B3
:10843000984710B070BD00BFE405002078390100F6
:1084400038B50546007C0828144604D101236B602A
:108450000024204638BD92B200F052FB0028F5D02F
:10846000F7E7000008B5017C082903D0024800F0B6
:108470000BFD08BD0020FCE72706002007B5012200
:108480000DF10701007C00F07DFB0028CCBF9DF8BA
:1084900007004FF0FF3003B05DF804FB08B512B2DF
:1084A000007C00F06FFB08BD036813B59B680446B1
:1084B000984740B10DF10701207C00F091FB9DF839
:1084C000070002B010BD4FF0FF30FAE7007C00F06B
:1084D00095BB000000214FF47A72C0E90112024AF4
:1084E000026008220274704708370100017C0829E5
:1084F00006D04901083101F0F801032000F03ABC30
:10850000002070472DE9F84F0E46017C08290446EB
:10851000174609D00A22594803F050FD58495748D8
:1085200003F0EAFC002099E05448DFF86CA1DFF882
:108530004C9103F0D1FC00255FFA85FB4FEA4B110B
:10854000083101F0F801032000F014FC5146804688
:10855000484603F0BAFC10222946484603F015FDB0
:108560004849484603F0B1FC10224146484603F012
:1085700027FDB8F1000F04D008F0FB08B8F1180F80
:1085800043D1414984F810B03C4803F09EFC1022CE
:10859000217C3A4803F014FD237C082BC2D03B4DCC
:1085A000DFF8D8802B88DFF8F4A001332B8004F0AB
:1085B000A1F92B8853FA80F080B2B0F5806F36BFF6
:1085C0004FF4806328802B802A88207C002301219F
:1085D00000F03AFAF51C06F1070915F8011F0A2206
:1085E000404603F0EBFC5146404603F06EFC4D451F
:1085F000F3D1224803F070FC3A46311D207C00F094
:108600004BFA30B9082323748CE70135082D93D138
:10861000C2E704F06FF900F56A55064618352046A2
:10862000FFF764FF17281BD0AE4219D204F062F99D
:1086300085421AD90A2004F077F9FCF7A7FC2046F6
:10864000FFF754FF0028DDD02046FFF74FFF172823
:10865000E5D10F49094803F04FFC0120BDE8F88F30
:1086600004F048F90028E5DBE0E70A49034803F095
:1086700043FC236820465B6A984753E7B006002016
:10868000CF360100E2360100EB3601000600002083
:10869000F43601009F360100DE360100DD310100B5
:1086A00038B50446007C082826D000F021FA04F0F2
:1086B00021F905462046FFF719FF48B104F01AF9E1
:1086C000401BB0F57A7F03D2012004F02DF9F1E7C9
:1086D0002046FFF70BFF10B1207C00F0A7F9227CA9
:1086E000064B0748002123F812100823237405497C
:1086F000BDE8384003F000BC38BD00BF04060020D0
:10870000B0060020C836010010B5037C082B0446D3
:1087100016D0FFF7EBFE182806D80A4B23FA00F014
:10872000C04300F0010010BD1C2807D1236820467B
:108730009B689847003018BF0120F4E70120F2E75A
:108740000020F0E70100100107B5002300931A464E
:108750001946034803F070FB03B05DF804FB00BF4B
:108760001406002003681B6B18470000024A0260D1
:108770008A694260704700BF78390100808B70477A
:10878000008C704713B502AB026803F8011D5468F2
:1087900019460122A04702B010BD10B50446238C33
:1087A00023B123682046DB689847F8E710BD000036
:1087B00010B50446007C082808D000F037F9227C68
:1087C000034B002123F812100823237410BD00BFAF
:1087D000040600200023C3830431007C00F02CBA7F
:1087E000007C00F041BA10B593B204460A46C18B32
:1087F000007C00F005FAE38B0344E38310BD13B55E
:10880000038C04461BB94FF0FF3002B010BD0122AB
:108810000DF10701007C00F0B5F90028F3DD238C91
:108820009DF80700013B2384EFE710B5038C044655
:1088300013B94FF0FF3010BD934294BF1AB212B279
:10884000007C00F09FF90028F3DD238C1B1A2384A1
:10885000F1E707B5038C4BB10DF10701007C00F087
:10886000BFF99DF8070003B05DF804FB4FF0FF303F
:10887000F9E7000013B5036804465B699847217C5B
:10888000104800F001FBD0B108226946207C00F0BE
:1088900079F9002813DD694604F1140003F0E0FAC9
:1088A0009DF804209DF805309DF8070003EB022396
:1088B000A3839DF8063000EB032080B2208402B031
:1088C00010BD00BF27060020F8B5037C082B044626
:1088D0000E4601D00020F8BD0025EFB27901083125
:1088E00001F0F801032000F045FA60B92774207CFC
:1088F0000828EFD00023668223843246022100F04C
:10890000A3F80120E7E71828F0D00135082DE4D1BD
:10891000EDE7000010B500224FF47A73C0E901239F
:10892000044B0360082304460374143003F07CFAFC
:10893000204610BD4837010070B590B0044604A829
:1089400015460E4603F070FA07A8FFF7E3FF6846E6
:1089500003F06AFA0D4902A8FFF7EAFC02A904A88D
:1089600000F0A1FE6A46314604A801F04DF8012846
:1089700009D12368064A1B6A0292019A039202A94E
:108980002A462046984710B070BD00BFE40500207D
:108990007839010007B5002300931A4619460348A9
:1089A00003F04AFA03B05DF804FB00BF1C06002088
:1089B00040010C300A46042300F0FC010C2000F0BA
:1089C000ABB90B464101083101F0F801184600F03F
:1089D000D1B908B50221FFF7F4FF08BD0B464101EC
:1089E0000C3101F0FC01184600F06EB938B50A0AE6
:1089F00005460C460421FFF7F1FFE2B205212846A7
:108A0000FFF7ECFF38BD08B50A460221FFF7E6FF85
:108A100008BD38B50A0A05460C461021FFF7DEFFEF
:108A2000E2B211212846FFF7D9FF38BD10B5014643
:108A300004461022034800F0DAFAFF212046FFF72F
:108A4000E2FF10BD27060020F8B51F464B1E042B81
:108A500004460E46154619D8FFF7E8FF46EA070216
:108A600000212046FFF7BAFF55B129462046FFF7FF
:108A7000BDFF07480122214600F0B9FA0120F8BDE8
:108A8000044B1988013189B21980EFE70020F6E71D
:108A9000270600202406002038B50B78FF2B05465A
:108AA00014460AD14B78FF2B0ED18B78FF2B0BD1BC
:108AB000CB78FF2B08D1002014E02BB94B781BB9E1
:108AC0008B780BB9C87868B16CB12846FFF770FF96
:108AD00021462846FFF79DFF04480422294600F05E
:108AE00086FA012038BD2046FCE700BF270600209B
:108AF00001460822014800F07ABA00BF270600208C
:108B0000B2F5006F2DE9F04128BF4FF40062DFF8A5
:108B1000708004460E4615462146404600F096F900
:108B2000032107462046FFF74CFF172801D01C28D9
:108B30001FD1AF42F0D33246214611482B4600F0F8
:108B4000DEF9202221460E4800F051FA2046FFF7B8
:108B500040FFC3060FD403212046FFF732FF06462D
:108B60000028F3D12046FFF761FF35462846BDE8CF
:108B7000F0810025DFE710212046FFF744FFF5E7ED
:108B800027060020F7B505460E460146134817464E
:108B900000F07AF904B274B903212846FFF711FFF7
:108BA000142805D020B1B0F11C0418BF4FF0FF34D9
:108BB000204603B0F0BDBC42A8BF3C46002CF7DD08
:108BC0000023009332462946A3B2044800F0E4F99A
:108BD00040222946014800F00AFAE9E7270600206A
:108BE00013B501240A46009401462346024800F0CA
:108BF000D3F9204602B010BD2706002070470000C0
:108C0000F7B505460E4601460A481C46174600F0D1
:108C10001DF9A04204D22946064800F017F904467F
:108C200000943B4632462946024800F03DF9204672
:108C300003B0F0BD2706002038B50B780546144672
:108C40002BB94B781BB98B780BB9C87840B144B1BC
:108C50002846FFF7ADFE28462146FFF7DAFE012041
:108C600038BD2046FCE7000038B501460446202206
:108C70000C4800F0BCF92046FFF7ABFE10F01005E1
:108C80000AD12046FFF7A5FE0307F4D52046182198
:108C9000FFF7B9FE284638BD20461021FFF7B3FE86
:108CA0000120F8E727060020024B0021187803F086
:108CB000F5BF00BF26060020024B0121187803F003
:108CC000EDBF00BF26060020F8B5114C114B05463C
:108CD0000F46204616460ECB04F06AF8FFF7E4FF75
:108CE000290A204604F071F8E9B2204604F06DF834
:108CF0003946204604F069F83146204604F065F80C
:108D0000FFF7DAFF204604F05FF80120F8BD00BF4E
:108D10002407002028060020F8B51D46134B064600
:108D20000F46134814460ECB04F042F8FFF7BCFF81
:108D3000310A0F4804F049F8F1B20D480C4E04F026
:108D400044F839460A4804F040F8013C6719BC422F
:108D500005D014F8011F304604F037F8F7E7FFF7A5
:108D6000ABFF034804F030F82846F8BD2806002081
:108D70002407002070B5114B114C05460E462046C5
:108D80000ECB04F015F8FFF78FFF290A204604F0F8
:108D90001CF8E9B2204604F018F83146204604F0E9
:108DA00014F80021204604F010F80546FFF784FF70
:108DB000204604F009F8284670BD00BF28060020B0
:108DC0002407002038B5174B174D1A7829703AB38D
:108DD00000244FF4FA601C7003F0A6FD01212878EE
:108DE00003F034FF114803F0CDFF21462046FFF782
:108DF000C1FF60F07F02D2B204212046FFF764FF7A
:108E000065010C35EDB2022229461E20FFF75CFFFA
:108E10000134022229461F20FFF756FF082CEFD10C
:108E200038BD00BF080000202606002024070020CF
:108E300038B520210546FFF7C4FD000284B2212188
:108E40002846FFF7BEFD204480B238BD70B50E46FF
:108E500000243046FFF7ECFF054618B13046FFF717
:108E6000E7FF0446AC42F4D1204670BD38B5262158
:108E70000546FFF7A6FD000284B227212846FFF72A
:108E8000A0FD204480B238BD70B50E4600243046A7
:108E9000FFF7ECFF054618B13046FFF7E7FF044641
:108EA000AC42F4D1204670BD2DE9F0410E4630466B
:108EB000242115469846BDF81870FFF782FD25213C
:108EC00004463046FFF77DFD284400EB042084B2C1
:108ED0007101204614313C443B464246A4B201F0A5
:108EE000FC01FFF719FF220A24213046FFF776FD27
:108EF000E2B225213046FFF771FDBDE8F08107B5EC
:108F0000009313460022FFF7CFFF03B05DF804FB88
:108F1000F8B506460F461D46144632B3144B1548A5
:108F20000ECB03F045FFFFF7BFFE310A114803F0F7
:108F30004CFFF1B20F4803F048FF39460D480D4F82
:108F400003F043FF6B1E661E1C44A64206D00021A0
:108F5000384603F03AFF06F8010FF6E7FFF7ACFEDC
:108F6000044803F031FF2846F8BD1546FBE700BF73
:108F7000280600202407002082B01046ADF8060025
:108F800049011A46BDF80600BDF80830183101F055
:108F9000F80102B0FFF7BCBF2DE9F7430E4680464B
:108FA0002821304691461D469DF82870FFF709FD9F
:108FB000000284B229213046FFF703FD0444A4B225
:108FC00000954B46224631464046FFF7D5FF5FB934
:108FD0002C44A4B2220A28213046FFF7FFFCE2B25B
:108FE00029213046FFF7FAFC03B0BDE8F08310B545
:108FF0000C4620460121FFF7F1FC01212046FFF736
:10900000E0FC0028F9D110BD044B4FF000421A607B
:1090100000229A6002221A71704700BF28060020C1
:10902000142200210E3005F086BF10B50E31044623
:1090300002F00EFF204610BD10B51C31044602F0B0
:1090400007FF204610BD10B52031044602F000FF96
:10905000204610BD10B52831044602F0F9FE204626
:1090600010BD406970478069704730204B1C087004
:10907000110902F00F02092A94BF3032373203F887
:1090800001290A460029F3D17047000007B50023E3
:1090900000931A461946034802F0CEFE03B05DF86D
:1090A00004FB00BF340600202DE9F0418EB00446D9
:1090B000884616460021202206A805F03CFFFF2323
:1090C0001A461946009302A802F0B6FE04F15405B0
:1090D000574B04934322039B059304A92846FFF7AB
:1090E00079FB013000F0A180524B069363688DF844
:1090F00021601BBA0793330A8DF820301C2280238D
:1091000006A926462846ADF82230FFF76CFB1A2246
:1091100000210DF11E0005F00EFF56F8080F069015
:10912000B388ADF81C30102206A92846FFF75BFB78
:109130002022002106A805F0FEFE0627202206A90F
:109140002846FFF750FB013FF8D13B4B069340F216
:109150003513ADF81C303D238DF81F3007238DF8F3
:10916000203001238DF821303368CDF82230B388C8
:10917000ADF8263031498DF81E8040F60C430DF1D4
:109180002A00ADF8283006F058FEE27A0CA92046F5
:10919000FFF76BFF227B0DF132012046FFF765FFE1
:1091A000627B0DA92046FFF760FF1E2206A9284614
:1091B000FFF719FBB8F1030F28D140F23243ADF8A5
:1091C0001830A37B8DF81A30E37B8DF81B30237C9D
:1091D0008DF81C30637C8DF81D3040F23643ADF8BD
:1091E0001E3094F824308DF8203094F825308DF816
:1091F000213094F826308DF822300C2294F8273054
:109200008DF8233006A92846FFF7EDFA0C4A0D4BDE
:1092100006A9CDE906232846FF2309228DF8203030
:10922000FFF7E1FA2846FFF7DBFA0EB0BDE8F08160
:109230007839010001010600638253638837010019
:1092400037060103060F3A3B2DE9F0478CB005467F
:109250008846174603F04EFB05F1540406462046A7
:10926000FFF708FB002809DC03F044FB801B4045A6
:1092700000F21081322003F057FBF0E7242203A90B
:109280002046FFF7D2FA9DF80C30022B40F0FD800B
:10929000B5F87030432B40F0F880049E36BA3E603B
:1092A000062205F108010AA805F012FE28B92B686C
:1092B0009E4202D36B689E4207D92046FFF76DFAA3
:1092C000002630460CB0BDE8F087079BC5F80E308D
:1092D000CC262046FFF793FA013EFAD1B04605F1BD
:1092E00024092046FFF74CFA002840F3CF8020469F
:1092F000FFF785FA0F2800F0818025DC032850D085
:109300000FDC0028EDD0012841D02046FFF777FA86
:10931000C7B2013FFFB2FF2FE3D02046FFF76FFA3D
:10932000F7E7062853D00C28EFD12046FFF767FA5D
:10933000C7B2781C05F0AAFD3A460146A86120464E
:10934000FFF773FAAB6967E0362868D00CDC332886
:1093500000F08D803528D8D12046FFF750FA2046FE
:10936000FFF74DFAC6B2BCE73B2873D0FF28B8D050
:109370003A28CAD12046FFF742FA042205F130010B
:109380002046FFF752FA2B6B1BBA2B63A9E7204646
:10939000FFF735FA042205F11C012046FFF745FAD4
:1093A0009FE72046FFF72BFA0422074605F120012C
:1093B0002046FFF73AFAFFB24FF0000A043F574544
:1093C0008FDD2046FFF71BFA0AF1010AF7E7204676
:1093D000FFF715FA0422074605F128012046FFF79A
:1093E00024FAFFB24FF0000A043F57457FF779AFE8
:1093F0002046FFF704FA0AF1010AF6E72046FFF7D4
:10940000FEF9C7B2781C05F041FD3A460146686195
:109410002046FFF70AFA6B6903F8078061E72046E8
:10942000FFF7EDF96B6A07468BB1494601A802F0D8
:109430000FFDEA6E029B9A4209D0FFB2013FFFB2D4
:10944000FF2F3FF44EAF2046FFF7D9F9F6E704228D
:109450004946A2E72046FFF7D2F9042205F134017C
:109460002046FFF7E2F96B6B1BBA6B6339E72046C6
:10947000FFF7C5F9042205F12C012046FFF7D5F9C5
:10948000EB6A1BBAEB62AB632BE700262046FFF7C3
:1094900084F916E7FF2614E72DE9F34704464FF455
:1094A000FA61012003F049F92746606047F8540B40
:1094B0003846FFF77DF944213846FFF705FA0028C2
:1094C00000F08B8003F016FA4FF00009804600256B
:1094D0004FF0030A94F85030032B1CD02BBB636869
:1094E0000133636003F006FA4FF47A72A0EB0800D0
:1094F0000121B0FBF2F2204692B2FFF7D5FD012325
:1095000084F85030002DE5D103F0F4F9636CA0EB42
:1095100008009842DBD93846FFF74AF963680133FF
:109520006360284602B0BDE8F087042B11D1636860
:109530000133636003F0DEF94FF47A72A0EB0800A8
:109540000321B0FBF2F2204692B2FFF7ADFD0223F9
:10955000D6E7012B19D101AAA16C2046FFF774FEB2
:109560000228064636D1019B636003F0C3F94FF42D
:109570007A72A0EB08000321B0FBF2F2204692B20F
:10958000FFF792FD84F85060BCE7022BBAD101AA24
:10959000A16C2046FFF758FE0528064615D1E36A60
:1095A00084F850A013B94FF46173E362236B13B9CD
:1095B000E36A5B082363D4E90C320AB95A00626398
:1095C000A363636BE363012584E7062802D184F873
:1095D000509097E7FF2EFAD094E70546A1E7F8B53B
:1095E00000250F460446C0E90B554563C0E91052FB
:1095F000836485608581FFF713FD3B68A360BB88AA
:10960000A38184F850502046BDE8F840FFF744BFDE
:1096100038B5044603F06EF90546206C00283ED0AC
:10962000E26CA91A17D44FF47A7005F57A7291FB9F
:10963000F0F300FB1311521A0133E264A26B5900DC
:109640008A42ACBFD21A0022A263E26B9142CCBF25
:109650000023D31AE36394F85030032B1DD1A36B7E
:10966000002B1ADC042384F850302046FFF714FF47
:10967000013094F85030032B00D063B9E36B002B1A
:1096800009DC002384F850302046FFF7C9FC20464F
:10969000FFF702FF0330256438BD0020E9E705F538
:1096A0007A73E364F7E74B684360002303817047F4
:1096B00030B50139084610F8013F002BFBD11C469C
:1096C0000A2511F8010F70B1032C14DC2E2806D1E5
:1096D000FF2B10DC1019013403710023F1E730383F
:1096E00005FB0303EDE7FF2B04DC032C02DC224423
:1096F0000120137130BD0020FCE7000007B50023F6
:1097000000931A461946034802F096FB03B05DF831
:1097100004FB00BF3C0600202DE9F74305460E463A
:1097200003F0E8F805F10C04288105F10801022294
:1097300002AD2046FFF757F8012325F8023D02222B
:1097400029462046FFF74FF84FF48073022229463E
:109750002046ADF80630FFF746F8002302222946DE
:109760002046ADF80630FFF73EF802222946204693
:10977000FFF739F8022229462046FFF734F837462A
:109780003378E3B13E46B04618F8013B0BB12E2BBF
:1097900013D1A6EB0709B9F1000F0CDD01220DF181
:1097A000050120468DF80590FFF71DF84A46394619
:1097B0002046FFF718F84746E2E74646E3E702A9E6
:1097C000012201F8033D2046FFF70DF84FF48076A3
:1097D000294602222046ADF80660FFF704F802226F
:1097E00029462046ADF80660FEF7FDFF012003B0D4
:1097F000BDE8F0832DE9F04387B006460F4690465A
:1098000003F078F806F10C0405462046FFF732F81D
:1098100000280BDC03F06EF8401BB84200F2EA802F
:10982000322003F081F8FBF7B1FBEEE7726A736850
:109830009A4240F0E280338D352B40F0DE802046A6
:10984000FEF79EFF0B2840F3DB800C220DEB02019C
:109850002046FEF7EAFFBDF80E203189130A43EADD
:109860000223BDF80C201BB29DB29142ADF8065008
:1098700001D1002B07DB2046FEF78FFF4FF6FC706F
:1098800007B0BDE8F08340F20F231D4005D020460D
:10989000FEF783FF4FF6FB70F2E7BDF812301F0AA8
:1098A00047EA0327BFB2AFB92046FEF776FF4FF66F
:1098B000FA70E5E79DF80A309BB92046FEF79FFF56
:1098C0002046FEF79CFF2046FEF799FF2046FEF754
:1098D00096FF0135BDF810305BBAAAB29BB29A422E
:1098E00014DA01220DF10A012046FEF79EFF9DF8D1
:1098F0000A30002BDED09DF80A305A1E8DF80A205F
:10990000002BD7D02046FEF77AFFF4E70026B146B9
:1099100001220DF105012046FEF787FF9DF8053075
:1099200013F0C00F0AD193B19DF805305A1E8DF87F
:10993000052043B12046FEF762FFF5E72046FEF71B
:109940005EFF8DF805909DF80530002BE0D10222D6
:1099500002A92046FEF769FF02220DF10A01204606
:10996000FEF763FF2046FEF74AFF2046FEF747FF5B
:109970002046FEF744FF2046FEF741FF02220DF18C
:1099800006012046FEF751FFBDF80830B3F5807F91
:1099900018D1BDF80A0040BA85B2012D12D1BDF828
:1099A000062052BA92B2042A05D02046FEF7F5FEF0
:1099B0004FF6F77064E708F104012046FEF735FF23
:1099C00028465DE70025BDF806305BBAAAB29BB217
:1099D0009A4205F1010503DA2046FEF710FFF2E78F
:1099E0000136B6B2B74293D12046FEF7D6FE4FF607
:1099F000F67045E74FF6FF7042E74FF6FE703FE71F
:109A00004FF6FD703CE700002DE9F341054688461E
:109A10001746FFF74DFE044600283BD1204B6A68ED
:109A20005B689A4238D002F065FF05F10C0600F041
:109A30000F0101F580613046FEF746FF01281CD179
:109A4000184B009335226B68019369463046FEF748
:109A5000C1FE78B141462846FFF75EFE50B1304660
:109A6000FEF7BEFE30B13A4641F288312846FFF794
:109A7000C1FE04463046FEF79BFE0B490B4802F040
:109A800024FA0A222146094802F081FA204602B04F
:109A9000BDE8F0810124F9E76FF00104F6E700BFAB
:109AA0003C060020783901008F370100B006002005
:109AB000006903681B691847006903685B691847F8
:109AC00013B5006949680368034C01919B690094D0
:109AD0006946984702B010BD7839010000690368F3
:109AE000DB691847006903689B6A18470069003002
:109AF00018BF01207047006C70470164704710B5B3
:109B000090F83830044633B920690368DB68984719
:109B1000002808DA10BD03689B6898470028F3D135
:109B20004FF0FF30F6E794F82220A2F10803022B51
:109B3000F0D8A36A002BC2BFE36A0133E3620A2AAA
:109B4000E8D1E36B013BE363002BE3D1092384F805
:109B50002230DFE710B50446006903681B6A9847A6
:109B600094F82230083B022B07D8A36A002B04DDAF
:109B70000028A2BFE36A1B18E36210BD73B590F81A
:109B80002230092B04460ED10026206903689B6809
:109B9000984740B120690368DB689847C5B20A2D31
:109BA0001CD184F8225094F822300A2B04D1E36BA4
:109BB00013B9092384F8223094F82230092B22D0DB
:109BC000206903689B68984794F822300A2B03D1D8
:109BD000E36B9842A8BF184602B070BD0D2DD4D0DB
:109BE000284605F01FF90028CFD0E06BADF80460DF
:109BF00010228DF804500021050101A806F086FA14
:109C00002844E063C1E70020E6E7000000234FF0AE
:109C1000FF32C0E90A23084A80F822301268026342
:109C2000064A4362126880F83830C36347F2305303
:109C300042630364704700BF10000020140000203E
:109C400038B504461D4600204FF47A73C4E9010379
:109C50000B4B2360C4E9041204F1180002F0E4F88D
:109C60000123258484F8443084F84530054904F103
:109C7000480002F0CAFD2046FFF7C8FF38BD00BF0C
:109C8000F4370100CE38010010B5044600690368BE
:109C90005B6A98472046BDE81040FFF7B7BF012335
:109CA00080F822307047000038B504460069154638
:109CB00002F00BF90449206902F007F929462069EE
:109CC000BDE8384002F018B9DF36010038B5044667
:109CD0000D460069114602F0F8F81D49206902F0AE
:109CE000F4F82946206902F0F0F81A49206902F0D8
:109CF00003F994F84530F3B16369B3B116492069AB
:109D000002F0E3F8D4E9040102F0DFF8238C502BD1
:109D100008D01249206902F0D8F80A22218C206963
:109D200002F033F9206902F0D7F80D4B0D491A689B
:109D30002046FFF7B9FF94F8443023B10A4A0B4993
:109D40002046FFF7B1FF012384F82230002038BD00
:109D5000B8370100BA370100C4370100242E0100D2
:109D60000C000020CB370100D6370100DC370100A2
:109D700038B504460069154602F0A7F80549206980
:109D800002F0A3F8294620690A22BDE8384002F013
:109D9000FEB800BFDF36010010B50446006902F0CE
:109DA0009BF8022384F8223010BD70B590F8223061
:109DB000012B04460D46164601D8FFF7EDFF20693A
:109DC0000368324629465B68BDE87040184770B5A5
:109DD00090F82230012B04460D4601D8FFF7DCFF36
:109DE0002069036829461B68BDE87040184710B514
:109DF0000446206903689B68984720B1206903687E
:109E0000DB689847F5E710BD2DE9F347994690F8D0
:109E10002230083B022B04460E469246DDE90A78C2
:109E200004D8FFF7E4FF2046FFF7F0FE94F8225035
:109E3000012D44D894F8443063B1D4E90401228C54
:109E40000368002934D121490091E16901919B699E
:109E500069462EE0206903689B6A98470028ECD089
:109E6000314652462046FFF731FF0646E0B9B9F1C8
:109E7000000F04D04A4616492046FFF715FF002F71
:109E800020DD3A4613492046FFF772FFB8F1000F74
:109E900018D001252046FFF77FFF2DB123683A46F1
:109EA0005B68414620469847304602B0BDE8F087DF
:109EB000DB6998470028D3D14FF0FF36F4E76FF005
:109EC0000106F1E7002DEFD1E4E700BF783901008A
:109ED00094370100A137010090F82230012B01D8FE
:109EE000FFF75ABF7047FFF7F7BF000007B5002321
:109EF0004FF0FF32CDE90023024AFFF785FF03B0A0
:109F00005DF804FBE73701002DE9F04790F82230B7
:109F1000012B044651D9DFF8D88000250327002300
:109F20006362022384F8223002F0E4FC4646824653
:109F30004FF00A090A2D46D002F0DCFC236CA0EB9E
:109F40000A00984245D2236820469B68984748B348
:109F500023682046DB689847431C0546ECD094F8FC
:109F60002230022B05D0032B0FD002F0C3FC824617
:109F7000E0E733782A2B01D083421AD17278731C20
:109F80000AB984F822701E46EFE7A0F13002092AD0
:109F900095BF636A042309FB032384F8223098BF2A
:109FA0006362E2E74FF47A7002F0BEFCC2E70A2D6A
:109FB00006D16FF00300BDE8F0876FF00100FAE70B
:109FC0006FF00200F7E7636AC72B02DC652B18BF4E
:109FD000002594F82230042BE9D1606AC72801DCFF
:109FE00065289CD10A2D18BF6FF00200E3E700BF7F
:109FF000B037010010B503680446DB68984794F851
:10A000002230A3F10802022AC0B232D9052B31D086
:10A01000072B39D0042B54D1226B137883420BD1F8
:10A02000531C2363537823B9C4E90A33052284F807
:10A0300022200A281DD136E0636B197881420BD1AA
:10A040005A1C62635B78002BF3D1012384F838300B
:10A05000062384F82230ECE71B4909688A42F7D1CD
:10A060001A4A12689342F3D10D28F1D1072384F8DC
:10A07000223010BDA0F13002092AE9D8A36A0A21D2
:10A0800001FB0323A362D4E70A28F2D194F8383005
:10A090009BB1092384F822300023E36394F8223033
:10A0A000083B022BE5D9042384F82230064B1B68B9
:10A0B0002363064B1B686363DBE7082384F82230C5
:10A0C000ECE70A28D5D1E9E71000002014000020B1
:10A0D00038B5044602F00EFC054694F82230083BE1
:10A0E000022B13D902F006FC236C401B98420DD2C0
:10A0F000236820469B68984718B12046FFF77AFFEF
:10A10000E8E74FF47A7002F00FFCE6E794F82230AB
:10A11000083B022B94BF00206FF0020038BD10B541
:10A1200090F82230083B022B044601D9FFF7D0FFFC
:10A13000A06A10BD7FB5054608460E46FFF7EFFF43
:10A140001649044601A802F060FB002C0EDD2146F2
:10A1500001A802F033FB48B90021284602F055FB64
:10A1600001A802F00DFB284604B070BDF36AA342BB
:10A1700009D0304602F064F9431C04D0C1B201A8F2
:10A1800002F0AAFBE7E7002C02DD039B9C42E3D12F
:10A1900001A9284602F0E5FAE2E700BFCE38010047
:10A1A00038B590F82230083B022B054601D9002033
:10A1B00038BDFFF7B4FF0130F9D02846EC6AFFF74D
:10A1C000AEFF8442B4BF00200120F1E7FFF7E8BFF3
:10A1D000FFF7E6BF07B5002300931A461946034868
:10A1E00001F02AFE03B05DF804FB00BF4406002026
:10A1F00000B55DF804FB0020704700B501205DF854
:10A2000004FB80687047C16070472DE9F8438046C1
:10A210000D46174601EB02090C46A145A4EB0506C5
:10A2200009D0D8F800304046DB689847431C03D07B
:10A2300004F8010BF1E73E463046BDE8F883C368F9
:10A24000013304D18069003018BF0120704701201C
:10A25000704743696BB1C269012A0AD95A1C42612D
:10A260001970C369013BC361436900221A70012060
:10A27000704700207047000010B5D0E904435A1C15
:10A2800042610A460248E118FFF7B7FF012010BDFE
:10A2900018030020C368013310B504460ED163696A
:10A2A000B3F5FA4F0EDA23682046DB68984720287A
:10A2B00006DD2368C1B25B6920469847012002E0B1
:10A2C0000130ECD1002010BD0346C068421C03D011
:10A2D0004FF0FF32DA607047196931B19A6922B1E3
:10A2E000481C1861013A08789A61704708B503461E
:10A2F000C068421C03D04FF0FF32DA6008BDD3E9DA
:10A300000412501C586111440148FFF774FFF5E72F
:10A31000180300200368FF211B68184710B5182098
:10A3200004F0B4FD044618B11822002104F003FE25
:10A33000204610BD70B506460C46D4B1237C656836
:10A340001B0704D4E16811B13046FFF7F3FF237C0B
:10A3500003F00F03042B03D1606908B104F09EFDE4
:10A36000206808B104F09AFD204604F097FD2C46C1
:10A37000E3E770BD2DE9F04F036885B0DB68054663
:10A380000E469847421C044604D14FF0FF3005B0FA
:10A39000BDE8F08F2D2832D12B682846DB6898471E
:10A3A000431C0446F1D04FF0FF330093A4F1300377
:10A3B000092B4FF000070DD84FF00A082B682846EC
:10A3C000DB689847A0F13003303C092B08FB0747B6
:10A3D0000446F3D92E2C14D024F02003452B10D0A2
:10A3E000009B7B437361337C022262F3030333746B
:10A3F0002B6828465B69E1B298470020C7E7012334
:10A40000D3E7384603F050FF2E2C8046894639D1D9
:10A410002B68DFF818B1DB68284698470027044608
:10A420004FF0000A52465B464046494603F0A6FFFD
:10A4300080468946A4F1300003F036FF42464B4681
:10A4400003F0E6FD2B688046DB682846894698477E
:10A45000A0F13003092B07F1FF370446E2D924F0BD
:10A460002003452B2AD12B682846DB6898472B28E8
:10A47000044609D12B682846DB68984704464FF00C
:10A48000010A0AE00027EAE72D28F8D12B682846C0
:10A49000DB6898474FF0FF0A04464FF0000B0A2292
:10A4A000A4F13003092B0DD802FB0B3B2B68039260
:10A4B000DB6828469847039A0446F1E74FF0010A03
:10A4C0004FF0000B009803F0EFFE42464B4603F0BE
:10A4D00055FFCDE90001584603F0E6FE80465046A0
:10A4E000894603F0D1FE02460B464046494603F03A
:10A4F00045FF80463846894603F0D6FE02460B46A5
:10A500004046494603F084FD02460B4600200749B9
:10A5100002F09EFC02460B46DDE9000103F02EFF2F
:10A5200004F024FA337C706103225EE700002440CB
:10A5300019B10A22496901F006BD084670470000BA
:10A54000F8B506462DED028BD1B391ED058A18EED4
:10A55000100A03F0BBFEB5EEC08AF1EE10FA044615
:10A560000D4606D51A49304601F0AFFC05F100430F
:10A570001D462946204604F0D9F90A22014607461D
:10A58000304601F00EFD1349304601F09EFC38467E
:10A5900003F07AFE02460B462046294603F036FDBC
:10A5A00009A3D3E9002303F033FD00220A4B03F093
:10A5B000E5FE04F0BBF90A220146304601F00AFD2F
:10A5C000BDEC028B0020F8BD9A9999999999A93F01
:10A5D000BB3D0100DD31010000002440F8B50368F7
:10A5E000DB6806460F469847222803D04FF0FF3419
:10A5F0002046F8BD3B7C042262F303033B7400F069
:10A6000003FB05460028F1D033683046DB689847E5
:10A61000431C044611D0222C36D01F2C34DD5C2C78
:10A6200004D02946E0B200F005FBEDE73368304680
:10A63000DB689847421C044603D1284600F022FB01
:10A64000D6E7622817D007DC2F2803D05C2801D07A
:10A650002228D9D12946E6E76E280FD004DC6628E7
:10A66000D2D129460C20DEE772280AD07428CBD13B
:10A6700029460920D7E729460820D4E729460A2099
:10A68000D1E729460D20CEE7284600F0DFFA002466
:10A690007861ADE738B50D461D49044601F015FC5B
:10A6A0007DB3013D15F8011F59B31F2907D9222990
:10A6B00005D05C2903D0204601F00BFCF2E75C21B9
:10A6C000204601F006FC29780C2914D007D8092966
:10A6D00015D00A2911D00829E4D16221EBE72229FB
:10A6E000E9D003D80D29DDD17221E4E72F29E2D08A
:10A6F0005C29E0D0D6E76621DDE76E21DBE7742137
:10A70000D9E72221204601F0E4FB002038BD00BF3C
:10A710007E3801004969FFF7BDBF0368DB6810B5EB
:10A7200004469847431C0AD02028236802DCDB68D3
:10A730002046F6E7C1B25B6920469847002010BD6D
:10A7400003682DE9F047DB6804460E4691469847BA
:10A750007B2803D04FF0FF30BDE8F087337C062222
:10A7600062F3030333742046FFF7D7FF23682046C4
:10A77000DB6898477D2844D02368C1B25B692046D6
:10A780009847FF274FF0000AFFF7C8FD054600284D
:10A79000E0D08FB3F0602046FFF7BFFF2946204688
:10A7A000FFF71CFF0130D5D02046FFF7B6FF6B69DD
:10A7B0002B602368C5F814A0DB68204698473A2828
:10A7C000C8D12046FFF7A9FF4A462946204600F097
:10A7D0001BF80130BED02046FFF79FFF23682046BC
:10A7E000DB6898472C28A8464FF00007CCD07D386E
:10A7F00018BF4FF0FF30AFE7C8F80400C0F808807A
:10A80000C9E70020A8E70000F7B504460D46174643
:10A81000FFF783FF013002D14FF0FF3011E02368D2
:10A820002046DB689847431C0646F5D02368C1B232
:10A830005B6920469847222E05D129462046FFF71E
:10A84000CDFE03B0F0BD2D2E03D0A6F13003092BB1
:10A8500004D829462046FFF78DFDF2E75B2E05D18F
:10A860003A462946204600F09DF8EAE77B2E05D1BE
:10A870003A4629462046FFF763FFE2E76E2E17D1DE
:10A8800002AE002346F8083D236804221B693146C6
:10A890002046984704280246BED12149304605F09B
:10A8A0000CFB0028B8D12B7C6FF303032B74C8E793
:10A8B000662E19D1002300938DF8043023680522F9
:10A8C0001B696946204698470528A5D105221549E8
:10A8D000684605F0F2FA00289ED12B7C28750122EB
:10A8E00062F303032B74ACE7742E95D102AE002300
:10A8F00046F8083D236804221B69314620469847E4
:10A900000428024688D10849304605F0D6FA0028C6
:10A9100082D12A7C012363F303022A742B7590E70A
:10A920006E3801007338010079380100F8B5064629
:10A9300017460D4611B900242046F8BDFFF7EEFC7E
:10A9400004460028F7D02846FFF7E7FE3A4621469E
:10A950002846FFF759FF0130EED121463046FFF778
:10A96000E9FCE8E70022FFF7E1BF000010B588B07E
:10A970004FF0FF3200230392094A00920446CDE9CA
:10A9800001330846CDE90413079309B105F079FABC
:10A99000069069462046FFF7E5FF08B010BD00BFEE
:10A9A000AC3801002DE9F8430368DB6804460F4624
:10A9B000914698475B2803D04FF0FF30BDE8F883FD
:10A9C0003B7C052262F303033B742046FFF7A5FEA0
:10A9D00023682046DB6898475D282BD02368C1B2E6
:10A9E0005B6920469847FF26FFF798FC054600283C
:10A9F000E2D0D6B1F8602046FFF78FFE4A462946DE
:10AA00002046FFF701FF06460028D5D12046FFF774
:10AA100084FE23682046DB6898472C28A846E3D0AC
:10AA20005D3818BF4FF0FF30C8E7C8F80400C0F821
:10AA30000880E0E70020C1E738B5054651B3CC688F
:10AA40007B2101F046FA013002D14FF0FF3038BDD2
:10AA5000B4B121682846FFF71DFE0130F5D03A2138
:10AA6000284601F036FA0130EFD02146284600F0A2
:10AA700013F80130E9D0646814B12C212846E0E7CE
:10AA80007D21284601F025FA01304FF0FF3018BF34
:10AA90000020DCE70846DAE7E9B10B7C03F00F039E
:10AAA000062B18D8DFE803F004070D0F111315006B
:10AAB0000A4901F00ABA0B7D0BB10949F9E70949C6
:10AAC000F7E7FFF735BDFFF73BBDFFF723BE00F00B
:10AAD0000EB8FFF7B1BF0020704700BF6E3801000D
:10AAE00079380100733801001046FFF7D5BF38B53B
:10AAF0000546F1B1CC685B2101F0EBF9013002D1E0
:10AB00004FF0FF3038BD54B121462846FFF7C4FF4F
:10AB10000130F5D0646814B12C212846ECE75D21A2
:10AB2000284601F0D6F901304FF0FF3018BF002061
:10AB3000E8E70846E6E7CB680022D0B201320BB165
:10AB40005B68FAE77047C86820B11AB1013AD2B21F
:10AB50004068F9E7704738B5CC68154634B12946E6
:10AB6000206805F026F908B16468F7E7204638BD8B
:10AB70004AB1CB6813B9CA6070470B4659680029BF
:10AB8000FBD15A6093607047F8B505460E461746EC
:10AB90001C4673B1186808B104F080F9384605F016
:10ABA00055F92246206031462846BDE8F840FFF7B7
:10ABB000DFBFF8BD10B50C46FFF7B0FB28B1037C32
:10ABC0004461022262F30303037410BD70B50D46A5
:10ABD000194604461646FFF7EDFF3246034629465E
:10ABE0002046BDE87040FFF7CFBF000007B5002347
:10ABF00000931A461946034801F01EF903B05DF8A8
:10AC000004FB00BF4C06002038B50C2004F03EF9D0
:10AC1000044650B1064820604FF480752A46002152
:10AC200004F089F900236560A360204638BD00BFA9
:10AC300050070020D1E90123934204D20A68D0547E
:10AC40008B6801338B60002070470000826838B544
:10AC5000044622B10368134413F8013C1BB121469A
:10AC60000020FFF7E7FFA06804F010F9054628B1BF
:10AC7000034905F0E2F8204604F010F9284638BDF3
:10AC80005007002008B104F009B9704710B5054C11
:10AC9000204601F021F920460349BDE8104001F0AB
:10ACA0000BB900BFB0060020C8380100F0B503782A
:10ACB0009FB0044643B3194B194F1B68986803F0C3
:10ACC0009FFF2046164905F03FF91EAD012445F8C7
:10ACD000780D3946002005F037F91E2C264645F838
:10ACE000240002D001340028F3D10E4B009F1C68D1
:10ACF00074B12168384605F096F838B9636829467A
:10AD000030469847FFF7C2FF1FB0F0BDA468EFE7D9
:10AD10000549064801F0E6F8F4E700BF38000020D6
:10AD2000B837010098060020CF380100B006002097
:10AD3000F8B505460C200F4604F0A8F80C4B044665
:10AD40001860284605F09DF8013004F09FF8294668
:10AD5000064605F072F8284605F093F800233354B0
:10AD6000044B1A68A260C4E900671C60F8BD00BF0C
:10AD7000980600205806002070B51648164D01F0C0
:10AD8000BDFBC4B20A2C0CD00D2C0AD0082C15D156
:10AD90002146104801F09DF82B7873B1013B2B70D0
:10ADA0000BE02B780D4E0E490A480024F45401F0B4
:10ADB0008CF83046FFF77AFF2C7070BD21460548AD
:10ADC00001F087F82B783A2B9FBF5A1C2A70034A50
:10ADD000D454F2E7B00600209C0600205C06002058
:10ADE000CC38010010B5044C204601F081FB10B1B5
:10ADF000FFF7C2FFF8E710BDB0060020044A0023A9
:10AE00001370044A01460448136001F030BB00BFD0
:10AE10009C06002058060020B006002070B50446AD
:10AE20000D4601F067FDA061A068036829461B6814
:10AE3000BDE87040184770B504460D46164601F04F
:10AE400059FDA061A0680368324629465B68BDE8E9
:10AE50007040184710B50446C06804F01FF820463B
:10AE600010BD2DE9F04105460E4601F043FD4FF4BB
:10AE70007A778046A86803689B689847044658B963
:10AE800001F074FD01F036FDAB8AA0EB08007B43B6
:10AE90009842EFD3204605E0A8680368DB6898472E
:10AEA00030700120BDE8F08138B514882144154682
:10AEB000FFF7D7FF08B101342C8038BD2DE9F74FDB
:10AEC00002AD002625F8026D8A462A46C16804466E
:10AED000FFF7EAFF18B9002003B0BDE8F08FE36880
:10AEE0000DF1080993F8008009F8036D0127BDF8FA
:10AEF0000630052B07D14FF0FF33A068E3630368EA
:10AF00005B6A9847E7E749462046FFF7AAFF002813
:10AF1000E1D0BDF80630E268591CADF806109DF886
:10AF20000510D1549DF8053003F07F0207FB02663F
:10AF30001A064FEAC717DAD49DF8063008F0F00871
:10AF4000013BB8F1300F8AF800301DD12A46E16884
:10AF50002046FFF7A9FF0028BDD02A46E168204619
:10AF6000FFF7A2FF0028B6D0E2689AF80030134439
:10AF700059789D78137805EB01259B07ADB201D573
:10AF80000235ADB2022701E000273D46BDF806B00C
:10AF9000A7EB0B0707EB0B0296422AD9494620463E
:10AFA000FFF75FFF002896D0A06B88B1B8F1300F93
:10AFB0000ED19AF80020C2F1FF2202F57F02FE3284
:10AFC0005A44AA4204D902689DF8051012689047B5
:10AFD000BDF80620218A914208D9E1689DF8050054
:10AFE0008854BDF806200132ADF806200BF1010BA4
:10AFF000D0E7A26B22B9218A594538BFADF80620A7
:10B00000BDF8060068E773B50025DC1103F07F0684
:10B01000A3B20CB146F080060DF1080C681C654423
:10B02000C0B205F8046C0546002CEED1C0F1040551
:10B03000515501ADA04205DD231A1344615D5971DC
:10B040000134F7E7013002B070BDF8B50646174687
:10B050001C46FFF7D8FFB368C0B21A680444C0F1B9
:10B0600005015568394422461846A847054601F0AF
:10B0700041FCB061A8B2031B58425841F8BD10B55D
:10B08000C368E0221A70C36800225A7004468068C0
:10B09000E168036802225B689847A0684FF0FF33BD
:10B0A000E36303685B699847A06803685B6A984735
:10B0B00001F020FCC4E9060010BD023330B598B29F
:10B0C0000C46631A14F8015B9BB21DB1431C155466
:10B0D00098B2F6E7C11A0A44191202F8021C02F8E3
:10B0E000013C30BD38B50546806808B9002038BD40
:10B0F00003689B6A9847EC6B68B9002CF6D1A86886
:10B100006FF00203EB6303685B699847A868036804
:10B110005B6A9847EAE7B4FA84F04009E7E7000081
:10B120002DE9FF470C9D9DF840A00446894617462F
:10B130001E46FFF7D7FF8046002840F0DF80A0685A
:10B1400003689B6A9847002840D00123E3826E4B36
:10B15000029345F25443ADF80C3004238DF80E30C1
:10B16000052302A91944E26811F8051CD1540133E2
:10B170000C2BF6D1002D3DD09DF838309DF83420B1
:10B180005B0143F0040343EAC203DBB2BAF1000FF0
:10B1900001D043F002031FB1002E2DD143F08003F4
:10B1A000E2681373638AE2681B125373E368628A6E
:10B1B0009A73218A484604F0A7FE238A11309842E8
:10B1C0001DD9A06803685B6A984797E0A068216B67
:10B1D0000368A28E39B1DB6998470128B5D06FF0BA
:10B1E0000103E3638AE049499B690291E16A0391A3
:10B1F00002A9F1E72B46C9E743F0C003D0E749466F
:10B200000F23E2682046FFF758FF814605B3218AE5
:10B21000284604F079FE09F102031844238A984273
:10B22000CFD84B462946E2682046FFF746FF218AE1
:10B2300005460F9804F068FE238A0230284498429D
:10B24000BFD82B46E2680F992046FFF736FF8146AC
:10B2500017B3218A384604F057FE09F10203184457
:10B26000238A9842ADD84B46E26839462046FFF71C
:10B2700024FF814686B1218A304604F045FE09F15B
:10B2800002031844238A98429BD84B46E268314611
:10B290002046FFF712FF8146A9F105039BB2E26841
:10B2A00010212046FFF7D1FE01F024FBC4E906007F
:10B2B0004FF47A75A06803689B68984758B901F005
:10B2C00019FBE369C01AA38A6B439842F2D36FF06B
:10B2D0000303E36375E70DF107012046FFF7EEFD79
:10B2E00004287FF46EAFE368DD785DB901F002FBFE
:10B2F0004FF00108E06184F82050E563404604B057
:10B30000BDE8F087E5635CE700044D517839010042
:10B3100010B586B0012404940B9C03949DF828403A
:10B3200002949DF824400194089C0094FFF7F8FED5
:10B3300006B010BD2DE9F3470446FFF7D3FE804663
:10B34000D0B101F0D7FA628A4FF47A735343E269BD
:10B35000821A9A42074603D8A269821A93421FD2E0
:10B3600094F8203063B16FF00303A068E3630368CF
:10B370005B6A98474FF00008404602B0BDE8F0878E
:10B38000E268C0211170E2685370A068E168036848
:10B3900002225B689847C4E90677012384F82030CD
:10B3A000A06803689B6898470028E5D00DF1070165
:10B3B0002046FFF783FD83B20646002B73D0E36877
:10B3C000E7611A7802F0F002302A57D1626A002A47
:10B3D000D2D09DF807209918901C49781D5C05EB88
:10B3E0000125ADB2D11C19442A46184403F08AFD48
:10B3F000E3689DF807202B44134400229A70E1680B
:10B400009DF807C091F8009009F00609B2B20CF15E
:10B410000200B9F1020F0844666A0CF10303A2EBC3
:10B420000C0225D12B440CF1050C11F803E00B4460
:10B43000521B93F801A06544053A29440AEB0E2AF1
:10B44000B047E36840221A70E36883F80190E3682C
:10B450001FFA8AFA4FEA2A229A70E36883F803A057
:10B46000A068E168036804225B689847A76183E7E6
:10B470002B44033A521B1944B0477DE7C02A0BD135
:10B48000D0221A70E36800225A70A068E16803684D
:10B4900002225B6898476FE7D02A7FF46DAF0023E4
:10B4A00084F8203068E72046FFF71CFE002808BF1C
:10B4B0004FF0000860E72DE9F0470446884617463C
:10B4C0001D469DF82060FFF70DFE50B3B4F81090B4
:10B4D0004046494604F018FDEB1D1844814520D331
:10B4E00041460523E2682046FFF7E7FD00211FFAE9
:10B4F00081FC4318AC459BB2E26801F1010104D222
:10B5000017F80CC002F803C0F1E7002EA3F1050301
:10B5100020469BB214BF31213021BDE8F047FFF730
:10B5200094BD0020BDE8F08773B505460E4614466D
:10B530006AB1018A104604F0E7FC0346002200923B
:10B54000314622462846FFF7B6FF02B070BD1346CB
:10B55000F4E7F7B505460E461F46144662B1018A68
:10B56000104604F0D1FC0346009722463146284697
:10B57000FFF7A1FF03B0F0BD1046F4E770B50D462C
:10B580000446018A2846164604F0BEFC45B3012E47
:10B5900026D8238A0930834222D32046FFF7A2FD12
:10B5A000F0B1E38A01339BB2C3B1E382E38AE2687C
:10B5B0001B125371E368E28A9A71E26829460723F5
:10B5C0002046FFF77AFDE3681E54031FE268204619
:10B5D0009BB28221BDE87040FFF737BD0123E4E74D
:10B5E000002070BD0022FFF7C9BF70B50D460446AC
:10B5F000018A284604F088FC25B3238A0930834257
:10B6000020D32046FFF76EFDE0B1E38A01339BB201
:10B61000B3B1E382E38AE2681B125371E368E28A02
:10B620009A71E268294607232046FFF746FD431F2B
:10B63000E26820469BB2A221BDE87040FFF705BD3D
:10B640000123E6E7002070BD0163828670474162F6
:10B650007047C06B704738B504460D4609B90020E5
:10B6600038BD038A4BB9084603F010FCE060E0687F
:10B670002582003018BF0120F2E7C06804F0DEFA2E
:10B680000028F3D1EBE7000070B50C4B0025044611
:10B69000456040F8283B0E4600F0C6FB4FF0FF33F4
:10B6A000E363A660A56325824FF480712046FFF70F
:10B6B000D2FF0F236382A382204670BDE8380100C9
:10B6C00007B5002300931A461946034800F0B4FB5F
:10B6D00003B05DF804FB00BFA00600208271054A9C
:10B6E000417112680449B2FBF1F14FF47A724A4396
:10B6F000C26070471800002040420F0038B5044671
:10B700000D464079022101F0A1FA01F0F3F8A0F50D
:10B71000FA60A060657438BD70B505460E46002419
:10B72000687901F0CDFAB042A3B206D1EA689A4234
:10B7300004F10104F4D84FF0FF33184670BD30B562
:10B740000D46D1B0044601F0D5F83DB9A368C31A3F
:10B75000B3F5FA6F02D2207C51B030BD0025022132
:10B76000A06025606079257101F070FA012001F078
:10B77000DBF80121607901F069FA2946607901F06E
:10B780008DFAA379153B012B00F28C8040F24C40DE
:10B79000013800BF00BF00BF00BF00BF00BF00BF37
:10B7A00000BF00BF00BF00BF00BF00BF00BF00BFA1
:10B7B00000BF00BF00BF00BF00BF00BF00BF00BF91
:10B7C00000BF00BF00BF00BF00BF00BF00BF00BF81
:10B7D00000BF00BF00BF00BF00BF00BF00BF00BF71
:10B7E00000BF00BF00BF00BF00BF00BF00BF00BF61
:10B7F00000BF00BF00BF00BF00BF00BF00BF00BF51
:10B8000000BF00BF00BFC3D16079022101F01EFA62
:10B81000607C00283BD0013800BF00BF00BF00BFE4
:10B8200000BF00BF00BF00BF00BF00BF00BF00BF20
:10B8300000BF00BF00BF00BF00BF00BF00BF00BF10
:10B8400000BF00BF00BF00BF00BF00BF00BF00BF00
:10B8500000BF00BF00BF00BF00BF00BF00BF00BFF0
:10B8600000BF00BF00BF00BF00BF00BF00BF00BFE0
:10B8700000BF00BF00BF00BF00BF00BF00BF00BFD0
:10B8800000BF00BF00BF00BF00BF00BFC3D172B682
:10B8900000212046FFF740FF013007D1002020742F
:10B8A00062B659E7142001F03FF8ADE701212046C8
:10B8B000FFF732FF0130F1D0002500212046FFF7CD
:10B8C0002BFF01214DF805002046FFF725FF0DEB6A
:10B8D00005030835B5F5A07F5860EED162B60022A9
:10B8E0005DF832500DEBC203691C586801D0431C4F
:10B8F00002D1002020742FE7D1108542635C4FEA0B
:10B900004303DBB202F1010238BF43F00103282AEE
:10B910006354E5D16178237822790B44A1780B44F4
:10B92000E1780B44DBB29A42E3D10120E2E7000068
:10B930002DE9F8430D462DED028B11460446FFF725
:10B94000FEFE00287ED0A3790B3B0B2B7AD8DFE8D4
:10B9500003F0063F79797979797979796565A37802
:10B96000E07808EE103A0106B8EE488A48BFFFEECC
:10B97000007A00F00F0048BF37EEC88A02F094FC4E
:10B9800031A3D3E9002302F0F9FC064618EE100AB1
:10B990000F4602F09BFC0B4602463946304602F049
:10B9A00037FB02F0E3FF03466DB102F08FFC2AA3E0
:10B9B000D3E9002302F0E2FC254B002202F028FB31
:10B9C00002F0D4FF0346BDEC028B1846BDE8F883B5
:10B9D000E078A67800F00F0002F066FC1AA3D3E925
:10B9E000002302F0CBFC07EE906AF8EE677A8046FF
:10B9F00017EE900A894602F069FC02460B46404663
:10BA0000494602F005FB02F0B1FF3206034648BF8B
:10BA100080F00043002DD6D01846C6E7A678E3781C
:10BA2000300200F4FE40184307EE900AF8EEE77A81
:10BA300017EE900A02F04AFC03A3D3E9002302F0B8
:10BA40009DFCE0E7034BBEE79A9999999999B93F14
:10BA5000000040400000C07FCDCCCCCCCCCCFC3F23
:10BA6000D0B50446FFF76BFE90B3A3790B3B0B2BCD
:10BA70002ED8DFE803F006062D2D2D2D2D2D2D2D92
:10BA80001C1C607802F010FC14A3D3E9002302F020
:10BA900075FC064620780F4602F006FC02460B466F
:10BAA0003046394602F0B4FA02F060FFD0BD20887B
:10BAB00040BA80B207EE900AF8EEE77A17EE900AE5
:10BAC00002F004FC05A3D3E9002302F057FCEBE7E6
:10BAD0000148EBE7AFF300800000C07F9A99999985
:10BAE0009999B93F10B50446C06803F0D7F9B4F985
:10BAF0000600002802DB002101F0A8F8204610BD56
:10BB000070B50546C0680E4603F0C8F9EC7C2A7C87
:10BB100094420CBF0324042414FB06F4A4B2AC80AA
:10BB2000204603F0B3F9E86028B12246002103F073
:10BB300002FA6E8070BDA8806880FBE7F0B4FF2930
:10BB4000C1F38107C1F38112C1F30115477401F0FC
:10BB500003078CBF002101210170C168C47C067CF1
:10BB6000C2740574877461B1A41B6142A2EB050520
:10BB700061416A426A41914203D04188F0BCFFF7BB
:10BB8000BFBFF0BC704738B5437804460D4633B1AB
:10BB9000B0F90600002802DB002101F057F86378B5
:10BBA000E5804BB12846012101F050F828460021DC
:10BBB000BDE8384001F072B838BD70B50E460021BE
:10BBC000044641700172C160416119461546FFF794
:10BBD000B5FF31462046FFF793FF20462946FFF781
:10BBE000D2FF204670BD70B540F2FA5404FB00F35A
:10BBF00003F500431B14B3F5FF7F98B222DAFE2B46
:10BC0000D8B242DDC0F1FE00C5B20023FF204E1CB9
:10BC1000C943C9B27043013201EB2020504300F404
:10BC20007F4406FB03F006FB05F301EB202001EB4C
:10BC3000232150434A43120244EA102002F47F02B7
:10BC4000104370BDB3F57F7F0DDAB0F53F7FDBB2F7
:10BC50008BBFC3F1FC030233D8B2DBB294BFFF2029
:10BC6000FF230025D3E7A04211D040F2FA44A042BE
:10BC7000DBB204D80433DDB20020FF23C7E7C3F1F1
:10BC8000FA03DBB20020FF25C1E70023FBE7002316
:10BC90001846F8E770B50446083015460E4600F021
:10BCA000C3F8FF23064A84F822300023266025715A
:10BCB0002361A382C4E906222384204670BD00BF0D
:10BCC000BB3D01000161828270470000024B0029E8
:10BCD00008BF194681617047BB3D0100024B002936
:10BCE00008BF1946C1617047BB3D01000184704720
:10BCF00073B50D4601690446164639B92B4BC26827
:10BD00005B689A4202D1002002B070BDA28A002A6C
:10BD1000F9D094F8223005F007000341DB0738D54D
:10BD200015F47E7F08BF238C206804BF03F47E7364
:10BD30001D43036800292ED05B6A98470128E2D191
:10BD40003C21206800F0C5F80A222946206800F04E
:10BD50001CF9237933BB1649206800F0ADF8A169BE
:10BD6000206800F0B2F82021206800F0B2F8E16904
:10BD7000206800F0AAF82379B3B90E49206800F0D2
:10BD80009BF83146206800F0A0F8206803689B6AA1
:10BD900098470120B8E708490091E16801911B6AC2
:10BDA0006946CAE70549D7E70549E7E7A80600203D
:10BDB000F0380100F6380100783901001125010042
:10BDC0000139010008B5FFF793FF08BD07B500234F
:10BDD00000931A461946034800F02EF803B05DF8A8
:10BDE00004FB00BFA80600202DE9F84306460D46D7
:10BDF000071D00F10709002417F8011B0A22284635
:10BE000000F0DCF82E218046284600F062F84F450D
:10BE100040440444F0D10A22F179284600F0CEF8DB
:10BE20002044BDE8F8830000024A0260002242601C
:10BE3000704700BF7839010030B58371034D9DF81C
:10BE40000C30056001714271C37130BD7839010059
:10BE5000024A02600A684260704700BF78390100F8
:10BE60000B68436070472DE9F04106460D4601EB33
:10BE700002080C464445A4EB050707D0336814F8C4
:10BE8000011B1B68304698470028F3D13846BDE8AF
:10BE9000F08170B5044608460D4603F0F2FF2368B2
:10BEA0000246294620465B68BDE87040184709B144
:10BEB000FFF7EFBF0846704708B5FFF7F8FF08BD6A
:10BEC00003688A685B680968184708B5FFF7EFFFE1
:10BED00008BD03681B6818470149FFF7DABF00BFB8
:10BEE000CC38010038B50546FFF7E1FF0446284687
:10BEF000FFF7F2FF204438BD38B50546FFF7D7FFFE
:10BF000004462846FFF7E8FF204438BD70B58AB0E4
:10BF10000D460AA9002301F8043D012A98BF0A2210
:10BF2000B5FBF2F402FB1456F3B2092E94BF303382
:10BF30003733DBB2254601F8013D002CF0D1FFF785
:10BF4000B6FF0AB070BD2DE9F04107460E46154612
:10BF50002AB90368C9B21B68BDE8F04118470A2A2C
:10BF600005D1002905DBBDE8F041FFF7CFBFD2B214
:10BF7000F9E72D21FFF7ADFF2A4604467142384606
:10BF8000FFF7C4FF2044BDE8F081FFF7DCBF38B500
:10BF90000546FFF7D8FF04462846FFF79DFF2044DB
:10BFA00038BD10B42AB903685DF8044B1B68C9B2E8
:10BFB0001847D2B25DF8044BFFF7A8BFFFF7F1BFF7
:10BFC00038B50546FFF7EDFF04462846FFF784FF26
:10BFD000204438BDFFF7E5BF2DE9F84F1946064666
:10BFE000104614461D469DF8287002F061FC28B1E9
:10BFF0004C493046BDE8F84FFFF74BBF25F00049EC
:10C000004FF0FF32484B2046494602F051FC48B9F8
:10C010004FF0FF32444B2046494602F02BFC08B952
:10C020004249E6E74FF06042414B2046294602F084
:10C0300035FC08B13F49DCE74FF060423E4B2046FB
:10C04000294602F00DFC0028F4D1002200232046EE
:10C05000294602F005FCD0B12D213046FFF739FF0B
:10C0600005F1004382461D463449DFF8D8904FF071
:10C07000000B00204FF000085FFA8BF39F4208D9B5
:10C0800042464B4602F0A4FA0BF1010BF4E782465C
:10C09000EAE722462B4601F0BBFF0D46044602F0BC
:10C0A00045FC0A22014680463046FFF72FFF8244B6
:10C0B000A7B3404602F0E8F802460B462046294660
:10C0C00001F0A4FF04460D4630461D49DFF8749088
:10C0D000FFF7DFFE4FF000088244013FFFB2FF2F61
:10C0E0001CD04B4642462046294602F047F90D46F1
:10C0F000044602F0F3FB0A22014683463046FFF76E
:10C1000022FF8244584602F0CFF802460B462046F2
:10C11000294601F07BFF04460D46DEE75046BDE8A8
:10C12000F88F00BF7C390100FFFFEF7F80390100ED
:10C13000FFFFEF4184390100FFFFEFC10000E03F46
:10C14000DD310100000024409DF800100091FFF750
:10C1500043BF08B54022002102F0EDFE0022C0E9F5
:10C16000102208BD026C10B5531C446C03F03F0351
:10C170009C421CBF8154036410BD0023C0E91033EE
:10C180007047D0E9102393421FBFC25C013303F014
:10C190003F03436414BF10464FF0FF307047D0E9AF
:10C1A0001030181A48BF40307047D0E9102393422E
:10C1B00014BFC05C4FF0FF307047036C406C01331C
:10C1C00003F03F031B1A5842584170470649074A7B
:10C1D000074B9B1A03DD043BC858D050FBDC00F032
:10C1E00037F8F4F72DF80000CC3D010000000020E6
:10C1F00088020020FEE7FEE7FEE7FEE7FEE7FEE737
:10C20000FEE7FEE7FEE7FEE7044B1868421C04BFAA
:10C21000034B1878831F5842584170473001001073
:10C22000E00F00F0074B1B78062B09D1064B1B686B
:10C23000C3F30313033B032B02D8044AD05C7047BB
:10C2400000207047E00F00F0E80F00F08C3901008B
:10C2500008B5FFF7D9FF28B1654B664A1B68C3F3E1
:10C2600004231360FFF7DEFF10B1634B634A1A60CB
:10C27000FFF7CAFF28B1624B624A1B68C3F342331F
:10C280001360FFF7CFFF20B15F4AD36823F08073BC
:10C29000D360FFF7B9FF40B14FF080430022C3F8ED
:10C2A0000C21C3F81021C3F83825FFF7BBFF10B1EC
:10C2B000564B03221A60FFF7B5FF40B1544B0522DD
:10C2C0001A6001229A6700229A603F225A60514BFD
:10C2D0001A68511C0BBF504B504B1A781B6802BF99
:10C2E00008331B68C3F30313062A4DD1033B032B0A
:10C2F00003D84B4AD35C002B46D04FF08052494BB9
:10C30000D2F80414C3F82015D2F80814C3F8241581
:10C31000D2F80C14C3F82815D2F81014C3F82C1551
:10C32000D2F81414C3F83015D2F81814C3F8341521
:10C33000D2F81C14C3F84015D2F82014C3F84415E1
:10C34000D2F82414C3F84815D2F82814C3F84C15B1
:10C35000D2F82C14C3F85015D2F83014C3F8541581
:10C36000D2F83414C3F86015D2F83814C3F8641541
:10C37000D2F83C14C3F86815D2F84014C3F86C1511
:10C38000D2F84424C3F87025FFF73EFF28B1264BAE
:10C39000264A1B6803F04F031360FFF735FF48B1CF
:10C3A0004FF08043D3F80024D20744BF6FF001025E
:10C3B000C3F80024174B1B68062B09D1174B1B68C9
:10C3C000033B022B81BF1A4A136843F48063136056
:10C3D000184AD2F8883043F47003C2F88830BFF3AB
:10C3E0004F8FBFF36F8F144B144A1A6008BD00BF04
:10C3F000240300104035014074C007400DF0ADBA71
:10C40000440200103C050040F0ED00E0A0050040B3
:10C410001056004030010010E00F00F03401001011
:10C420008839010000C0004058020010E40E0040AE
:10C430003C17004000ED00E0180000200090D00301
:10C4400010B5044600F056FAE06023682046DB6829
:10C450009847002808DA00F04DFAE368C01AA3688C
:10C460009842F2D34FF0FF3010BD012070470368AF
:10C470001322DB69184770470369C3F81C15036969
:10C48000D3F81C21002AFBD00022C3F81C21012074
:10C490007047000010B490F95C30144C5909012227
:10C4A000203103F01F0302FA03F344F8213003693B
:10C4B0005DF8044B0421C3F8081303695A6003694B
:10C4C000DA6003690022C3F8002502694FF0FF33E8
:10C4D000C2F80C350269C2F814350269C2F8083591
:10C4E00002691430C2F81035FFF747BE00E100E0E2
:10C4F0001430FFF754BE1430FFF757BE1430FFF767
:10C5000040BE0000036990F85E2010B5C3F80C250A
:10C51000036990F85D20C3F8142590F86120036941
:10C52000012A01BF90F85F40C3F81045036990F8F5
:10C53000604006BFC3F8084503690022B1F5966F55
:10C54000C3F86C2569D9B1F5166F69D9B1F5965F55
:10C5500069D9B1F5165F68D9B1F5615F67D9B1F5F1
:10C56000964F66D9B1F5E14F65D9B1F5164F64D94B
:10C57000B1F5614F64D9B1F5963F64D9B1F5E13FAA
:10C5800063D9B1F5613F63D9364B994263D9B1F5AF
:10C59000E12F63D9B1F5612F94BF4FF070634FF075
:10C5A00080530269C2F8243503690422C3F80025C8
:10C5B00001690023C1F808310169C1F81C31016922
:10C5C00001230B6001698B600169C1F8042390F9B4
:10C5D0005C20510902F01F0293406031224A42F868
:10C5E000213090F95C30002BBDBF03F00F0302F641
:10C5F000FC32D2189B18B5BF60236022137683F8F3
:10C60000002390F95C300122590903F01F0302FA5C
:10C6100003F3154A42F8213010BD4FF49E23C0E7C2
:10C620004FF41D23BDE7114BBBE7114BB9E7114B8D
:10C63000B7E7114BB5E7114BB3E74FF41D03B0E774
:10C640004FF46B03ADE70E4BABE74FF0EB73A8E78E
:10C650004FF06C73A5E74FF08063A2E74FF0E863FB
:10C660009FE700BF90D0030000E100E000B013009E
:10C670000050270000F03A0000A04E0000C07500F6
:10C6800000903A012DE9F0411E4600254FF47A73DF
:10C69000C0E901530D4B044640F8143B1746884649
:10C6A000FFF757FD0A4AC4F8108084F85C7052F80E
:10C6B000263084F85D309DF8183052F8233084F825
:10C6C0005E3084F861502046BDE8F0819839010061
:10C6D0000839010010B50369D3F8082104464AB1AE
:10C6E000D3F818151430C9B2FFF73CFD23690022B6
:10C6F000C3F8082110BD00000148FFF7EBBF00BFE1
:10C70000B006002007B5192300930222182303491D
:10C710000348FFF7B7FF03B05DF804FB00200040BB
:10C72000B006002010B5044628B103F053FA90FB80
:10C73000F4F303FB1404204610BD884210B50446F0
:10C7400003DA081AFFF7EEFF0444204610BD10B5C7
:10C75000029C401AE41A6043521A90FBF2F018440B
:10C7600010BD0023C0E9003310B50C68836004607D
:10C770004C6844608C688460C1E900338B6010BDF4
:10C7800010B50446006802F089FB204610BD10B5C4
:10C790000446006808B102F081FB00232360C4E96D
:10C7A000013310BD38B504460D460068013103F071
:10C7B00045FA10B1C4E90005012038BD036810B581
:10C7C000044623B143688B4201D3012010BD2046AB
:10C7D000FFF7E8FF0028F9D0A368002BF5D1226805
:10C7E0001370F2E770B50E46114604461546FFF782
:10C7F000E5FF20B92046FFF7CAFF204670BDA560BF
:10C800003146206803F019FBF7E738B500230446EA
:10C81000C0E9003383600D4639B1084603F031FBAF
:10C82000294602462046FFF7DDFF204638BD38B5D1
:10C83000054600680C4668B16A688B689A4207D35F
:10C84000096803F0FAFAA368AB600023A36038BD5F
:10C8500002F024FB23682B6063686B60A368AB6005
:10C860000023C4E90033F1E7884210B50B460446C3
:10C8700004D0096821B19A68FFF7B4FF204610BDC3
:10C88000FFF785FFFAE710B500230446C0E900333F
:10C890008360FFF7E9FF204610BD884210B50446CB
:10C8A00001D0FFF7C4FF204610BD70B505460E4607
:10C8B00009B9002070BD6AB1846814442146FFF7AD
:10C8C0007DFF0028F5D02868AB683146184403F096
:10C8D000B4FAAC600120EDE707B500238DF8041031
:10C8E000012201A98DF80530FFF7DFFF03B05DF8E5
:10C8F00004FBFEE70A4B19680A4B30B5D3F8040570
:10C900000C060D0A44EA00024FF47A712B46A2FB92
:10C91000014501FB0355E00B40EA454030BD00BF37
:10C92000140700200010014038B5044648B1FFF755
:10C93000E1FF054600F01AF8FFF7DCFF401BA042BC
:10C94000F8D338BD074B0022C3F8042182B0D3F8D6
:10C950000431054A0193019B13680133DBB2136074
:10C9600002B0704700100140140700207047704764
:10C9700008B500F017F8FFF7FAFF0120FFF7D4FF22
:10C98000F7F7DCF8034CF7F7DBF8002CFBD0AFF33C
:10C990000080F8E70000000002F078BA02F076BAF2
:10C9A00002F07CBA2A4BE02283F811234FF40032C4
:10C9B000C3F880211A604FF080430122C3F8182584
:10C9C0009A6003F588330021C3F808150221C3F8E3
:10C9D0000413C3F844131A604FF01023D3F8002255
:10C9E000002A03DBD3F80432002B2FDA194B012283
:10C9F000C3F80425D3F80024002AFBD04FF01022FE
:10CA00001521C2F80012D3F80024002AFBD04FF001
:10CA100010231522C3F804220E4B1A46D3F8001433
:10CA20000029FBD00021C3F80415D2F80034002BF4
:10CA3000FBD0BFF34F8F0849084BCA6802F4E0628D
:10CA40001343CB60BFF34F8F00BFFDE7704700BFBC
:10CA500000E100E000E0014000ED00E00400FA0524
:10CA6000192837B50CD84B4B53F82030052B00F064
:10CA7000828007D8032B12D07BD8022B00F0818054
:10CA8000002074E01D2B78D003D81C2BF8D1052290
:10CA900006E01E2B73D01F2BF2D1082200E00222E9
:10CAA0003D4B196808296EDD0A296FDD0D29B5BFD8
:10CAB0000C240E24022303233848C0F8F035012348
:10CAC000C0F8003500200546030103F1804303F55B
:10CAD000E04301300828C3F81455C3F81055F3D1CA
:10CAE0002F4B18682F4B1B6800021B0303F4805365
:10CAF00000F4E0601843294BC3F81805C3F8142567
:10CB0000C3F810250DF10602C3F82C260122C3F844
:10CB100030261A60D3F80021002AFBD00022C3F887
:10CB2000002101225A601D4B1A46D3F80401002847
:10CB3000FBD00020C3F8040101209860D2F8143122
:10CB4000002BFBD00023C2F81431BDF906209A4215
:10CB5000124AB8BFADF80630A142C2F80035BDF99F
:10CB6000060004D035BF611A091BC840884003B0D5
:10CB700030BD032294E7042292E7062290E70722C1
:10CB80008EE701228CE70824002395E70A2401237D
:10CB900092E700BF08390100280000200070004023
:10CBA0002C00002020070020192830B53CD8224B4B
:10CBB00053F82000214B00221D4653F82240B4F1C7
:10CBC000FF3F32D11E4C45F822006FEA41411D4D16
:10CBD0001D4B246853F822306FEA514125F812109A
:10CBE000012101FA04F4C3F86005013CC3F86405AF
:10CBF00005EB4202C3F86805C3F86C050020C3F8D2
:10CC00000015C3F80C05C3F80405C3F80845C3F8BC
:10CC10001405C3F81005C3F82025C3F82415C3F87C
:10CC20002815C3F82C05996030BD8442CAD0013262
:10CC3000032AC2D1F8E700BF083901001C00002018
:10CC40003000002018070020C039010019280FD833
:10CC5000114B53F8203003290AD8DFE801F00216FF
:10CC60000A1003F5E0734FF0A042002142F82310B0
:10CC7000704703F5E0734FF0A0420C21F6E703F58F
:10CC8000E0734FF0A0420421F0E703F5E0734FF0AA
:10CC9000A0420321EAE700BF0839010019280CD897
:10CCA000064B53F82020012393404FF0A04211B9C6
:10CCB000C2F80C357047C2F80835704708390100D2
:10CCC00019289FBF4FF0A043054AD3F8103552F8FA
:10CCD00020009ABF23FA00F000F001000020704706
:10CCE0000839010038B50025057329B90B4B0C4AEA
:10CCF0000C48252101F08AFE01600B4951F82220E1
:10CD0000027151F8233083719DF8103051F82330AF
:10CD100043710223C371856038BD00BFCC39010067
:10CD20002F3A0100DA39010008390100037B23B9E9
:10CD300043738373036101230373704784B00DF160
:10CD4000100C0CE90E009DF8081002680023012960
:10CD5000C2F80035039B12D00BD303290CD0C2F8C4
:10CD60005435019BC2F824350123C2F8003504B0C4
:10CD7000704743F00203F2E743F00403EFE743F0A8
:10CD80000603ECE710B5FFF7D1FF03688279C3F81B
:10CD900008254279C3F80C250279C3F81025034B06
:10CDA000BDE810400ECBFFF7C9BF00BF3807002019
:10CDB00010B485B001AC84E80E0094E80E0005B014
:10CDC0005DF8044BFFF7BABF70470368C3F81C1542
:10CDD000D3F80821002AFBD0D3F818050022C3F8A5
:10CDE0000821C0B27047000007B5094B09490A483D
:10CDF0004FF080421A6000229A6002221A710B23BF
:10CE000000930C220D23FFF76DFF03B05DF804FBC8
:10CE10003807002000300240240700200B4601465E
:10CE2000184601F015BE0000C0F3C7537F3B162B18
:10CE3000024605DC002B04DB0348184122EA00000F
:10CE4000704700F000407047FFFF7F0000000000C7
:10CE50002DE9F04FDFF82C938DB006460F461446AF
:10CE60001D4600F095F999F90080B8F1FF3FCDE932
:10CE7000000136D022462B462046294601F018FDF7
:10CE8000834670BB32463B463046394601F010FDC2
:10CE90008246002840F0A280304639460022002316
:10CEA00001F0D4FC10B3002200232046294601F0F3
:10CEB000CDFC8346002867D09FEDA77B0122AC4BB9
:10CEC000CDF828A00292CDE90467CDE906458DEDA5
:10CED000087B0393B8F1000F41D09FEDA17B8DED4E
:10CEE000007BDDE900010DB0BDE8F08FDDE9000158
:10CEF00000F066FF8046002800F08D804FF0000AA9
:10CF00004FF0000BDDE9000152465B4601F09EFC4C
:10CF10000028E6D03046394600F052FF0028E0D025
:10CF20002046294600F04CFF0028DAD099F900305D
:10CF30008F4A039204210022022BCDE90467CDE938
:10CF40000645CDE908AB02910A9203D002A800F091
:10CF50003DFF50B901F08AFD2223036005E002A8DD
:10CF600000F034FF002800F09B800A9B1BB101F009
:10CF70007DFD0A9B03609DED087B8DED007BDDE967
:10CF800000010DB0BDE8F08F2046294600F018FFE3
:10CF90000028A6D0002200232046294601F060FC8C
:10CFA00000289ED0724A99F90030CDF828B00121AE
:10CFB000CDE90467CDE90645CDE90212002B74D016
:10CFC0006C490020022BCDE9080172D101F04EFD21
:10CFD000212303600A9B002BCDD0C8E70022002349
:10CFE0002046294601F032FC00283FF47AAF624B1C
:10CFF0005F49CDF828B000220120B8F1020FCDE939
:10D0000004670290CDE90645CDE908230391A6D136
:10D01000CDE9002365E73046394600F0D1FE00280F
:10D020003FF46CAF2046294600F0CAFE00283FF4CA
:10D0300065AFDDE900231046194601F039FC99F986
:10D0400000A000286BD10323DFF824C10A902946F1
:10D05000204602930022494BCDF80CC0CDE906458D
:10D06000CDE9046701F08AF904460D46BAF1000FD4
:10D0700025D1DFF814B14FF0604A0022002330467A
:10D080003946CDE908AB01F0EBFB38BB02A800F054
:10D090009DFE00289ED101F0E9FC2223036099E760
:10D0A00001F0E4FC212303605FE79FED2B7B8DED16
:10D0B000087B02A800F08AFE00288BD186E79FED4E
:10D0C0002A7B00220023304639468DED087B01F093
:10D0D000C7FBA0B9BAF1020FDDD0D7E72046294639
:10D0E00000F07CFE22462B4601F0B0FBA0B9244B99
:10D0F00099F900A04FF06042CDE90823EAE7204605
:10D10000294600F06BFE22462B4601F09FFB18B922
:10D11000184B0022CDE9082399F900A0DAE7012293
:10D12000134BCDF828800292CDE90467CDE906457E
:10D130000393BAF1000FB8D000220023104619461D
:10D1400001F046FABAF1020FCDE908013FF43EAF13
:10D15000AFE700BFAFF30080000000000000000058
:10D16000000000000000F03F000000000000F07F21
:10D170006C3A01000000F0FF0000F03F0000E03FCB
:10D18000FFFFEFC734000020FFFFEF470000000063
:10D190002DE9F04F23F0004555EA020493B00DD07D
:10D1A0006B4E21F00044B4420F4682460BDD04F181
:10D1B000404404F5801454EA0A0350D16549002024
:10D1C00013B0BDE8F08F9B46944647D0B542EEDCE5
:10D1D0005F4EB5425DD0002F80468946CDE90023E1
:10D1E0005BDB0026BCF1000F0ED1594B9D423FD0B6
:10D1F000584B9D4200F08880BBF1804F00F09C802E
:10D20000554B9B4500F0B8834046494600F0D4FD9D
:10D21000BAF1000F06D1002C59D04E4B27F04042F6
:10D220009A4254D0FF0F013F56EA070373D04B4B8D
:10D230009D4240F39B8003F104739D4240F33E8482
:10D24000474B9C4272DDBBF1000F72DD3EA3D3E978
:10D2500000231046194601F091F8B1E728B1414882
:10D2600013B0BDE8F04F00F0B3BDA542F7DCAFE767
:10D2700004F1404303F5801353EA0A039ED0384B70
:10D280009C4240F38383BBF1000F52DBDDE90001D8
:10D2900096E7BCF1000F9ED089E7334B9D4231DC0D
:10D2A000A3F154739D429CDD2B15A3F2FF33142B85
:10D2B00040F3A583C3F134032CFA03F202FA03F31B
:10D2C00063458ED102F00102C2F102068AE7BBF18A
:10D2D000000F05DA02460B4600201E4901F078F9DE
:10D2E000002FBFF66DAF04F1404404F5801454EAFA
:10D2F000060300F03F84012E7FF462AF01F100438A
:10D3000019465DE702266DE7BBF1000FC0F24883C6
:10D310004046494654E742464B461046194600F0FF
:10D3200075FE02460B4601F053F949E7BBF1000FC9
:10D330008CDB0020002143E742464B4640464946ED
:10D3400001F01CF83CE700BF9C7500883CE4377E88
:10D350000000F07F0000F03F0000E03F0000E041EF
:10D36000FFFFEF3F703A0100FFFF3F43B4F5801F1E
:10D3700080F261830022D24B01F000F86FF0340C90
:10D380000C462315CF4DC4F31302A3F2FF3342F032
:10D390007F546344AA420B9344F4401440F33F8308
:10D3A000C94B9A4240F304849FEDAF7B8DED087B1F
:10D3B0008DED107B9FEDAE7B0B9B8DED067B0133DE
:10D3C0000B93A4F580140025DDE90623214682464F
:10D3D00000F01CFEA346DDE9062380468946504640
:10D3E0002146CDE90CAB00F013FE02460B460020AF
:10D3F000B64901F0EDF80A460146CDE90E12134692
:10D4000049460246404600F0B9FF631043F000531E
:10D4100082468B4603F500238C46CDE904AB5919AF
:10D42000D3460023CDE902BC0293DDE902AB002024
:10D4300004460D4602460B465046594600F09EFFF4
:10D4400002460B464046494600F0E0FDDDE9062372
:10D45000804689462046294600F0D8FD02460B4604
:10D46000DDE90C0100F0D2FD52465B4600F086FF7C
:10D4700002460B464046494600F0C8FDDDE90E2352
:10D4800000F07CFFDDE90445CDE9060122462B468C
:10D490002046294600F072FF77A3D3E90023044613
:10D4A0000D4600F06BFF76A3D3E9002300F0B0FD3A
:10D4B00022462B4600F062FF73A3D3E9002300F05D
:10D4C000A7FD22462B4600F059FF71A3D3E90023A4
:10D4D00000F09EFD22462B4600F050FF6EA3D3E9DC
:10D4E000002300F095FD22462B4600F047FF6CA379
:10D4F000D3E9002300F08CFD2246804689462B4666
:10D500002046294600F03AFF02460B46404649466F
:10D5100000F034FF524604460D465B46DDE9040147
:10D5200000F076FDDDE9062300F028FF22462B46B9
:10D5300000F06EFD5246804689465B46504659468D
:10D5400000F01CFF0022624BCDE90C0100F060FDF1
:10D5500042464B4600F05CFD02980D4604462246CA
:10D560002B465046594600F009FF002282468B4662
:10D57000574B2046294600F049FDDDE90C2300F019
:10D5800045FD02460B464046494600F03FFDDDE9B9
:10D59000042300F0F3FE2246804689462B46DDE94F
:10D5A000060100F0EBFE02460B464046494600F0FD
:10D5B0002FFD8046894602460B465046594600F0EC
:10D5C00027FD029838A3D3E9002304460D4600F056
:10D5D000D5FE5246CDE904015B462046294600F0BF
:10D5E00015FD02460B464046494600F00FFD30A3AC
:10D5F000D3E9002300F0C2FE2FA3D3E90023804625
:10D6000089462046294600F0B9FE02460B464046B0
:10D61000494600F0FDFCDDE9102300F0F9FC8046EE
:10D620000B98894600F040FE424682468B464B46A8
:10D63000DDE9040100F0ECFCDDE9082300F0E8FC82
:10D6400052465B4600F0E4FC029852465B460446B4
:10D650000D4600F0DBFCDDE9082300F0D7FCDDE936
:10D66000042337E0AFF3008000000000000000005A
:10D67000000000000000F03FEF4E454A287ECA3F00
:10D6800065DBC9934A86CD3F01411DA96074D13F36
:10D690004D268F515555D53FFFAB6FDBB66DDB3F48
:10D6A000033333333333E33F000000E009C7EE3F79
:10D6B000FD033ADC09C7EE3FF5015B14E02F3EBEE7
:10D6C000000040438E98030079B60B000000F03F45
:10D6D0000000084000F09AFC0B46024649464046CE
:10D6E00000F094FC013E56EA070382468B4600F0A8
:10D6F0005E819FEDD37B8DED047BDDE9001200237D
:10D700000E461746CDE902670293DDE90267084637
:10D710003B461146324600F079FC22462B4600F08B
:10D720002DFEDDE90023804689465046594600F02B
:10D7300025FE02460B464046494600F069FC32464B
:10D74000804689463B4620462946CDE9008900F0BF
:10D7500015FE0B46024606460F464046494600F077
:10D7600057FCD14B994204460D468A4640F324812A
:10D7700001F13F4303F5E003034340F0FF81B2A30F
:10D78000D3E90023DDE9000100F042FC3246804687
:10D7900089463B462046294600F038FC02460B46A7
:10D7A0004046494601F07AF8002840F0E781A84653
:10D7B0004FEA2853A3F2FE324FF48013134153442F
:10D7C000C3F30A52B94DA2F2FF321541C3F3130459
:10D7D00023EA05010020C2F1140B44F48014BAF1CD
:10D7E000000F02460B4644FA0BFB30463946B8BFE1
:10D7F000CBF1000B00F00AFC06460F463246DDE98D
:10D8000000013B4600F004FC4FEA0B5A0D46002491
:10D810008FA3D3E900232046294600F0AFFD32460E
:10D82000804689463B462046294600F0EFFB0246EB
:10D830000B46DDE9000100F0E9FB87A3D3E90023F3
:10D8400000F09CFD86A3D3E9002306460F46204640
:10D85000294600F093FD02460B463046394600F05B
:10D86000D7FB06460F4602460B464046494600F0A7
:10D87000CFFB42464B4604460D4600F0C7FB02462E
:10D880000B463046394600F0C1FB224680468946A9
:10D890002B462046294600F071FD73A3D3E90023EF
:10D8A00006460F4600F06AFD71A3D3E9002300F09D
:10D8B000ADFB32463B4600F061FD6FA3D3E9002388
:10D8C00000F0A6FB32463B4600F058FD6CA3D3E9BE
:10D8D000002300F09BFB32463B4600F04FFD6AA35D
:10D8E000D3E9002300F094FB32463B4600F046FDAE
:10D8F00002460B462046294600F088FB06460F46A6
:10D9000002460B462046294600F038FD0022CDE9AC
:10D9100000014FF080433046394600F077FB024665
:10D920000B46DDE9000100F053FE424606460F4675
:10D930004B462046294600F021FD42464B4600F06A
:10D9400067FB02460B463046394600F05FFB224635
:10D950002B4600F05BFB02460B460020544900F0CA
:10D9600055FB8A44BAF5801FC0F232815146DDE989
:10D97000042300F003FD23E4002FFFF645AC4046EE
:10D98000494613B0BDE8F04F00F056B9BBF1000FA7
:10D99000BFF6CFACDDE90034184604F100410FE4D6
:10D9A00042464B460020424900F012FE08E49FED3B
:10D9B000387B8DED047BA0E63E4B21F00048984576
:10D9C00040F3EA803C4B0B4403430AD132463B46CA
:10D9D00000F01CFBDDE9002300F056FF00283FF4B7
:10D9E000E7AEDDE904012CA3D3E9002300F0C6FC77
:10D9F00029A3D3E9002300F0C1FCFFF7E1BBBCF190
:10DA0000000F40F0D280C3F1140345FA03F202FA8A
:10DA100003F3AB4200F0E0806646FFF7E9BB9FED01
:10DA2000207B8DED087B8DED107B9FED057B002528
:10DA30008DED067BC8E44FF0000CA2E4AFF300804C
:10DA4000000000000000F03FFE822B654715973C68
:10DA500000000000432EE63FEF39FAFE422EE63F7B
:10DA6000396CA80C615C20BED0A4BE726937663EDA
:10DA7000F16BD2C541BDBB3E2CDE25AF6A56113FCE
:10DA800093BDBE166CC1663F3E5555555555C53FB5
:10DA9000000000000000F0BF59F3F8C21F6EA5019E
:10DAA0000000000000000000FFFF8F40FFFF0F009C
:10DAB0000000F03FFFCB904000346F3F5A4B9C4238
:10DAC0007FF734AC594B9C423FF7BDAB0022574B1C
:10DAD00000F09CFA44A3D3E9002304460D4600F06D
:10DAE0004DFC43A3D3E9002382468B4620462946BA
:10DAF00000F044FC0022CDE902014D4B20462946AE
:10DB000000F03CFC02460B463BA1D1E9000100F0CD
:10DB10007DFA22462B4600F031FC02460B460020DF
:10DB2000444900F073FA2246804689462B46204637
:10DB3000294600F023FC02460B464046494600F0C9
:10DB40001DFC2FA3D3E9002300F018FC02460B466E
:10DB5000DDE9020100F05AFA02460B46804689468A
:10DB60005046594600F054FA002004460D465246ED
:10DB70005B46AFE502460B46FFF7CFBBDDE904018C
:10DB800021A3D3E9002300F0F9FB1FA3D3E900236D
:10DB900000F0F4FBFFF714BB264B98453FF708AEA7
:10DBA000DDE902239246934631E60026FFF72CBBBF
:10DBB0009FED177B8DED087B9FED177B8DED107B27
:10DBC0009FED177B4FF480258DED067BFFF7FCBBA7
:10DBD0005A4600F091F9CAE602F00102C2F10206CB
:10DBE000FFF706BBAFF30080000000604715F73F6A
:10DBF00044DF5DF80BAE543E555555555555D53F50
:10DC0000FE822B654715F73F9C7500883CE4377E04
:10DC10000000004003B8E23F06D0CF43EBFD4C3E8E
:10DC2000000000000000F83FFEFFEF3F0000F03F63
:10DC30000000D03F0000E03F5E4A8A432DE9F041FA
:10DC400004460D4600F0958000290B4606468446A2
:10DC500056DD0F1500F0A580C3F31303A7F2FF37BD
:10DC600043F480134FEADC72F80702EB43034FEAF8
:10DC70004C0504D5ED0F05EB43034FEA8C05002658
:10DC80007F10B44616224FF400110CEB01009842AD
:10DC90004FEAD5744FEA450503DC1B1A00EB010C73
:10DCA0000E44013A04EB43034FEA5101EDD1104613
:10DCB000964620244FF0004209E051D05B00013C21
:10DCC00003EBD5734FEA52024FEA450537D063455F
:10DCD00002EB0E01F1DD002901EB020E0ADBE0464A
:10DCE000A3EB0C03A94288BF03F1FF336D1A104464
:10DCF000C446E3E7BEF1000FF1DB0CF10108EFE7EA
:10DD000021F00042024329D0002942D10146CA0A2B
:10DD1000153B4905002AFAD012F4801001D044E0E6
:10DD200060465200D40200F1010CF9D5CCF1200478
:10DD300001FA0CFCE1401F1A41EA02038CE72B4375
:10DD400021D14408731003F17F53F20703F5001348
:10DD500048BF44F0004403EB07512046BDE8F08182
:10DD6000A942ABD8002901EB020EC3DB9846002381
:10DD7000BCE702460B4600F001FB22462B4600F0B2
:10DD800047F9BDE8F081411C16BF421C013654081A
:10DD9000D8E7024600F03AF902460B4600F018FCBC
:10DDA000DCE71A4631463B46B6E78C4620244FF066
:10DDB000FF30BFE70000F07F21F0004319467047B5
:10DDC00041F0004101F58010C00F704700207047FE
:10DDD00000200149704700BF0000F87F2DE9F041A5
:10DDE000C1F30A57A7F2FF35132D82B002460B4646
:10DDF0000C464FEAD178064633DC002D4EDB3C4919
:10DE0000294103EA0100104326D049080B4052EA99
:10DE100003060CD04FF48023132D24EA010143FAAA
:10DE200005F444EA01040CBF4FF0004600263149D6
:10DE300001EBC8082346D8E900453246204629466A
:10DE400000F0E6F8CDE9000122462B46DDE90001AD
:10DE500000F0DCF802460B461046194602B0BDE859
:10DE6000F081332D07DDB5F5806FF5D100F0D0F8E6
:10DE700002460B46F0E7A7F213474FF0FF31F94097
:10DE80000842E9D049080842D1D04FF0804320EA47
:10DE9000010143FA07F741EA0706C8E721F000410C
:10DEA0000143D9D0C3F3130101434E420E43114D38
:10DEB0005C0C360B640406F4002305EBC80243EA4D
:10DEC0000401D2E900450B4602462946204600F0EF
:10DED0009FF8CDE9000122462B46DDE9000100F064
:10DEE00095F821F00041024641EAC873B4E700BF4B
:10DEF000FFFF0F00783A0100F8B5C1F30A5304465A
:10DF00000D460E4617460BBB21F000460346334331
:10DF10001BD0354B002200F031FA344B9F420446AF
:10DF20000D4635DBC1F30A530E46363B3B4440F207
:10DF3000FE72934232DC002B11DD26F0FF4626F400
:10DF4000E00646EA035520462946F8BD40F2FF7236
:10DF50009342EBD102460B4600F05AF8F8BD13F19C
:10DF6000350F28DA4CF250339F4222462B460ADD09
:10DF700019A1D1E9000100F03DF817A3D3E900236E
:10DF800000F0FCF9F8BD16A1D1E9000100F032F86B
:10DF900013A3D3E9002300F0F1F9F8BD22462B4684
:10DFA0000DA1D1E9000100F025F80BA3D3E900236E
:10DFB00000F0E4F9F8BD26F0FF4626F4E00636331B
:10DFC00046EA0355204629460022094B00F0D6F9BF
:10DFD000F8BD00BFAFF300809C7500883CE4377E3D
:10DFE00059F3F8C21F6EA50100005043B03CFFFF7B
:10DFF0000000903C03F0004321F0004242EA03019C
:10E00000704700BF81F0004102E000BF83F0004391
:10E0100030B54FEA41044FEA430594EA050F08BFC3
:10E0200090EA020F1FBF54EA000C55EA020C7FEA87
:10E03000645C7FEA655C00F0E2804FEA5454D4EB04
:10E040005555B8BF6D420CDD2C4480EA020281EACE
:10E05000030382EA000083EA010180EA020281EA06
:10E060000303362D88BF30BD11F0004F4FEA013158
:10E070004FF4801C4CEA113102D0404261EB410167
:10E0800013F0004F4FEA03334CEA133302D05242ED
:10E0900063EB430394EA050F00F0A780A4F10104A9
:10E0A000D5F1200E0DDB02FA0EFC22FA05F28018E3
:10E0B00041F1000103FA0EF2801843FA05F35941C9
:10E0C0000EE0A5F120050EF1200E012A03FA0EFC48
:10E0D00028BF4CF0020C43FA05F3C01851EBE37172
:10E0E00001F0004507D54FF0000EDCF1000C7EEB8F
:10E0F00000006EEB0101B1F5801F1BD3B1F5001FCD
:10E100000CD349085FEA30004FEA3C0C04F10104EB
:10E110004FEA445212F5800F80F09A80BCF1004F14
:10E1200008BF5FEA500C50F1000041EB045141EA96
:10E13000050130BD5FEA4C0C404141EB010111F497
:10E14000801FA4F10104E9D191F0000F04BF014642
:10E150000020B1FA81F308BF2033A3F10B03B3F120
:10E1600020020CDA0C3208DD02F1140CC2F10C02B0
:10E1700001FA0CF021FA02F10CE002F11402D8BF0E
:10E18000C2F1200C01FA02F120FA0CFCDCBF41EADA
:10E190000C019040E41AA2BF01EB0451294330BDA9
:10E1A0006FEA04041F3C1CDA0C340EDC04F1140486
:10E1B000C4F1200220FA04F001FA02F340EA03005D
:10E1C00021FA04F345EA030130BDC4F10C04C4F1A3
:10E1D000200220FA02F001FA04F340EA0300294683
:10E1E00030BD21FA04F0294630BD94F0000F83F4CD
:10E1F000801306BF81F480110134013D4EE77FEAB0
:10E20000645C18BF7FEA655C29D094EA050F08BFFB
:10E2100090EA020F05D054EA000C04BF19461046DC
:10E2200030BD91EA030F1EBF0021002030BD5FEA20
:10E23000545C05D14000494128BF41F0004130BD48
:10E2400014F580043CBF01F5801130BD01F000459C
:10E2500045F0FE4141F470014FF0000030BD7FEA0F
:10E26000645C1ABF194610467FEA655C1CBF0B460A
:10E27000024650EA013406BF52EA033591EA030F21
:10E2800041F4002130BD00BF90F0000F04BF002119
:10E29000704730B54FF4806404F132044FF000054C
:10E2A0004FF0000150E700BF90F0000F04BF0021C5
:10E2B000704730B54FF4806404F1320410F000452B
:10E2C00048BF40424FF000013EE700BF42004FEA26
:10E2D000E2014FEA31014FEA02701FBF12F07F43A3
:10E2E00093F07F4F81F06051704732F07F4208BF5A
:10E2F000704793F07F4F04BF41F40021704730B561
:10E300004FF4607401F0004521F000411CE700BFAC
:10E3100050EA010208BF704730B54FF000050AE02F
:10E3200050EA010208BF704730B511F0004502D530
:10E33000404261EB41014FF4806404F132045FEA32
:10E34000915C3FF4D8AE4FF003025FEADC0C18BFDB
:10E3500003325FEADC0C18BF033202EBDC02C2F1CD
:10E36000200300FA03FC20FA02F001FA03FE40EA5F
:10E370000E0021FA02F11444BDE600BF70B54FF063
:10E38000FF0C4CF4E06C1CEA11541DBF1CEA135541
:10E3900094EA0C0F95EA0C0F00F0DEF82C4481EAA9
:10E3A000030621EA4C5123EA4C5350EA013518BFC9
:10E3B00052EA033541F4801143F4801338D0A0FBB6
:10E3C00002CE4FF00005E1FB02E506F00042E0FB63
:10E3D00003E54FF00006E1FB03569CF0000F18BF69
:10E3E0004EF0010EA4F1FF04B6F5007F64F5407411
:10E3F00004D25FEA4E0E6D4146EB060642EAC621A4
:10E4000041EA55514FEAC52040EA5E504FEACE2E10
:10E41000B4F1FD0C88BFBCF5E06F1ED8BEF1004F13
:10E4200008BF5FEA500E50F1000041EB045170BD8F
:10E4300006F0004646EA010140EA020081EA0301D3
:10E44000B4EB5C04C2BFD4EB0C0541EA045170BDCF
:10E4500041F480114FF0000E013C00F3AB8014F149
:10E46000360FDEBF002001F0004170BDC4F1000492
:10E47000203C35DA0C341BDC04F11404C4F1200513
:10E4800000FA05F320FA04F001FA05F240EA02006E
:10E4900001F0004221F0004110EBD37021FA04F6A4
:10E4A00042EB06015EEA430E08BF20EAD37070BD5E
:10E4B000C4F10C04C4F1200500FA04F320FA05F0BD
:10E4C00001FA04F240EA020001F0004110EBD370BF
:10E4D00041F100015EEA430E08BF20EAD37070BD2F
:10E4E000C4F1200500FA05F24EEA020E20FA04F308
:10E4F00001FA05F243EA020321FA04F001F00041B7
:10E5000021FA04F220EA020000EBD3705EEA430E27
:10E5100008BF20EAD37070BD94F0000F0FD101F056
:10E520000046400041EB010111F4801F08BF013C8F
:10E53000F7D041EA060195F0000F18BF704703F0CD
:10E540000046520043EB030313F4801F08BF013D54
:10E55000F7D043EA0603704794EA0C0F0CEA135510
:10E5600018BF95EA0C0F0CD050EA410618BF52EACA
:10E570004306D1D181EA030101F000414FF00000D0
:10E5800070BD50EA410606BF1046194652EA4306DE
:10E5900019D094EA0C0F02D150EA013613D195EA52
:10E5A0000C0F05D152EA03361CBF104619460AD19A
:10E5B00081EA030101F0004141F0FE4141F47001A4
:10E5C0004FF0000070BD41F0FE4141F4780170BD94
:10E5D00070B54FF0FF0C4CF4E06C1CEA11541DBFF9
:10E5E0001CEA135594EA0C0F95EA0C0F00F0A7F8FB
:10E5F000A4EB050481EA030E52EA03354FEA013128
:10E6000000F088804FEA03334FF0805545EA13133A
:10E6100043EA12634FEA022245EA111545EA106502
:10E620004FEA00260EF000419D4208BF964244F199
:10E63000FD0404F5407402D25B084FEA3202B61AB8
:10E6400065EB03055B084FEA32024FF480104FF48C
:10E65000002CB6EB020E75EB030E22BFB61A754600
:10E6600040EA0C005B084FEA3202B6EB020E75EB93
:10E67000030E22BFB61A754640EA5C005B084FEAFB
:10E680003202B6EB020E75EB030E22BFB61A7546C8
:10E6900040EA9C005B084FEA3202B6EB020E75EBD3
:10E6A000030E22BFB61A754640EADC0055EA060E94
:10E6B00018D04FEA051545EA16754FEA06164FEAD7
:10E6C000C30343EA52734FEAC2025FEA1C1CC0D183
:10E6D00011F4801F0BD141EA00014FF000004FF010
:10E6E000004CB6E711F4801F04BF01430020B4F1D1
:10E6F000FD0C88BFBCF5E06F3FF6AFAEB5EB030C89
:10E7000004BFB6EB020C5FEA500C50F1000041EB85
:10E71000045170BD0EF0004E4EEA113114EB5C0452
:10E72000C2BFD4EB0C0541EA045170BD41F4801125
:10E730004FF0000E013C90E645EA060E8DE60CEA2D
:10E74000135594EA0C0F08BF95EA0C0F3FF43BAF4A
:10E7500094EA0C0F0AD150EA01347FF434AF95EA01
:10E760000C0F7FF425AF104619462CE795EA0C0FE5
:10E7700006D152EA03353FF4FDAE1046194622E7B2
:10E7800050EA410618BF52EA43067FF4C5AE50EA8C
:10E7900041047FF40DAF52EA43057FF4EBAE12E77C
:10E7A0004FF0FF3C06E000BF4FF0010C02E000BF5D
:10E7B0004FF0010C4DF804CD4FEA410C7FEA6C5C40
:10E7C0004FEA430C18BF7FEA6C5C1BD001B050EAE3
:10E7D000410C0CBF52EA430C91EA030F02BF90EACE
:10E7E000020F0020704710F1000F91EA030F58BF8D
:10E7F000994208BF90422CBFD8176FEAE37040F0EF
:10E80000010070474FEA410C7FEA6C5C02D150EA8C
:10E81000013C07D14FEA430C7FEA6C5CD6D152EA47
:10E82000033CD3D05DF8040B704700BF844610460C
:10E8300062468C461946634600E000BF01B5FFF70B
:10E84000B7FF002848BF10F1000F01BD4DF808EDDB
:10E85000FFF7F4FF0CBF012000205DF808FB00BFAC
:10E860004DF808EDFFF7EAFF34BF012000205DF806
:10E8700008FB00BF4DF808EDFFF7E0FF94BF012053
:10E8800000205DF808FB00BF4DF808EDFFF7CEFF54
:10E8900094BF012000205DF808FB00BF4DF808ED93
:10E8A000FFF7C4FF34BF012000205DF808FB00BF64
:10E8B0004FEA410C7FEA6C5C02D150EA013C0AD17C
:10E8C0004FEA430C7FEA6C5C02D152EA033C02D16E
:10E8D0004FF0000070474FF0010070474FEA4102CF
:10E8E00012F5001215D211D56FF47873B3EB6252A2
:10E8F00012D94FEAC12343F0004343EA505311F0C9
:10E90000004F23FA02F018BF404270474FF000005A
:10E91000704750EA013005D111F0004008BF6FF098
:10E92000004070474FF00000704700BF4A0011D20E
:10E9300012F5001211D20DD56FF47873B3EB625259
:10E940000ED44FEAC12343F0004343EA505323FA65
:10E9500002F070474FF00000704750EA013002D1DA
:10E960004FF0FF3070474FF0000070474FEA410210
:10E97000B2F1E04324BFB3F5001CDCF1FE5C0DD91D
:10E9800001F0004C4FEAC0024CEA5070B2F1004F67
:10E9900040EB830008BF20F00100704711F0804F6A
:10E9A00021D113F13872BCBF01F00040704741F42F
:10E9B00080114FEA5252C2F11802C2F1200C10FA33
:10E9C0000CF320FA02F018BF40F001004FEAC12317
:10E9D0004FEAD32303FA0CFC40EA0C0023FA02F3BB
:10E9E0004FEA4303CCE77FEA625307D150EA013391
:10E9F0001EBF4FF0FE4040F44000704701F0004061
:10EA000040F0FE4040F40000704700BF1FB51C46B8
:10EA1000094B1B680546D86852B1084B0091CDE9F7
:10EA2000013207492B46224600F0A8F901F044FDC7
:10EA3000044B1A46F2E700BF38000020883A010074
:10EA4000953A0100CE3801000A22002101F05EBB98
:10EA500010B5054C13462CB10A4601460220AFF30F
:10EA6000008010BD2046FCE700000000014B186844
:10EA7000704700BF3800002008B5074B044613B1AB
:10EA80000021AFF30080054B1868836A03B19847F3
:10EA9000204603F0EBFC00BF00000000243B010017
:10EAA0008A892DE9F041054610070C4658D44B6879
:10EAB000002B05DC0B6C002B02DC0020BDE8F08194
:10EAC000E66A002EF9D0002312F480522F68216AE2
:10EAD0002B6032D0606DA3895A0705D56368C01AD0
:10EAE000636B0BB1236CC01A00230246E66A216AED
:10EAF0002846B047431CA38906D129681D2948D858
:10EB0000294ACA40D60744D500226260D904226946
:10EB1000226004D5421C01D12B6803B96065616B8A
:10EB20002F600029C9D004F14403994202D028463D
:10EB300000F00AFA00206063C0E701232846B047CE
:10EB4000411CC8D12B68002BC5D01D2B01D0162B22
:10EB500001D12F60B1E7A38943F04003A381ADE762
:10EB60000F69002FA9D093070E6808BF4B690F608B
:10EB700018BF0023A6EB07088B60B8F1000F9CDDDF
:10EB800043463A46216AA66A2846B047002806DC72
:10EB9000A38943F04003A3814FF0FF308EE7074481
:10EBA000A8EB0008E9E700BF0100402038B50B6979
:10EBB00005460C46DBB118B183690BB900F072F859
:10EBC0000C4B9C4209D16C68B4F90C307BB12146E6
:10EBD0002846BDE83840FFF763BF074B9C4201D190
:10EBE000AC68F1E7054B9C4208BFEC68ECE70020FD
:10EBF00038BD00BFE43A0100043B0100C43A010003
:10EC0000014620B9044B0549186800F0C9B8044B07
:10EC10001868FFF7CBBF00BF243B0100ADEB00003D
:10EC200038000020002310B50446C0E9003383609B
:10EC300081814366C281C0E9043383611946082299
:10EC40005C3000F078F9054B6362054BA362054B1D
:10EC5000E362054B2462236310BD00BF29FD000061
:10EC60004FFD000087FD0000ABFD0000014900F0F2
:10EC700097B800BFADEB000070B54A1E682555433C
:10EC80000E4605F1740100F0ADF9044640B10021D3
:10EC9000C0E900160C30A06005F1680200F04BF9E5
:10ECA000204670BD836910B5044633BBC0E91233FA
:10ECB0000365124B124A1B688262984204BF01230B
:10ECC000836100F01FF86060204600F01BF8A06030
:10ECD000204600F017F80022E06004216068FFF78A
:10ECE000A1FF01220921A068FFF79CFF0222122147
:10ECF000E068FFF797FF0123A36110BD243B0100EB
:10ED00006DEC0000F8B51B4B1E68B369074613B9DC
:10ED10003046FFF7C7FF4836D6E90134013B03D53B
:10ED2000336833B13668F7E7B4F90C506DB1683425
:10ED3000F4E704213846FFF79FFF30600028F1D147
:10ED40000C233B6004462046F8BD0B4B6566C4E9C6
:10ED50000055A560C4E90335C4E9055508222946D4
:10ED600004F15C0000F0E7F8C4E90D55C4E9125560
:10ED7000E9E700BF243B01000100FFFF0EB403B52B
:10ED8000014603AB054853F8042B0068019300F0DB
:10ED9000ADF902B05DF804EB03B070473800002015
:10EDA0002DE9F8438046894600F14804002614B94D
:10EDB0003046BDE8F883D4E90175013F01D52468E8
:10EDC000F5E7AB89012B07D9B5F90E30013303D034
:10EDD00029464046C84706436835EEE770B50D4EF4
:10EDE0000D4CA41BA4100025A54209D10B4E0C4CC0
:10EDF00003F03EFBA41BA4100025A54205D170BD65
:10EE000056F8253098470135EEE756F825309847F3
:10EE10000135F2E708020020080200200802002065
:10EE20008402002010B5044600F022F82044407807
:10EE300000F0440010BD931E222B10B50C4604D9DF
:10EE400000230B701C46204610BD0A2A09D1002859
:10EE500007DA2D230B7040420121214401F00EFA04
:10EE6000F1E70021F9E7FFF7E6BFD0F8EC007047C3
:10EE7000044B054A1B681B6A002B08BF1346D3F8D6
:10EE8000EC007047380000209C000020024B014637
:10EE9000186800F0A7B800BF38000020024B0146F8
:10EEA000186800F051B800BF3800002082B001B9E6
:10EEB00001A942B14BB113780B601278101C18BF36
:10EEC000012002B070471046FBE76FF00100F8E741
:10EED00030B50024A24201D1002007E0035D0134D7
:10EEE0000D1915F8015CAB42F4D0581B30BD10B5BC
:10EEF000431E0A44914200D110BD11F8014B03F8A2
:10EF0000014FF7E7884210B501EB020307D8421E14
:10EF100099420AD011F8014B02F8014FF8E78342F9
:10EF2000F5D98118D21AD34200D110BD13F8014D82
:10EF300001F8014DF7E702440346934200D17047C0
:10EF400003F8011BF9E7000038B50546002945D054
:10EF500051F8043C0C1F002BB8BFE41802F0E8F98C
:10EF60001F4A1368104633B9636014602846BDE831
:10EF7000384002F0DEB9A3420CD9216862189342EE
:10EF800004BF1A685B68636004BF521822600460A3
:10EF9000ECE713465A680AB1A242FAD91968581820
:10EFA000A0420BD120680144581882421960DDD17B
:10EFB000106852685A6001441960D7E702D90C23DF
:10EFC0002B60D3E7206821188A4204BF1168526879
:10EFD000626004BF091821605C60C7E738BD00BFEC
:10EFE0004407002070B5CD1C25F0030508350C2D15
:10EFF00038BF0C25002D064601DBA94203D90C239E
:10F000003360002070BD02F093F9214A1468214654
:10F0100091B9204C23681BB9304600F017FE2060E0
:10F020002946304600F012FE431C24D10C233360E5
:10F03000304602F07EF9E4E70B685B1B18D40B2B1B
:10F040000FD90B60CD50CC18304602F072F904F1A4
:10F050000B00231D20F00700C31AD3D05A42E25000
:10F06000D0E78C424B6816BF636013600C46EBE739
:10F070000C464968CCE7C41C24F00304A04205D028
:10F08000211A304600F0E2FD0130CFD02560DBE7E9
:10F0900044070020480700209368013B002B10B470
:10F0A000936008DA9469A34201DB0A2903D15DF871
:10F0B000044B01F021B91368581C10601970084600
:10F0C0005DF8044B7047F8B506460F461446D51850
:10F0D000AC4201D1002007E03A4614F8011B30464B
:10F0E000FFF7DAFF431CF3D1F8BD00002DE9F04F24
:10F0F0009DB00C4617460393064618B183690BB9B9
:10F10000FFF7D0FD7B4B9C4257D17468A389180749
:10F110005DD52369002B5AD00023099320238DF855
:10F12000293030238DF82A304FF0010BB846454680
:10F1300015F8013B0BB1252B54D1B8EB070A0BD0C6
:10F1400053463A4621463046FFF7BDFF013000F0F6
:10F15000C280099B5344099398F80030002B00F0BB
:10F16000BA8000234FF0FF32CDE9052304930793C3
:10F170008DF853301A93A846052218F8011B5E48F3
:10F1800002F086F8049B78BBD90644BF20228DF894
:10F1900053201A0744BF2B228DF853202A782A2A9D
:10F1A0002AD0079AA84600200A25414611F8013BBB
:10F1B000303B092B69D960B324E0504B9C4201D10C
:10F1C000B468A3E74E4B9C4208BFF4689EE7214613
:10F1D000304601F003F900289ED04FF0FF301DB0FB
:10F1E000BDE8F08FA846A2E7434A801A0BFA00F068
:10F1F000184304904546BEE7039A111D1268039117
:10F20000002A01DB079204E0524243F00203079216
:10F21000049398F800302E2B0ED198F801302A2B49
:10F2200038D1039B1A1D1B680392002BB8BF4FF007
:10F23000FF3308F102080593324D98F800100322BD
:10F24000284602F025F840B14023401B03FA00F0A5
:10F25000049B034308F10108049398F800102A481E
:10F260008DF82810062208F1010702F011F8002895
:10F2700037D0264B1BBB039B073323F00703083310
:10F280000393099B4B44099350E705FB023201208D
:10F2900088468AE7002308F10108059319460A25E4
:10F2A000404610F8012B303A092A03D9002BC3D06D
:10F2B0000591C1E705FB012101238046F0E703AB7F
:10F2C00000932246124B04A9304600F0B5F8B0F185
:10F2D000FF3F8146D5D1A3895B063FF57EAF0998F4
:10F2E0007DE703AB00932246094B04A9304600F0AA
:10F2F0005FFBECE7E43A01002E3B0100043B010018
:10F30000C43A0100343B0100383B010039F40000ED
:10F31000C7F000002DE9F04788B0002B149F109E25
:10F32000DDE9121A1D4627F02007BBBF03F1004399
:10F330001D4600232D231446B8BF1446462F0B70DC
:10F3400004D0452F00D10136022300E0032307AA91
:10F35000049206AACDE902A2CDE9003622462B4648
:10F3600001F04EF9472F804602D1119BDB0726D5CD
:10F37000462F08EB060911D198F80030302B0AD13E
:10F380000022002320462946FFF760FA18B9C6F18B
:10F390000106CAF80060DAF8003099440022002320
:10F3A00020462946FFF752FA38B93022079B4B45D1
:10F3B00005D2591C07911A70F8E7CDF81C90079BED
:10F3C000159AA3EB08034046136008B0BDE8F08728
:10F3D000F7B500290446BABF49422D232B2309293A
:10F3E00004F8022B437020DD0DF107031F460A26A7
:10F3F00091FBF6F506FB15113031092D03F8011CC0
:10F4000003F1FF32294609DC3031023B02F8011CCE
:10F41000BB42224604D3101A03B0F0BD1346E7E7FF
:10F4200013F8012B04F8012BF2E730231944837001
:10F43000021DC170EFE700002DE9F04F91B00C46BE
:10F44000DDF8688016461F46054601F097FE036802
:10F450000893184600F015FD00230E93D8F80030ED
:10F460000990073323F0070303F1080294F818A06A
:10F47000D4F800B0C8F80020D3E90023C4E912236F
:10F48000D4E9128929F000430B93CDF828804FF07E
:10F49000FF32A94BDDE90A01FFF70AFA70BB4FF012
:10F4A000FF32A54BDDE90A01FFF7E4F930BB00228A
:10F4B000002340464946FFF7D3F910B12D2384F8C5
:10F4C00043309E4A9E4BBAF1470F8CBF90469846F8
:10F4D000032323612BF0040323604FF000090097FE
:10F4E00033460FAA2146284600F0ECF9013040F0DF
:10F4F00090804FF0FF3011B0BDE8F08F42464B4690
:10F5000040464946FFF7D4F910B18E4A8E4BDAE7F0
:10F510006368591C4BF480620EA90DA840D10623E4
:10F5200063600DF13303CDE901234FF0000C6368F4
:10F530002260CDE9030A009342464B46CDE9051C03
:10F540002846FFF7E7FE0AF0DF03472B804609D184
:10F550000D9BD81C02DB6268934247DDAAF1020AC8
:10F560005FFA8AFABAF1650F0D9924D8013952462B
:10F5700004F150000D91FFF72BFF0E9A1318012A8A
:10F580008146236102DC2268D10701D50133236162
:10F590009DF83330002BA2D02D2384F843309EE712
:10F5A000BAF1670F00F07881BAF1470FB9D1002B9B
:10F5B000B7D10123B4E7BAF1660F19D10029636806
:10F5C0000CDD216113B92268D20702D501330B4447
:10F5D00023610D9BA3654FF00009D9E713B9226899
:10F5E000D00701D50233F3E70123F1E74FF0670AB3
:10F5F000DDE90D32934205DB22682361D107E8D5AE
:10F600000133E5E7002BD4BFC3F102030123134408
:10F61000DEE723685A0507D4236942463146284667
:10F62000B84701302BD164E7BAF1650F40F2DD80B5
:10F6300000220023D4E91201FFF708F9002833D093
:10F640000123424A31462846B84701303FF451AFC2
:10F65000DDE90D239A4202DB2368D8070FD5DDE9E7
:10F66000082331462846B84701303FF442AF4FF0F7
:10F67000000804F11A090E9B013B434509DC23688D
:10F680009B0700F10481E0680F9B9842B8BF1846C1
:10F6900031E701234A4631462846B84701303FF456
:10F6A00028AF08F10108E6E70D9B002B2BDC0123B6
:10F6B000264A31462846B84701303FF41AAF0D9B21
:10F6C00023B90E9B13B92368D907D8D5DDE90823E0
:10F6D00031462846B84701303FF40BAF4FF00009E0
:10F6E00004F11A0A0D9B5B424B4501DC0E9B94E72B
:10F6F0000123524631462846B84701303FF4F9AE5F
:10F7000009F10109EEE70E9AA36D9A42A8BF1A46C5
:10F71000002A914607DD1346314642462846B8473F
:10F7200001303FF4E6AE04F11A034FF0000B29EA72
:10F73000E9790A9316E000BFFFFFEF7F80390100EF
:10F740003F3B01007C390100433B01006C38010064
:10F7500001230A9A31462846B84701303FF4C9AE22
:10F760000BF1010BD4F858A0AAEB09035B45EFDCC1
:10F77000DDE90D239A42D04415DB2368DA0712D461
:10F780000E9B0D99A3EB0A02A3EB010A9245A8BFB9
:10F790009246BAF1000F0EDC4FF000082AEAEA7A2E
:10F7A00004F11A0919E0DDE9082331462846B84773
:10F7B0000130E5D19DE65346424631462846B847DA
:10F7C0000130E9D195E601234A4631462846B8473B
:10F7D00001303FF48EAE08F10108DDE90D239B1ADC
:10F7E000A3EB0A034345EEDC49E70E9A012A01DC4C
:10F7F000DB073AD50123424631462846B847013057
:10F800003FF477AEDDE9082331462846B84701309A
:10F8100008F101083FF46DAE0E9B002203F1FF3AA0
:10F82000D4E912010023FFF711F8C8B95346424644
:10F8300031462846B84701300ED15AE601235246D8
:10F8400031462846B84701303FF453AE08F101086D
:10F850000E9B013B4345F1DC4B4604F15002DDE6D3
:10F860004FF0000804F11A0AF2E70123DFE7012351
:10F870004A4631462846B84701303FF43AAE08F1CF
:10F880000108E3680F9A9B1A4345F0DCFBE64FF052
:10F89000000804F11909F4E7002B3FF48AAE4FF099
:10F8A000000CCDE9051C0DF133012260CDE9030AFE
:10F8B000CDE90121009342464B462846FFF72AFD39
:10F8C000804645E62DE9F04791461F468A680B6958
:10F8D000DDF820809342B8BF1346C9F8003091F894
:10F8E000432006460C4612B10133C9F800302368A4
:10F8F000990642BFD9F800300233C9F800302568B4
:10F9000015F0060507D104F1190AE368D9F80020BB
:10F910009B1AAB4228DC94F843302268003318BFAE
:10F92000012392062DD404F1430239463046C047E4
:10F93000013020D02368E568D9F8002003F00603E1
:10F94000042B08BFAD1AA36822690CBF25EAE57530
:10F9500000259342C4BF9B1AED184FF000091A34DA
:10F960004D451AD1002008E0012352463946304661
:10F97000C047013003D14FF0FF30BDE8F0870135BB
:10F98000C3E7E1185A1C302081F84300224494F860
:10F99000451082F843100233C5E701232246394659
:10F9A0003046C0470130E6D009F10109D8E7000030
:10F9B0002DE9F04301F1430C0C46097E85B06E2918
:10F9C0001746064698460C9A00F0B38022D8632961
:10F9D00036D00AD8002900F0B980582900F0838079
:10F9E00004F1420584F8421032E0642901D069290B
:10F9F000F6D120681368050603F104012AD51B68B7
:10FA00001160002B03DA2D225B4284F843206F48FB
:10FA10000A2239E0732900F09D8008D86F2920D090
:10FA20007029DDD1236843F02003236003E07529AA
:10FA300017D07829D4D1782384F84530644855E02C
:10FA40001368191D1B68116004F1420584F84230E7
:10FA500001238CE01B68116010F0400F18BF1BB22F
:10FA6000CFE713682568181D1060280601D51B68AC
:10FA700002E06806FBD51B8854486F2914BF0A2290
:10FA80000822002184F843106568A560002DC0F2AB
:10FA90009580216821F004012160002B3DD1002DCB
:10FAA00040F08E806546082A0BD12368DB0708D515
:10FAB000236962689A42DEBF302305F8013C05F1F4
:10FAC000FF35ACEB05032361CDF800803B4603AA6C
:10FAD00021463046FFF7F6FE01304DD14FF0FF30A2
:10FAE00005B0BDE8F083394884F8451013682168F3
:10FAF0001D1D1B6815600A060BD5CA0744BF41F0DF
:10FB0000200121601BB9226822F02002226010220D
:10FB1000B7E74D0648BF9BB2EFE76546B3FBF2F18E
:10FB200002FB1133C35C05F8013D0B460029F5D1FA
:10FB3000B9E7136825686169181D106028061B68FD
:10FB400001D5196002E06A06FBD519800023236104
:10FB50006546B9E71368191D11601D6862680021C8
:10FB6000284601F095FB08B1401B60606368236183
:10FB7000002384F84330A7E723692A4639463046F4
:10FB8000C0470130AAD023689B0713D4E068039BC9
:10FB90009842B8BF1846A3E701234A463946304683
:10FBA000C04701309AD00135E368039A9B1AAB42F3
:10FBB000F2DCEBE7002504F11909F5E7002BACD1E5
:10FBC000037884F8423004F142056CE7473B0100BA
:10FBD000583B010038B5134B1C68A36B7BB9182048
:10FBE000FFF754F9104A114BA063C0E90023104BF2
:10FBF00083600B23838101220023C0E90423A16BCE
:10FC00000C480A694B690C4C504304FB0300A2FBEF
:10FC100004230344541C43F10005C1E9044525F0C5
:10FC2000004038BD380000200E33CDAB34126DE6F5
:10FC3000ECDE05002DF451582D7F954C024B0A4601
:10FC40000146186801F060BE3800002038B5064C47
:10FC5000002305460846236002F0F2FB431C02D154
:10FC6000236803B12B6038BD500800200CB430B5B8
:10FC7000174B0C1E9DB01D6808DA8B232B604FF0CC
:10FC8000FF301DB0BDE8304002B070474FF4027342
:10FC9000ADF8143014BF04F1FF33234604930793E7
:10FCA0004FF6FF7302900690ADF81630209A21AB04
:10FCB00002A92846019301F0A7FE431CBCBF8B2379
:10FCC0002B60002CDDD0029B00221A70D9E700BF08
:10FCD000380000200EB430B59CB01FAC4FF4017258
:10FCE00054F8045BADF814200290069000F0C9F8B7
:10FCF0000B4B039007900B930A48019400230F933A
:10FD000014934FF6FF73ADF816302A46234602A926
:10FD1000006801F0C9FF1CB0BDE8304003B0704777
:10FD20004BFD00003800002010B50C46B1F90E1054
:10FD300002F062FA0028ABBF636DA3891B1823F49D
:10FD40008053ACBF6365A38110BD002070472DE9CF
:10FD5000F0411F468B89DB0505460C46164605D546
:10FD600002230022B1F90E1001F016FAA389B4F9AA
:10FD70000E1023F48053A38132463B462846BDE84B
:10FD8000F04100F019BB10B50C46B1F90E1001F0AE
:10FD900003FA431CA38915BF606523F4805343F421
:10FDA0008053A38118BFA38110BDB1F90E1000F0DC
:10FDB0008BBBF8B506460F4616F8014BFFF758F80F
:10FDC000204417F8015B437803F00303012B08BFBD
:10FDD0002034FFF74DF82844427802F00302012A4C
:10FDE00008BF2035601B01D1002DE5D1F8BD10B54D
:10FDF00003461A785C1C3AB9013B11F8012B03F851
:10FE0000012F002AF9D110BD2346F2E7C9B20346FB
:10FE100010F8012B1AB18A42F9D11846704700290F
:10FE200018BF0023F9E710F8012B11F8013B012A54
:10FE300028BF9A42F7D0D01A7047034611F8012B19
:10FE400003F8012B002AF9D170470000024B01464C
:10FE5000186800F003B800BF3800002070B50646EF
:10FE600008460C4600F00DF8451C29463046FFF7C1
:10FE7000B9F8064618B12A462146FFF738F8304649
:10FE800070BD034613F8012B002AFBD1181A013864
:10FE9000704730B503461C785D1C44B912F1FF323F
:10FEA00004D311F8014B03F8014B14B930BD2B46B4
:10FEB000F1E7002AF2D11A70F0E710B56AB1013902
:10FEC000841810F8013B11F8012F934203D1A0428E
:10FED00001D0002BF5D1981A10BD1046FCE770B583
:10FEE0000139044602B970BD234611F8015F03F8D9
:10FEF000015B561E2DB91444A342F4D003F8015BF4
:10FF0000FAE71C463246EDE710B5034601448B4242
:10FF100002D01A785C1C0AB9181A10BD2346F6E7FD
:10FF200038B503460D4669B9BDE83840FFF76EBFE6
:10FF3000431C044629461846FFF768FF0028F7D1FE
:10FF4000204638BD0024F5E7134B2DE9F0411D682C
:10FF5000AC6D06460F46B4B95020FEF797FFA86572
:10FF6000C0E90044C0E90244C0E90444C0E90A44CD
:10FF7000C0E90C44C0E90E44C0E91044C0E9124491
:10FF8000846104774462AA6D394630460123BDE896
:10FF9000F04100F003B800BF38000020F0B518B9F8
:10FFA000106808B9F0BD204604460F4614F8015BFE
:10FFB00017F8016B1EB96DB915602846F2E7B54216
:10FFC000F6D1002BEFD114600370EBE72B460DE068
:10FFD00026B91C4623460F4613F8015B17F8016B40
:10FFE000B542F5D1002DF1D0002121701360D9E781
:10FFF0002DE9F0478046894692461E460F463D460B
:020000021000EC
:10000000089815F8014BFEF730FF2044437813F0B1
:10001000080332D12D2C32D17C78BD1C0122002E58
:100020005DD0102E09D1302C07D12B7803F0DF03DF
:10003000582B4FD16C7810260235002A14BF4FF090
:1000400000416FF000410027B1FBF6FC384606FB8B
:100050001C1EA4F13003092B17D81C46A64223DD31
:100060007B1C07D084451CD301D1A64519DB00FBBE
:100070000640012715F8014BEBE72F46BFE72B2C75
:1000800004BFBD1C7C781A46C9E7A4F14103192BB3
:1000900001D8373CE2E7A4F16103192B04D8573C9F
:1000A000DCE74FF0FF37E5E77B1C08D12223C8F8D7
:1000B00000300846BAF1000F07D1BDE8F08702B161
:1000C0004042BAF1000FF8D00FB105F1FF39CAF87C
:1000D0000090F2E73024002EAFD10826ADE7302C97
:1000E000A3D00A26A9E7000037B5064C064D2468C0
:1000F000246A002C08BF2C460094FFF779FF03B058
:1001000030BD00BF380000209C000020084B37B5F0
:100110001C68084D236A002B08BF2B46009313462A
:100120000A4601462046FFF763FF03B030BD00BF1B
:10013000380000209C0000202DE9F04780468946C9
:1001400092461E460F463D46089815F8014BFEF7AD
:100150008CFE2044437813F0080330D12D2C30D18D
:100160007C78BD1C0121002E5CD0102E09D1302CD2
:1001700007D12B7803F0DF03582B4ED16C78102673
:1001800002354FF0FF320023B2FBF6F206FB02FC11
:100190006FEA0C0C1846A4F13007092F17D83C461B
:1001A000A64223DD002B1EDB82421CD301D1A445D5
:1001B00019DB00FB0640012315F8014BEBE72F4646
:1001C000C1E72B2C04BFBD1C7C781946CBE7A4F1FA
:1001D0004107192F01D8373CE2E7A4F16107192F35
:1001E00004D8573CDCE74FF0FF33E5E7002B09DA92
:1001F0002223C8F800304FF0FF30BAF1000F07D1CA
:10020000BDE8F08701B14042BAF1000FF8D00BB160
:1002100005F1FF39CAF80090F2E73024002EB0D182
:100220000826AEE7302CA4D00A26AAE737B5064C3C
:10023000064D2468246A002C08BF2C460094FFF762
:100240007BFF03B030BD00BF380000209C000020C1
:10025000024B01461868FFF7F9BC00BF38000020C8
:1002600010B50446FEF704FE2044437803F0030370
:10027000022B08BF203C204610BD0000F0B51D4BEE
:100280008BB005460C466E4603F1200C1868596881
:10029000374603C7083363453E46F7D118681B79D4
:1002A0003B71931E222B38604FF0000304D923705A
:1002B0001C4620460BB0F0BD661EB5FBF2F00AAF3F
:1002C00002FB10553D44591C15F8285C06F8015FE7
:1002D000054668B9605423442246191B101B81420D
:1002E000E7DD1178187802F8010B03F80119F4E73B
:1002F0000B46E2E7693B0100F8B50E461446054699
:1003000018B183690BB9FEF7CDFC214B9C422AD171
:100310006C68A369A360A3891A072ED5236963B308
:1003200023692068C01A6369F6B28342374604DC49
:1003300021462846FEF73AFC28BBA368013BA36090
:1003400023685A1C22601E7063690130834204D006
:10035000A389DB0719D50A2E17D121462846FEF7B7
:1003600025FC90B10FE00B4B9C4201D1AC68D0E76B
:10037000094B9C4208BFEC68CBE72146284600F0B9
:100380002DF80028CCD04FF0FF373846F8BD00BF1D
:10039000E43A0100043B0100C43A010049B1FF2ADC
:1003A00085BF8A2303600A704FF0FF3098BF012099
:1003B000704708467047000038B5074C05460846A8
:1003C0001146002222601A4602F048F8431C02D16E
:1003D000236803B12B6038BD50080020324B70B544
:1003E0001D6806460C4625B1AB6913B92846FEF7D1
:1003F00059FC2E4B9C420FD16C68B4F90C309AB268
:1004000015072CD4D00611D40922326043F04003E2
:10041000A3814FF0FF303EE0254B9C4201D1AC68F8
:10042000EBE7244B9C4208BFEC68E6E7510712D586
:10043000616B41B104F14403994202D03046FEF7AA
:1004400083FD00236363A38923F02403A381002396
:10045000636023692360A38943F00803A3812369B0
:100460004BB9A38903F42073B3F5007F03D0214671
:10047000304600F0C7FEA28912F001030CD0002321
:10048000A36063695B42A361236953B9B4F90C307B
:1004900013F08000BAD170BD920758BF6369A360A2
:1004A000F2E70020F7E700BF38000020E43A01003F
:1004B000043B0100C43A010008B5062001F008FF22
:1004C000012001F0D3FF000038B5064C002305469B
:1004D0000846236001F07CFF431C02D1236803B16E
:1004E0002B6038BD500800202DE9F74F03690C69D7
:1004F000A3428046C0F28280013C01F114074FEA1A
:10050000840C00F1140657F8245056F8240006EB2A
:100510000C03013507EB0C090193B0FBF5F595B31E
:100520004FF0000A3846B646D34650F8042B93B233
:1005300005FB03A34FEA134A9BB2ABEB0303120C78
:10054000DEF800B005FB02A213FA8BF34FEA124A61
:100550001FFA82FBDEF80020CBEB124202EB2342B3
:100560009BB243EA024381454FEA224B4EF8043BDB
:10057000DBD256F80C3033B9019B043B9E421A463D
:1005800030D3C8F81040404601F0EAF8002825DBD7
:10059000013530464FF0000C57F8042BD0F800E03E
:1005A00093B2ACEB0303120C13FA8EF3C2EB1E42B0
:1005B00002EB23429BB243EA0243B9454FEA224C85
:1005C00040F8043BE8D256F8242006EB84032AB90D
:1005D000043B9E421A460BD3C8F81040284603B08D
:1005E000BDE8F08F1268043B002ACAD1013CC5E780
:1005F0001268043B002AEFD1013CEAE70020EEE755
:100600002DE9F04F456A97B016461F460446DDF8BF
:100610008C80CDE902673DB91020FEF737FC60629F
:10062000C0E901550560C560636A196851B15A682F
:100630004A60012393408B60204600F0AFFE636A5E
:1006400000221A603B1EBBBF23F00043039300232C
:100650000122ACBFC8F80030C8F80020B24BDDF86A
:100660000C8033EA08031BD1229A42F20F73136005
:10067000029B23B9C8F31300002800F04F85249B88
:1006800053B9AA4B21E0AA4B05930833249A13606F
:10069000059817B0BDE8F08FA44B05930333F5E739
:1006A000DDE902670022002330463946FEF7CEF826
:1006B000824660B1229A01231360249B002B00F034
:1006C0002A859C4B249A1360013B0593E0E714AB09
:1006D000019315AB009332463B46204601F0B7F834
:1006E000C8F30A558346002D7CD0C7F3130343F0AB
:1006F0007F59B04649F44019A5F2FF35CDF84CA01A
:1007000000228D4B40464946FDF780FC80A3D3E98B
:100710000023FDF733FE80A3D3E90023FDF778FC27
:10072000064628460F46FDF7BFFD7DA3D3E900230B
:10073000FDF724FE02460B4630463946FDF768FCBD
:1007400006460F46FEF7CAF80022824600233046CE
:100750003946FEF785F848B15046FDF7A5FD32460B
:100760003B46FEF773F808B90AF1FF3ABAF1160FE3
:1007700059D8724901EBCA01DDE90223D1E9000130
:10078000FEF78CF8002850D00AF1FF3A00231293AC
:10079000149B5D1BB5F1010849BFC5F1010300239E
:1007A00008934FF0000858BF0893BAF1000F3EDBE2
:1007B0000023D044CDF834A00993209B092B00F2EC
:1007C0009080052BC4BF043B2093209BA3F1020320
:1007D000CCBF00250125032B00F28F80DFE803F05A
:1007E0007D7F3171DDE914531D4405F2324020282C
:1007F00013DDC0F14000029B08FA00F805F2124038
:1008000023FA00F048EA0000FDF73EFD0123804690
:10081000A1F1F879013D139372E7029BC0F120002A
:1008200003FA00F0F0E70123B1E71290B0E7089B6C
:10083000A3EB0A030893CAF10003099300230D9365
:10084000BBE701230C93219B002B59DD06939946AE
:10085000666A00227260042202F1140098427168F4
:1008600070D9204600F066FD636A30601B6805930E
:10087000B9F10E0F00F2EB80002D00F0E8809DED45
:10088000027BBAF1000F8DED107B79DD2B4A0AF067
:100890000F0302EBC30393ED007B4FEA2A16F00629
:1008A0008DED0A7B6AD5264BDDE91001D3E90823DB
:1008B000FDF78EFECDE9020106F00F060325204F5D
:1008C00051E001230C93219B534403F1010906934A
:1008D0004B46012BB8BF0123BAE70023B2E7002340
:1008E000F0E70125002320930C954FF0FF3306938A
:1008F0009946002212232192AAE701230C93F4E7E0
:100900000123069399461A46F5E700BFAFF300802E
:1009100061436F63A787D23FB3C8608B288AC63F05
:10092000FB799F501344D33F0000F07F983C0100B7
:100930008F3C01006D3801000000F83FC83C010009
:10094000A03C010001317160520085E7F10708D534
:10095000DDE90A01D7E90023FDF710FDCDE90A0121
:10096000013576100837002EF0D1DDE90A23DDE9E4
:100970000201FDF72DFECDE902011AE002259EE7F6
:1009800000F0A080CAF100069F4BA04F06F00F02B6
:1009900003EBC203D3E90023DDE91001FDF7EEFC10
:1009A000CDE90201361100230225002E7FD1002B54
:1009B000E1D1129B002B00F08780DDE90267002265
:1009C000934B30463946FDF74BFF00287CD0B9F1F8
:1009D000000F79D0069B002B35DD0AF1FF330A9317
:1009E000394600228B4B3046FDF7C8FCCDE90201A9
:1009F000069F01352846FDF757FCDDE90223FDF788
:100A0000BDFC0022844BFDF703FB0546A1F15076A7
:100A1000002F5DD10022814BDDE90201FDF7F6FADE
:100A20002A463346CDE90201FDF738FF002840F0A1
:100A300088822A4606F10043DDE90201FDF710FF36
:100A4000002840F07C82DDE91023CDE90223159BCC
:100A5000002BC0F25081BAF10E0F00F34C816A4BAB
:100A600003EBCA0393ED007B219B002B8DED067BEE
:100A700080F2D880B9F1000F00F3D48040F05E829C
:100A80000022664B51EC170BFDF778FCDDE90223E1
:100A9000FDF7FAFE4F464E46002840F03482059B93
:100AA000059A5D1C312313700AF1010A2FE2F20747
:100AB00005D5D7E90023FDF761FC01350123761048
:100AC000083772E7022574E7CDF828A04F4691E772
:100AD0004D4B03EBC70353E902010C9B002B47D09E
:100AE00002460B4600204E49FDF772FD2A4633466A
:100AF000FDF78CFACDE90E01059DDDE90201FDF758
:100B0000EDFE0646FDF7D0FB02460B46DDE902018D
:100B1000FDF77CFA303605F8016BDDE90E23CDE9EF
:100B20000201FDF79DFE002863D1DDE902230020CC
:100B30003749FDF76BFADDE90E23FDF791FE00283A
:100B400040F0B780059BEB1A9F427FF77CAF0022F5
:100B5000304BDDE90E01FDF711FC0022CDE90E015D
:100B60002C4BDDE90201FDF709FCCDE90201C4E7E8
:100B700033462A46FDF702FC059BCDE90E01DD193F
:100B80001E46DDE90201FDF7A9FE0746FDF78CFBD5
:100B9000303702460B46DDE90201FDF737FA06F869
:100BA000017BAE42CDE902014FF0000226D11C4B81
:100BB000DDE90E01FDF72CFA02460B46DDE90201E4
:100BC000FDF76CFE002874D1DDE90E2300201449E6
:100BD000FDF71CFA02460B46DDE90201FDF740FE77
:100BE00000283FF430AF15F8013C302B05F1FF32FF
:100BF00002D0DDF828A04AE01546F4E7054BFDF7E2
:100C0000BDFBCDE90201BCE7C83C0100A03C0100EE
:100C10000000F03F0000244000001C400000144091
:100C20000000E03FDDE90267059DDDE9062330466F
:100C30003946FDF7CDFCFDF751FE8046FDF734FB4C
:100C4000DDE90623FDF79AFB02460B46304639469E
:100C500008F13006FDF7DAF905F8016B059EAE1BC9
:100C6000B14502460B4639D1FDF7D2F9DDE906233D
:100C700006460F46FDF712FEC8B9DDE906233046E9
:100C80003946FDF7E3FD10B118F0010F0FD15946B9
:100C9000204600F083FB0023229A2B700AF1010307
:100CA0001360249B002B3FF4F3AC1D60F0E4CDF8FF
:100CB00028A015F8012C392A05F1FF3308D1059A2F
:100CC0009A4209D10A9B01330A93302313701346C9
:100CD0001A7801321A708CE71D46EAE700229B4B16
:100CE000FDF74CFB0022002306460F46FDF7AEFD44
:100CF00000289AD0CBE70C9A002A00F08B80209A2B
:100D0000012A6EDC139A002A67D003F23343DDE92F
:100D10000857089A01211A4420460892984400F086
:100D2000DDFB0646002D0CDDB8F1000F09DD454561
:100D3000089A2B46A8BF4346D21A0892ED1AA8EB90
:100D40000308099BEBB10C9B002B67D08FB1314698
:100D50003A46204600F062FC5A46014606462046C6
:100D600000F0C5FB59460A90204600F017FB0A9B8D
:100D70009B46099BDA1B04D05946204600F04EFCE6
:100D800083460121204600F0A9FB0D9B0746002B5E
:100D900000F0CB811A460146204600F03FFC209B24
:100DA000012B074640DC029B002B39D1039BC3F388
:100DB0001303002B36D1039B23F000431B0D1B05AF
:100DC0002BB1089B0133089308F101080123099313
:100DD0000D9B002B2AD1012030E0149BC3F1360378
:100DE00095E7099B09F1FF37BB42BFBF099B0997F4
:100DF000FA1A0D9BBBBF9B180D93DF1B0027B9F19F
:100E0000000FB5BF089B089DA3EB09054B46B8BF73
:100E100000237EE7DDE908570C9E83E7099AABE7DC
:100E20000023D4E7029BD2E7002309933B6907EB39
:100E30008303186900F004FBC0F12000404410F067
:100E40001F0047D0C0F12003042B3BDD089BC0F1FD
:100E50001C000344089305448044089B002B05DDD7
:100E600059461A46204600F027FC8346B8F1000F89
:100E700005DD39464246204600F01EFC0746129B1F
:100E800053B33946584600F06BFC002824DA00239F
:100E900059460A22204600F098FA0C9B0AF1FF3AC4
:100EA0008346002B00F04881002331460A22204669
:100EB00000F08BFA069B002B06464FDC209B022B92
:100EC0004CDD11E0C9D0089A1C331A4408921D4425
:100ED0009844C2E70346F6E7B9F1000F38DC209BDF
:100EE000022B35DDCDF81890069B63B939460522F3
:100EF000204600F06AFA01460746584600F030FCEA
:100F000000283FF7CCAD219B059D6FEA030A4FF007
:100F100000093946204600F041FA002E3FF4B7AEF2
:100F2000B9F1000F05D0B14503D04946204600F085
:100F300035FA3146204600F031FAA8E600273E4651
:100F4000E1E7DDF828A03E46A9E500BF0000244007
:100F50000C9BCDF81890002B00F0F580002D05DDDE
:100F600031462A46204600F0A7FB0646099B002B87
:100F70004CD07168204600F0DDF932690232054636
:100F8000920006F10C010C30FDF7B1FF0122294659
:100F9000204600F091FB059B0893029B03F00103A0
:100FA000B1460993064639465846FFF79DFA494629
:100FB000054600F13008584600F0D2FB3246029058
:100FC0003946204600F0E6FBC368024603BB0146F3
:100FD0000A90584600F0C4FB0A9A03461146204680
:100FE0000A9300F0DBF90A9BA3B9209A92B9099AF7
:100FF00082B9B8F1390F29D0029B002B01DD05F130
:101000003108089B5D1C83F8008082E73046C2E708
:101010000123E3E7029A002A04DB24D1209A12BBC1
:10102000099A02BB002BECDD59460122204600F054
:1010300043FB3946834600F093FB002803DCE0D1F4
:1010400018F0010FDDD0B8F1390FD8D1089B089AFC
:101050005D1C3923137015F8013C392B05F1FF3263
:101060004ED0013353E0089A002B02F1010506DD52
:10107000B8F1390FEAD008F10108089BC3E7059BD6
:10108000069A05F8018CEB1A934221D059460023A9
:101090000A22204600F099F9B14583464FF000033B
:1010A0004FF00A024946204605D100F08EF98146EC
:1010B0000646089577E700F088F931468146002317
:1010C0000A22204600F081F90646F2E74FF00009B7
:1010D00059460122204600F0EFFA3946834600F0D7
:1010E0003FFB0028B7DC02D118F0010FB3D115F88F
:1010F000013C302B05F1FF327FF40BAF1546F6E7CC
:10110000059B934205D1059A0AF1010A3123137018
:10111000FFE615469FE7174BFFF7D7BA249B002B36
:101120007FF4B1AA144BFFF7D0BA209B012B7FF7B5
:101130003AAE0D9B09934EE6069B002B03DC209BE9
:10114000022B3FF7D1AE059D39465846FFF7CCF943
:1011500000F1300805F8018B059B069AEB1A9A42BC
:10116000B4DD594600230A22204600F02EF98346BA
:10117000EAE700BF6C3801008F3C0100044B1B689C
:10118000186A044B002808BF1846F030704700BFAB
:10119000380000209C00002038B5074C0546084662
:1011A0001146002222601A4601F03AF9431C02D18E
:1011B000236803B12B6038BD5008002070B50E467F
:1011C000B1F90E10002996B014461D4607DA002327
:1011D0002B60B3891A0610D44FF480630EE06A4680
:1011E00001F0CCF80028F2DB019A02F47042A2F57B
:1011F00000535A425A412A60EEE740230020236000
:1012000016B070BD8B8973B59D0706460C4607D591
:1012100004F14703236023610123636102B070BDC1
:1012200001AB6A46FFF7CAFF009905463046FDF755
:10123000D9FE48B9B4F90C309A05EFD423F0030372
:1012400043F00203A381E3E70D4BB362A38920605F
:1012500043F08003A381009B6361019B20615BB12C
:10126000B4F90E10304601F09BF828B1A38923F0A1
:10127000030343F00103A381A3891D43A581CDE7A7
:101280006DEC000000000000000000000000000005
:1012900001F0FF01102A2BDB10F0070F08D010F827
:1012A000013B013A8B422DD010F0070F42B3F6D12B
:1012B000F0B441EA012141EA014122F007047FF044
:1012C00000070023F0E80256083C85EA010586EA9B
:1012D000010685FA47F5A3FA87F586FA47F6A5FAD7
:1012E00087F68EB9EED1F0BC01F0FF0102F00702E3
:1012F00032B110F8013B013A83EA010313B1F8D18E
:101300000020704701387047002D06BF354603386E
:10131000073815F0010F07D1013015F4807F02BFA7
:10132000013015F4C03F0130F0BC0138704700BFF8
:101330007047704770B5456A04460E463DB91020A7
:10134000FDF7A4FD6062C0E901550560C560656AEE
:10135000EB6883B1636ADB6853F82600B8B90121F2
:1013600001FA06F56A1D9200204600F0BFFA60B14E
:10137000C0E901650EE021220421204600F0B6FA02
:10138000636AE860DB68002BE4D1002070BD02686E
:1013900043F826200023C0E90333F7E770B5446A19
:1013A00006460D463CB91020FDF770FD7062C0E99D
:1013B00001440460C4603DB1736A6A68DB6853F835
:1013C0002210296043F8225070BD2DE9F0410D69CB
:1013D0001F4606460C4601F1140C0023DCF8000001
:1013E00081B202FB01710F0C000C02FB007089B28C
:1013F000013301EB00419D424FEA10474CF8041BBA
:10140000ECDCD7B1A368AB4212DC61683046013135
:10141000FFF790FF2269023204F10C01804692002E
:101420000C30FDF764FD21463046FFF7B7FF444618
:1014300004EB850301355F6125612046BDE8F0813D
:10144000020C12040346B2B90304102013F07F4FBC
:1014500004BF1B02083013F0704F04BF1B0104309F
:1014600013F0404F04BF9B000230002B06DB5B00F3
:1014700003D5013070470020E8E72020704703685B
:1014800013F0070201460BD0DA0723D4980749BFAF
:101490005B089B0801200B605CBF0B60022070475B
:1014A00098B2A8B91B0C102013F0FF0F04BF1B0A41
:1014B00008301A0704BF1B0904309A0704BF9B08B1
:1014C0000230DA0702D45B0806D001300B607047A7
:1014D0001046E9E7002070472020704710B50C4601
:1014E0000121FFF727FF01224461026110BD2DE9B0
:1014F000F74F14460A6923699A42B8BF0B468846DB
:10150000BCBFA0461C46D8F81070D4F81090D8F88C
:101510000830D8F8041007EB0906B342B8BF013110
:10152000FFF708FF00F1140505EB860E2B4600229D
:10153000734516D304F1140208F1140102EB890378
:1015400001EB87070093009B019293420CD8002E79
:1015500003DD5EF8043D002B5DD0066103B0BDE8FD
:10156000F08F43F8042BE3E7B2F800B0BBF1000FB3
:1015700023D08946AC464FF0000859F8044BDCF8FC
:1015800000A0A3B21FFA8AFA0BFB03A34FEA144A86
:10159000DCF8004043444FEA14480BFB0A8404EB98
:1015A0001344E2469BB243EA04434F454FEA1448D2
:1015B0004AF8043B2BD8CCF80480019BB3F802A076
:1015C0000432BAF1000F20D02B688946A8464FF0AC
:1015D000000BB9F800C0B8F802400AFB0C445C44A8
:1015E000C4469BB243EA04434CF8043B59F8043B1D
:1015F000B8F804B01B0C0AFB03B303EB14434F45CC
:101600004FEA134B05D8C8F8043004359BE7D4469D
:10161000B3E7E046DDE7013E99E700002DE9F84336
:10162000154612F0030206460F4607D0013A214C38
:10163000002354F82220FFF7C8FE0746AD1035D02E
:10164000746A3CB91020FDF721FC7062C0E90144C6
:101650000460C460D6F82480D8F808404CB940F241
:1016600071213046FFF73AFF0023C8F8080004460E
:1016700003604FF00008EB070AD539462246304692
:10168000FFF735FF394681463046FFF787FE4F4664
:101690006D100BD0206838B9224621463046FFF73E
:1016A00026FF2060C0F800800446E4E73846BDE825
:1016B000F88300BF903D01002DE9F0470C464FEA4A
:1016C000621A236949680AEB0309A36807461646AC
:1016D00009F10105AB4232DB3846FFF72BFE002350
:1016E000804600F114011A4653452BDB20692AEA93
:1016F000EA7A04F1140316F01F0201EB8A0103EBEE
:10170000800C25D0C2F1200E00201E688A4696402B
:1017100030434AF8040B53F8040B9C4520FA0EF0B2
:1017200014D8486008B109F10205013D3846C8F8EF
:1017300010502146FFF732FE4046BDE8F0870131E8
:101740005B00C7E741F823200133CDE75146DCE7D2
:10175000043953F8042B41F8042F9C45F9D8E4E7E9
:1017600003690A699B1A30B50CD192001430143108
:101770008418114454F8045D51F8042D954203D0A7
:1017800005D30123184630BDA042F3D3FAE74FF04A
:10179000FF33F7E72DE9F0470D4607461146284687
:1017A0001446FFF7DDFF061E08D131463846FFF725
:1017B000C1FD0123C0E90436BDE8F087A4BF23467C
:1017C0002C4638466168A6BF1D4600260126FFF755
:1017D000B1FD2B69C660266905F1140904F11402F4
:1017E00002EB860709EB830800F114054FF0000EA9
:1017F00052F804AB59F8044B1EFA8AF1A3B2C91A85
:10180000230CC3EB1A4303EB214389B24FEA234E67
:10181000C84541EA0343944645F8043BE8D8BC4533
:1018200004D355F8043D83B10661C5E75CF8041B99
:101830001EFA81F31A1402EB11429BB243EA0243EF
:101840004FEA224E45F8043BE9E7013EE9E72DE97E
:10185000F743012199469046DDE90A65FFF76AFDE5
:10186000C9F30A540746C9F3130334BBB8F10002A5
:10187000019327D002A840F8082DFFF700FE009939
:10188000F0B1019AC0F1200302FA03F30B43C24006
:101890007B610192019BBB61002B14BF02210121DE
:1018A0003961C4B1A4F2334404443460C0F135005A
:1018B0002860384603B0BDE8F08343F48013D5E7D1
:1018C0007961E7E701A8FFF7DAFD019B7B61012160
:1018D00039612030E5E707EB8103A0F23240306048
:1018E0001869FFF7ADFDC0EB4110E1E738B502FB29
:1018F00001F42146FDF776FB054618B1224600218A
:10190000FDF719FB284638BDF8B5074614460E46C4
:1019100021B91146BDE8F840FDF764BB22B9FDF7D7
:1019200013FB25462846F8BD00F04AFDA0420FD221
:1019300021463846FDF756FB05460028F2D03146D1
:101940002246FDF7D4FA31463846FDF7FDFAE9E7BD
:101950003546E7E72DE9F0478E689E4282460C4601
:101960009046994637D88A8912F4906F31D025680D
:1019700009696F1A6569022305EB450595FBF3F5C7
:1019800009F101033B449D4238BF1D46530530D544
:101990002946FDF727FB064650B90C23CAF800304C
:1019A000A38943F04003A3814FF0FF30BDE8F087E7
:1019B0003A462169FDF79BFAA38923F4906343F02B
:1019C0008003A381266165613E44ED1B2660A5600E
:1019D0004E464E4500D94E46324641462068FDF7F8
:1019E00091FAA3689B1BA36023681E442660002015
:1019F000DCE72A46FFF788FF06460028E2D1216986
:101A00005046FDF7A1FAC8E72DE9F04F9DB080469A
:101A100003938B891D060C4616460FD50B696BB9CF
:101A20004021FDF7DFFA2060206128B90C23C8F8B7
:101A300000304FF0FF30C7E040236361002309937B
:101A400020238DF8293030238DF82A304FF0010BF8
:101A500037463D4615F8013B0BB1252B3ED1B7EB80
:101A6000060A0BD05346324621464046FFF772FF26
:101A7000013000F0A480099B534409933B78002B6C
:101A800000F09D8000234FF0FF32CDE90523049341
:101A900007938DF853301A932F46052217F8011B30
:101AA0004F48FFF7F5FB049BD0B9D90644BF20226D
:101AB0008DF853201A0744BF2B228DF853202A7823
:101AC0002A2A15D0079A2F4600200A25394611F8F0
:101AD000013B303B092B4DD9B8B10FE02F46B8E799
:101AE0003F4A801A0BFA00F0184304903D46D3E7B2
:101AF000039A111D12680391002A01DB079204E08A
:101B0000524243F00203079204933B782E2B0CD1F0
:101B10007B782A2B33D1039B1A1D1B680392002B61
:101B2000B8BF4FF0FF33023705932E4D39780322AB
:101B30002846FFF7ADFB38B14023401B03FA00F005
:101B4000049B034301370493397827488DF8281004
:101B500006227E1CFFF79CFB002838D0234B13BBCA
:101B6000039B073323F0070308330393099B4B447C
:101B700009936DE705FB023201200F46A6E700231B
:101B80000137059319460A25384610F8012B303ADB
:101B9000092A03D9002BC8D00591C6E705FB01210E
:101BA00001230746F0E703AB00932246104B04A93C
:101BB0004046FDF741FCB0F1FF3F8146D6D1A389F5
:101BC0005B063FF536AF09981DB0BDE8F08F03AB5B
:101BD00000932246064B04A94046FDF7E9FEEAE7DA
:101BE0002E3B0100343B0100383B010039F400007A
:101BF0005519010038B54B1C144603D14FF0FF3581
:101C0000284638BD938923F020039381636B526883
